:020000040800F2
:1000000008E7012061020008372900082F290008AD
:100010003329000899070008C92E000800000000D5
:10002000000000000000000000000000A101000826
:100030009D07000800000000FD01000839290008A4
:100040008502000885020008850200088502000874
:100050008502000885020008850200088502000864
:100060008502000885020008850200088502000854
:100070008502000885020008850200088502000844
:100080008502000885020008850200088502000834
:100090008502000885020008850200088502000824
:1000A0008502000885020008850200088502000814
:1000B0008502000885020008612900088502000801
:1000C00085020008850200088502000885020008F4
:1000D00085020008792E00088502000885020008C4
:1000E00085020008850200088502000885020008D4
:1000F00085020008850200088502000885020008C4
:1001000085020008850200088502000885020008B3
:1001100085020008850200088502000885020008A3
:100120008502000885020008850200088502000893
:1001300085020008590800088502000885020008A9
:100140008502000885020008850200088502000873
:100150008502000885020008850200088502000863
:100160008502000885020008850200088502000853
:1001700085020008850200088502000800000000D2
:100180008502000885020008DFF810D000F06AFA46
:10019000004800471DD20008AFF3008008E70120A7
:1001A0002C4B19680868B0E8F04F80F30988BFF35A
:1001B0006F8F4FF0000080F311887047000000003F
:1001C00008480068006880F308884FF0000080F35A
:1001D000148862B661B6BFF34F8FBFF36F8F00DF35
:1001E00000BF00BF08ED00E0DFF80C00016841F43B
:1001F00070010160704700BF88ED00E0EFF30980F7
:10020000BFF36F8F134B1A681EF0100F08BF20ED5D
:10021000108A20E9F04F106009B44FF0500080F3CD
:100220001188BFF34F8FBFF36F8F19F0A7F94FF00D
:10023000000080F3118809BC19680868B0E8F04F25
:100240001EF0100F08BFB0EC108A80F30988BFF3CE
:100250006F8F7047AC020020EFF3058070470000FD
:100260000948016841F47001016008488047084866
:100270000047FEE7FEE7FEE7FEE7FEE7FEE7FEE7F4
:10028000FEE7FEE7FEE7000088ED00E04D290008EC
:10029000890100082DE9F05F0546002092469B4643
:1002A00088460646814640241BE02846414647468C
:1002B000224600F031F953465A46C01A914110D3F4
:1002C00011461846224600F018F92D1A67EB01086E
:1002D0004F4622460120002100F00FF917EB0009DC
:1002E0004E41201EA4F10104DFDC484631462A4677
:1002F0004346BDE8F09F000000487047ECDB010872
:100300000649074A0868504343F23902104408601E
:100310004008704701490860704700002C03002026
:100320006D4EC64110B5431A934209D283188818FE
:1003300003E010F8011D03F8011D521EF9D210BD93
:1003400040EA01039B0703D009E008C9121F08C057
:10035000042AFAD203E011F8013B00F8013B521ED7
:10036000F9D210BDD2B201E000F8012B491EFBD238
:1003700070470022F6E710B513460A4604461946B0
:10038000FFF7F0FF204610BD421C10F8011B0029AA
:10039000FBD1801A704730B504460020034600E0C8
:1003A0005B1C934203D2E05CCD5C401BF8D030BDB7
:1003B00070B5064602F0CAFD046805460A2200210F
:1003C000304600F0B9F82C6070BD2DE9FE4F81EA8F
:1003D000030404F0004421F0004100944FF0000BAE
:1003E00023F0004350EA01045ED052EA03045BD0DC
:1003F000C3F30A54C1F30A552C44A4F2F334019414
:10040000A0FB0254C1F3130141F48011C3F31303A1
:1004100043F4801301FB024400FB034E840A970A55
:1004200044EA815447EA8357A4FB076802958D0A82
:1004300005FB07854FEA932C04FB0C542705029D0E
:100440004FEA065847EA1637B5EB08056EEB070C7E
:10045000870E920E47EA811742EA8312A7FB020138
:10046000B6EB0B0164EB00042B0D43EA0C335E1872
:1004700044EB1C50DA465146E7FB0201C5F3130476
:100480004FEA0B3343EA14534FEA0432019C43EA28
:100490000603A4F10C040294009CCDE900B400F022
:1004A00092F803B0BDE8F08F00200146F9E70EB5E1
:1004B00040F2334102910021CDE900110A460B467A
:1004C00000F081F803B000BDC1F30A5210B5C1F3CA
:1004D000130140F2FF3341F480119A4201DA002007
:1004E00010BD40F233439A42A2F2334203DC52423F
:1004F00000F012F810BD904010BD202A04DB203A15
:1005000000FA02F1002070479140C2F1200320FA66
:1005100003F3194390407047202A04DB203A21FA64
:1005200002F00021704721FA02F3D040C2F120020C
:1005300091400843194670472DE9F04791460F4610
:1005400080460446002614F8015B2DB1FFF7D4FE67
:100550000068405DC007F6D12B2D02D02D2D18D09C
:10056000641E4A463946204600F08EF827B13968A5
:10057000A14201D1C7F8008071054FF002040BD5EC
:100580004042002803DD02F0E1FC0460A007BDE862
:10059000F08746F48066E4E70028F8DA02F0D6FC3B
:1005A00004606FF00040F2E710B5141E73F1000410
:1005B00008DA401C41F1000192185B411A4301D155
:1005C00020F0010010BD2DE9F04D92469B4611B17F
:1005D000B1FA81F202E0B0FA80F220329046FFF7E1
:1005E0008CFF04460F4640EA0A0041EA0B015346DD
:1005F0005A46084313D0114653EA010019D0C8F1F6
:1006000040025046FFF788FF05460E4650465946C1
:100610004246FFF772FF084305D0012004E0204660
:100620003946BDE8F08D0020054346EAE0762C43CC
:1006300037430A986305E40AA0EB08000022FD0A8C
:1006400044EA47540A3002D500200146E9E7010593
:1006500010196941DDE9084500196941BDE8F04D0F
:10066000A2E70000064C074D06E0E06840F00103F9
:1006700094E8070098471034AC42F6D3FFF788FDA2
:100680002CE301084CE301082DE9F05F8246007875
:10069000002715468B460AF10104B946302801D0DF
:1006A0009DB113E014F8010B0127782803D05828D6
:1006B00001D045B10AE00DB1102D07D1002710255A
:1006C00014F8010B02E0082500E00A250026B046D8
:1006D0000EE005FB080005FB06F1012701EB1046C3
:1006E0001FFA80F8B6F5803F00D3B94614F8010B25
:1006F000294600F018F80028EBDABBF1000F05D00E
:100700000FB1641E00E05446CBF80040B9F1000F71
:1007100006D002F01BFC02210160C81EBDE8F09F5C
:1007200048EA0640FAE73A2800D2303820F02002A2
:10073000412A01D3A2F13700884201D34FF0FF30A4
:10074000704770B58C1810F8015B15F0070301D1E4
:1007500010F8013B2A1106D110F8012B03E010F824
:10076000016B01F8016B5B1EF9D12B0705D4002347
:10077000521E0DD401F8013BFAE710F8013BCB1AE9
:10078000921C03E013F8015B01F8015B521EF9D5DE
:10079000A142D8D3002070BD00BFFEE770470168BA
:1007A00001F58051896921F00202016801F580514B
:1007B0008A617047016801F58051896941F0020240
:1007C000016801F580518A617047016801F5805127
:1007D000896921F40052016801F580518A617047EE
:1007E000016801F58051896941F40052016801F501
:1007F00080518A617047000008B508490968C90836
:100800004FF47A72B1FBF2F14143009100BF00BF97
:1008100000994A1E00920029F9D108BD000000206D
:1008200038B5044600200090206800F580508069AB
:1008300040F48011206800F580508161206800F547
:100840008050806900900120FFF7D6FF0099206852
:1008500000F58050816138BD10B50A49886A05F0FD
:1008600001FC08B10BF026FD4FF48031054800680B
:1008700000F58050416140210248006800F5805039
:10088000416110BDF004002030B50346147955795C
:1008900044EA0520084C0C442064D478240695785A
:1008A00044EA0544557844EA0524157844EA0500ED
:1008B000014C0C44606430BD0080024070B5AEB0A5
:1008C00004460E46002526B14FF40061E160C900E0
:1008D000A160002011901290139014901590169022
:1008E000E06918B94FF48060179001E0002017907C
:1008F0004FF400701890002019901A901B904FF040
:1009000000401C9000201D9040201E9000201F9051
:100910002090219010202290002023902490259058
:100920002690802027900020289029902A902B90B4
:100930002C902D902068056870480540DDE9110174
:1009400008431399084314990843A168084315996B
:10095000084316990843E168084317990843189912
:100960000843199908431A9908431B9908430543FA
:100970002068056020680568012000F0F3F9206810
:100980000560DDE91C0108431E9908431F990843CF
:100990002099084321990843229908432399084341
:1009A0002168486020684568012000F0DBF9206874
:1009B000456024982168886025982168C86020686F
:1009C00085694FF641700540DDE9261040EA014097
:1009D00028990843299908432A9908432B990843E1
:1009E00005432068856120688569012000F0BAF917
:1009F00020688561DDE92C0108432168C861206811
:100A0000C569012000F0AEF92068C56100200190A1
:100A10004FF000700290002003904FF400100490FB
:100A20000020059006900790089004200990C005CA
:100A30000A9040120B9080010C9040120D90802083
:100A40000E9000200F901090206800F5805085696E
:100A50002B480540DDE90101084303990843049947
:100A600008430599084306990843079908430899DC
:100A70000843099908430543206800F580508561C3
:100A8000206800F580508569012000F06BF920682E
:100A900000F580508561DDE90A0108430C9908439F
:100AA0000D9908430E9908430F9940EA8100109967
:100AB000084340F40001206800F580500160206880
:100AC00000F580500568012000F04CF9206800F521
:100AD00080500560A069012809D1206800F5805088
:100AE000C06908490843216801F58051C8610021A7
:100AF00020466269FFF7C8FE2EB070BD0F8120FF4F
:100B0000233FDEF84000010038B504460020009085
:100B10002068006820F004002168086020680068F0
:100B200000900120FFF768FE00982168086038BD3A
:100B300038B50446002000902068006840F00400AA
:100B4000216808602068006800900120FFF754FECB
:100B500000982168086038BD38B504460020009030
:100B60002068006820F0080021680860206800689C
:100B700000900120FFF740FE00982168086038BD12
:100B800038B50446002000902068006840F0080056
:100B9000216808602068006800900120FFF72CFEA3
:100BA00000982168086038BD70B504461D460023D2
:100BB000B5F5804F13D154F822300C480340D1E9E9
:100BC000000640EA06108E6840EA06208E8940EA58
:100BD00006408E693043034344F8223003E06FF04F
:100BE000704044F82200002070BD00000000F0CFEB
:100BF00010B503460022086853F82020124802402E
:100C0000D1E901042043CC6820430C6920434C699E
:100C100020438C692043CC6920430C6A20434C6AF2
:100C200020438C6A2043CC6A2043CC6B20430C6B5E
:100C3000204302438868082801D142F04002086836
:100C400043F82020002010BD8000F0FF30B503469F
:100C50000024501C53F8204004F04044D1E9000522
:100C600040EA05108D6840EA05208D8940EA054577
:100C7000088A401E45EA0055087D801E45EA00604E
:100C80008D6928430443501C43F82040002030BDA8
:100C900070B50446A56D00F093FE064694F8350045
:100CA000022808D08020606500BF002084F834004E
:100CB00000BF012070BD2068006820F01600216888
:100CC00008602068406920F0800021684861206C3D
:100CD00008B9A06C28B12068006820F008002168DD
:100CE00008602068006820F00100216808600FE0BB
:100CF00000F066FE801B05280AD92020606500BF31
:100D0000002084F8340000BF032084F83500D1E7C8
:100D10002068006800F001000028E9D194F85C1018
:100D20003F208840A86000BF002084F8340000BF46
:100D3000012084F835000020BCE7014691F8350019
:100D4000022803D08020486501207047052081F8E3
:100D500035000868006820F001000A681060002073
:100D6000F3E7000070B5044600F02AFE064625466B
:100D7000681C10B104480078054400BF00F020FE54
:100D8000801BA842FAD370BD2400002070B5044631
:100D90000D461646002200BF94F84500012801D1F7
:100DA000022070BD012084F8450000BF022084F8B5
:100DB0004400A56200221FE005EB42114FF0004005
:100DC000086044F2F4504860C2EBC21000EB4000EF
:100DD00006EB80008860A069012803D1486820F0F4
:100DE00000404860581E904204D905EB4210203064
:100DF000C86000E0CD60521C9A42DDD3206800F547
:100E00008050C560012084F8440000BF002084F8B1
:100E1000450000BF00BFC4E770B504460D46164646
:100E2000002200BF94F84500012801D1022070BDC6
:100E3000012084F8450000BF022084F84400E562E8
:100E400000221BE005EB42114FF480100860C2EB5A
:100E5000C21000EB400006EB80008860E06918B922
:100E6000086840F440000860581E904204D905EB21
:100E700042102030C86000E0CD60521C9A42E1D39D
:100E8000206800F580500561012084F8440000BF0F
:100E9000002084F8450000BF00BFC8E701460022DB
:100EA00000BF91F84500012801D1022070470120C0
:100EB00081F8450000BF022081F84400886A00687C
:100EC00000F00040002838D1886A006800F4807083
:100ED000F0B1886B401C8863886B012801D1886A57
:100EE00008638B6A4B63886A0068C0F30D40021F79
:100EF000CA63086B83680B64886AC06888620120D3
:100F000081F8440000BF002081F8450000BFCDE714
:100F1000886A006800F4007048B1886A086300239A
:100F20004B6301238B63886AC068886205E0886B25
:100F3000401C8863886AC0688862012081F8440088
:100F400000BF002081F8450000BF0120AEE700008F
:100F50002DE9FC4104460025002001909D4E00270C
:100F6000804614B90120BDE8FC8194F8440028B9FA
:100F7000002084F84500204600F03AF900BF002028
:100F800000909548006840F4804093490860084606
:100F9000006800F48040009000BF00BF8F480068E8
:100FA00020F400008D49086008460068216A084363
:100FB0008A490860206800F58050006840F001010F
:100FC000206800F58050016000F0FAFC07460FE051
:100FD00000F0F6FCC01BB0F5FA7F09D9032084F8B5
:100FE000440000BF002084F8450000BF0320BAE79A
:100FF000206800F58050006800F001000028E7D16B
:101000002068056925F01C0500F056FE0646744868
:10101000864205D37348864202D245F008051AE09D
:101020007048864205D36B48864202D245F00C05D3
:1010300011E06848864203D36B48864200D20AE03A
:101040006948864205D36948864202D245F00405C4
:1010500001E045F01005206805614FF400420021D1
:10106000204600F04DFB48B14FF0010841462046B4
:10107000FFF724FC012084F8440074E7FF20FFF709
:1010800071FE6068002871D000F09AFC074600BF2E
:1010900001AA0121204600F0F9F900F091FCC01BE3
:1010A00041F2883188420FD94FF00108414620466D
:1010B000FFF704FC012084F8440000BF002084F8FE
:1010C000450000BF03204EE7019800F0040004280B
:1010D000DED182020021204600F012FB48B14FF021
:1010E000010841462046FFF7E9FB012084F844004F
:1010F00039E700F065FC074600BF01AA0121204640
:1011000000F0C4F900F05CFCC01B41F28831884259
:101110000FD94FF0010841462046FFF7CFFB0120D1
:1011200084F8440000BF002084F8450000BF03207D
:1011300019E7019800F020002028DED101AA112132
:10114000204600F0A3F948B14FF00108414620467F
:10115000FFF7B4FB012084F8440004E7019800F491
:10116000005020B14FF40061E16002E00EE0002188
:10117000E16044F2100101980840884202D1002148
:10118000A1601EE04FF48041A1601AE0E068C0F366
:10119000CF00A168C1F34F0140EA010200212046BF
:1011A00000F0AEFA48B14FF0010841462046FFF783
:1011B00085FB012084F84400D5E640F6FF70FFF778
:1011C000D1FD41462046FFF779FB012084F8440019
:1011D0000020C8E6008793034438024004380140E9
:1011E000002D3101C00E160200E1F50580D1F00896
:1011F00010B586B0044600BF00BF002000909E4896
:10120000006840F001009C4908600846006800F052
:101210000100009000BF00BF00BF00BF00BF002062
:1012200000900846006840F0010008600846006829
:1012300000F00100009000BF00BF00BF00BF00BF72
:10124000002000900846006840F001000860084651
:10125000006800F00100009000BF00BF00BF00BFA9
:1012600000BF002000900846006840F004000860BD
:101270000846006800F00400009000BF00BF00BFF7
:1012800000BF00BF002000900846006840F0040046
:1012900008600846006800F00400009000BF00BF2E
:1012A00000BF00BF00BF002000900846006840F06B
:1012B000040008600846006800F00400009000BFC9
:1012C00000BF00BF00BF00BF0020009008460068BC
:1012D00040F0400008600846006800F040000090C0
:1012E00000BF00BF00BF00BF00BF00200090084645
:1012F000006840F0400008600846006800F04000C8
:10130000009000BF00BF00BF00BF00BF00200090E2
:101310000846006840F0400008600846006800F099
:101320004000009000BF00BF00BF00BF00BF002012
:1013300000900846006840F4807008600846006825
:1013400000F48070009000BF00BF00BF00BF00BF6E
:10135000002000900846006840F0007008600846D1
:10136000006800F00070009000BF00BF00BF0020C8
:1013700000900846006840F08060086008460068F9
:1013800000F08060009000BF00BF00BF0020009010
:101390000846006840F0006008600846006800F0F9
:1013A0000060009000BF00BF00BF022001900290CB
:1013B00000200390032004900B20059001A92F48E2
:1013C00000F0E6F90420019001A92C4800F0E0F9B2
:1013D0008020019001A9294800F0DAF9022001904B
:1013E00001A9274800F0D4F91020019001A9244850
:1013F00000F0CEF92020019001A9214800F0C8F9A1
:101400004FF40060019001A91E4800F0C1F94FF4AB
:101410000050019001A91B4800F0BAF94FF4804038
:10142000019001A9174800F0B3F9082001900120AC
:101430000290002003900320049001A9124800F0BC
:10144000A7F900BF002208210F4800F0ADFA00BF45
:10145000322002F039F800BF012208210A4800F0CA
:10146000A3FA00BF002206213D2000F010FB3D2022
:1014700000F0FDFA06B010BD303802400000024016
:101480000008024000180240000C02402DE9F04123
:1014900004460E4617460025A84694F844008228C4
:1014A00002D10220BDE8F081822084F84400206847
:1014B000056905F01C05208A4FF4784101EAC02037
:1014C0000543481100EA8610054325F0020545F062
:1014D00001052068056100F073FA804612E000F013
:1014E0006FFAA0EB0800B0F5803F09D3012084F823
:1014F000440000BF002084F8450000BF0320D1E76E
:101500002068056905F001000028E8D120684069DD
:1015100080B23860012084F844000020C2E710B592
:10152000044600BF94F84500012801D1022010BDF7
:10153000012084F8450000BF022084F844002046C2
:10154000FFF71EFB2046FFF7F3FA2046FFF768F986
:101550002046FFF745F92046FFF72CF9012084F8D3
:10156000440000BF002084F8450000BF00BFDEE754
:1015700010B5044600BF94F84500012801D10220AF
:1015800010BD012084F8450000BF022084F844000B
:101590002046FFF71AF92046FFF701F92046FFF72A
:1015A000B3FA2046FFF73CF92046FFF7D5FA0120B1
:1015B00084F8440000BF002084F8450000BF00BF4D
:1015C000DEE770B5024600230025002400BF92F834
:1015D0004500012801D1022070BD012082F845009C
:1015E00000BF022082F8440049B9012082F844007B
:1015F00000BF002082F8450000BF0120ECE7D06A60
:10160000006800F0004048B1122082F8440000BF9A
:10161000002082F8450000BF0120DDE740F2F450D1
:10162000814208D9B1FBF0F3B1FBF0F600FB1610D4
:1016300010B15B1C00E00123012B13D1D06A0068BC
:1016400040F04050D66A3060C1F30C00D66A70603A
:10165000D06A006840F00040D66A3060D06AC06846
:10166000D06232E000242EE0D06A006820F04050C2
:10167000D66A30602CB9D06A006840F08050D66AD3
:10168000306040F2F450D66A7060581EA04210D10B
:10169000D06A006840F00050D66A3060581EC0EB37
:1016A000C01000EB4000A1EB8005C5F30C00D66A2A
:1016B0007060D06A006840F00040D66A3060D06A3E
:1016C000C068D062641C9C42CED3106800F5805084
:1016D000406900F0040048B10426106800F580500D
:1016E00046610026106800F580504660012082F8AF
:1016F000440000BF002082F8450000BF00BF6BE738
:101700002DE9F04104460E4617460025A84694F8F8
:101710004400422802D10220BDE8F081422084F832
:1017200044002068056905F01C05208A4FF47841C3
:1017300001EAC0200543481100EA8610054345F040
:10174000020545F00105B8B22168486120680561CD
:1017500000F036F9804612E000F032F9A0EB080004
:10176000B0F5803F09D3012084F8440000BF002079
:1017700084F8450000BF0320CEE72068056905F026
:1017800001000028E8D1012084F844000020C3E7CC
:10179000F8B502460B460025002400200021DEE0BB
:1017A000012606FA01F51E6806EA0504AC4275D169
:1017B0001E7906F00306012E04D01E7906F00306FA
:1017C000022E13D190684F000326BE40B0434F0055
:1017D000DE68BE4030439060506801268E40B043C2
:1017E0001E79C6F300168E40304350601E7906F015
:1017F0000306032E09D0D0684F000326BE40B04335
:101800004F009E68BE403043D0601E7906F003064C
:10181000022E13D1CF0802F1200656F827004E07FA
:10182000F70E0F26BE40B0434F07FF0E1E69BE40A5
:101830003043CF0802F1200646F8270010684F0019
:101840000326BE40B0431E7906F003064F00BE409B
:10185000304310605E6806F08056B6F1805F7DD13F
:1018600000BF00260096404E366846F480463E4F44
:101870003E603E46366806F48046009600BF00BFD4
:101880003A4E8F0856F827008E07370F0F26BE40B6
:10189000B043374EB24202D1002624E05EE0354E1E
:1018A000B24201D101261EE0334EB24201D10226DE
:1018B00019E0324EB24201D1032614E0304EB2425A
:1018C00001D104260FE02F4EB24201D105260AE0D5
:1018D0002D4EB24201D1062605E02C4EB24201D176
:1018E000072600E008268F073F0FBE4030431F4EFB
:1018F0008F0846F82700264E3068A0435E6806F43D
:101900008036B6F5803F00D12043214E3060361D31
:101910003068A0435E6806F40036B6F5003F00D19B
:1019200020431B4E361D3060361D3068A0435E6874
:1019300006F48016B6F5801F00D12043144E0836F9
:101940003060361D3068A0435E6806F40016B6F5B8
:10195000001F00D120430E4E0C363060491C102968
:10196000FFF41EAFF8BD00004438024008380140C3
:10197000000002400004024000080240000C024047
:10198000001002400014024000180240001C0240F7
:10199000003C014010B5426921EA020302EA010459
:1019A00043EA0443836110BD0AB1816101E00B0485
:1019B0008361704701480068000C7047002004E014
:1019C00001480068704700001C00002003480068C0
:1019D0000349097808440149086070471C00002049
:1019E0002400002010B50D48006840F400700B4939
:1019F00008600846006840F4806008600846006897
:101A000040F480700860032000F080F80F2000F0A0
:101A100007F800F02BF8002010BD0000003C024049
:101A200070B504460E4800784FF47A71B1FBF0F0BF
:101A30000C490968B1FBF0F5284600F09BFC08B1A1
:101A4000012070BD102C07D200222146501E00F04C
:101A50001EF80548046001E00120F2E70020F0E7ED
:101A600024000020000000202000002070470146D4
:101A70000846002809DB00F01F0301229A404309B1
:101A80009B0003F1E023C3F8002100BF70472DE95C
:101A9000F05F80460D461646002701F03BFA0746E8
:101AA00039462A46334601F00700C0F1070ABAF169
:101AB000040F02D94FF0040A01E0C0F1070AD14631
:101AC00000F1040ABAF1070F02D24FF0000A01E058
:101AD000A0F1030AD4464FF0010A0AFA09FAAAF162
:101AE000010A0AEA020A0AFA0CFA4FF0010B0BFA91
:101AF0000CFBABF1010B0BEA030B4AEA0B0421468A
:101B0000404601F00FFABDE8F09F000000BF00F072
:101B10000702064B19684FF6FF031940044B0B43AD
:101B200043EA0221014B196000BF70470CED00E051
:101B30000000FA0570B504460D460CB9012070BDD1
:101B40005848006800F00700A84209D255490D70B6
:101B50000846006800F00700A84201D00120EEE727
:101B6000207800F0020002281DD1207800F0040047
:101B7000042805D14C48006840F4E0504A49086008
:101B8000207800F00800082805D14748006840F494
:101B90006040454908604448006820F0F000A168B2
:101BA000084341490860207800F00100A8B360684C
:101BB000012807D13C4808380068C0F34040B8B954
:101BC0000120BCE76068022802D06068032807D1C2
:101BD000354808380068C0F3406048B90120AEE7D6
:101BE000314808380068C0F3400008B90120A6E772
:101BF0002D48006820F00300616808432A49086006
:101C0000FFF7DEFE064609E0FFF7DAFE801B41F231
:101C10008831884202D9032091E707E02248006812
:101C200000F00C006168B0EB810FEDD11D48006839
:101C300000F00700A84209D91A490D70084600684B
:101C400000F00700A84201D0012078E7207800F0DA
:101C50000400042807D11448006820F4E050E1682B
:101C6000084311490860207800F00800082808D1CE
:101C70000D48006820F46040216940EAC1000A492B
:101C8000086000F03FF808490968C1F30311074AEA
:101C9000515CC8400649086006480068FFF7C0FE6E
:101CA00000204CE7003C024008380240B4A901087B
:101CB000000000202000002001480068704700005C
:101CC0000000002000B5FFF7F7FF04490968C1F3E1
:101CD0008221034A515CC84000BD00000838024020
:101CE000C4A9010800B5FFF7E7FF04490968C1F37B
:101CF0004231034A515CC84000BD00000838024030
:101D0000C4A901082DE9F047002400250026A146BA
:101D10002548006800F00C0020B1042805D00828F0
:101D20003AD105E0DFF8849039E0DFF8849036E0BE
:101D30001D48001F006800F03F041B48001F00689A
:101D400000F4800078B11A481749091F0968C1F3E7
:101D50008811A0FB01700146224600233846FEF799
:101D600099FA05460EE011480F49091F0968C1F3A9
:101D70008811A0FB01700146224600233846FEF779
:101D800089FA05460848001F0068C0F30140401C5E
:101D90004600B5FBF6F902E0DFF8109000BF00BF87
:101DA0004846BDE8F0870000083802400024F400EF
:101DB00000127A00F8B504460CB90120F8BD20786D
:101DC00000F00100002874D0F948006800F00C0011
:101DD00004280DD0F648006800F00C00082813D144
:101DE000F348001F006800F48000B0F5800F0BD1AD
:101DF000EF4808380068C0F34040002859D06068B8
:101E0000002856D10120D9E700BF6068B0F5803FB7
:101E100008D1E7480838006840F48030E4490839C0
:101E200008601EE06068B0F5A02F0DD1E0480838CA
:101E3000006840F48020DE490839086008460068E0
:101E400040F4803008600CE0D9480838006820F47D
:101E50008030D749083908600846006820F480209F
:101E6000086000BF606890B1FFF7AAFD054606E074
:101E7000FFF7A6FD401B642801D903209EE7CC484C
:101E800008380068C0F340400028F1D011E0FFF7A7
:101E900097FD054606E0FFF793FD401B642801D936
:101EA00003208BE7C24808380068C0F34040002890
:101EB000F1D1207800F0020002285FD1BC48006810
:101EC00000F00C0058B1BA48006800F00C00082877
:101ED0001CD1B748001F006800F48000B0B9B448B6
:101EE00008380068C0F3400020B1E068012801D044
:101EF000012063E7AE480838006820F0F800216947
:101F000040EAC100AA490839086037E0E06800B338
:101F10000120A8490860FFF753FD054606E0FFF7DA
:101F20004FFD401B022801D9032047E7A04808388D
:101F30000068C0F340000028F1D09D4808380068D0
:101F400020F0F800216940EAC10099490839086089
:101F500014E0002097490860FFF732FD054606E0CF
:101F6000FFF72EFD401B022801D9032026E79048E9
:101F700008380068C0F340000028F1D1207800F054
:101F8000080008282CD16069A8B101208A4908609E
:101F9000FFF716FD054606E0FFF712FD401B02287D
:101FA00001D903200AE782486C300068C0F3400082
:101FB0000028F1D014E000207F490860FFF700FD01
:101FC000054606E0FFF7FCFC401B022801D9032070
:101FD000F4E677486C300068C0F340000028F1D187
:101FE000207800F00400042870D1002770483830B1
:101FF000006800F0805090B900BF002000906C484D
:102000003830006840F0805069493831086008462F
:10201000006800F08050009000BF00BF01276748B3
:10202000006800F48070B0B96448006840F48070C3
:1020300062490860FFF7C4FC054606E0FFF7C0FCF4
:10204000401B022801D90320B8E65C48006800F470
:1020500080700028F2D000BFA068012808D1544841
:102060006830006840F001005149683108601DE0A7
:10207000A06805280DD14E486830006840F0040083
:102080004B49683108600846006840F0010008606C
:102090000CE047486830006820F00100444968318E
:1020A00008600846006820F00400086000BFA068CF
:1020B000A8B1FFF785FC054609E0FFF781FC401B4E
:1020C00041F28831884202D9032077E626E0384879
:1020D00068300068C0F340000028EED013E0FFF73E
:1020E0006FFC054608E0FFF76BFC401B41F28831AE
:1020F000884201D9032061E62D4868300068C0F3AA
:1021000040000028EFD1012F07D12948383000685E
:1021100020F0805026493831086000BFA0690028AF
:1021200045D02348006800F00C0008285DD0A06965
:10213000022845D100201F490866FFF741FC0546EB
:1021400006E0FFF73DFC401B022801D9032035E6DD
:10215000174808380068C0F340600028F1D1D4E97E
:1021600007010843616A40EA81110122A06AC2EBBB
:10217000500041EA00412C20005D41EA00600C491A
:10218000091F086001200B490866FFF719FC054686
:1021900006E0FFF715FC401B022801D903200DE6DD
:1021A000034808380068C0F340600028F1D049E0D7
:1021B0000838024000004742800E4742007000404D
:1021C000002021490866FFF7FBFB054606E0FFF704
:1021D000F7FB401B022801D90320EFE51B480068EC
:1021E000C0F340600028F2D12CE0A069012800D1A2
:1021F000E4E51648001D0668A069012820D006F411
:102200008001E06981421BD106F03F01206A8142D2
:1022100016D147F6C0703040616AB0EB811F0FD114
:1022200006F440310122A06AC2EB5000B1EB004F2E
:1022300006D106F070612C20005DB1EB006F01D07B
:102240000120BBE50020B9E500004742003802400C
:1022500070B504460E4615460CB9012070BD94F8C1
:10226000490028B9002084F84800204600F01CF8F6
:1022700004F108012068FEF7BBFC3146A268206823
:10228000FEF7E4FC2946236BD4E90102FEF78CFC3F
:10229000A168206850F8210040F00100A268216880
:1022A00041F822000020D9E710B586B0044600BFEF
:1022B000002000902248006840F00100204908609A
:1022C0000846006800F00100009000BF00BF00BF9A
:1022D000002000901A480838006840F008001849AB
:1022E000083908600846006800F00800009000BF48
:1022F00000BF00BF002000900846006840F01000BA
:1023000008600846006800F01000009000BF00BFA1
:102310004CF20370019002200290012003900220F1
:1023200004900C20059001A90648FFF731FA4FF6FA
:102330008070019001A90448FFF72AFA06B010BD89
:1023400038380240000C024000100240042808D136
:102350004FF0E021096941F004014FF0E0221161E2
:1023600007E04FF0E021096921F004014FF0E0227D
:102370001161704770B504462546681EB0F1807F34
:1023800001D301200FE0681E4FF0E02148610F21CA
:102390004FF0FF3000F0C6FD00204FF0E0218861D3
:1023A00007200861002070BD10B504460CB901205B
:1023B00010BD94F83D0028B9002084F83C00204668
:1023C00000F025F8022084F83D00211D206800F06F
:1023D000E9FA012084F8460000BF84F83E0001219C
:1023E0003F200155402001554120015500BF00BF4D
:1023F000012084F842004320015544200155452026
:10240000015500BF012084F83D000020D0E770474F
:10241000014691F83D00012801D0012070470220BB
:1024200081F83D000868C06840F001000B68D86082
:102430001A4B086898421BD00868B0F1804F17D03B
:10244000174B0868984213D0164B086898420FD073
:10245000154B086898420BD0144B0868984207D077
:10246000134B0868984203D0124B086898420CD16D
:102470000868806800F00702062A0CD00868006827
:1024800040F001000B68186005E00868006840F043
:1024900001000B6818600020C0E700000000014048
:1024A0000004004000080040000C0040000401400F
:1024B000004001400018004070477047014600226C
:1024C000002391F83D2091F83E3042EA0300704726
:1024D0002DE9F84F0446206805682068C668206822
:1024E00047694FF00009CA4605F00F09B9F1000F1E
:1024F0000AD105F0200038B106F0200020B12046B6
:1025000000F0F1FABDE8F88FB9F1000F72D007F0D2
:10251000010018B906F4907000286BD005F0010096
:1025200030B106F4807018B1206C40F001002064D6
:1025300005F0040030B107F0010018B1206C40F044
:102540000200206405F0020030B107F0010018B16C
:10255000206C40F00400206405F0080048B106F04B
:10256000200010B907F0010018B1206C40F00800FD
:102570002064206C70B305F0200028B106F0200024
:1025800010B1204600F0AFFA20684069C0F3801A0D
:10259000206C00F0080010B9BAF1000F23D02046DB
:1025A00000F076FA2068406900F04000402816D11B
:1025B0002068406920F0400021684861A06B50B15C
:1025C0005648A16B0865A06BFEF7B7FB10B1A06B76
:1025D000016D88470CE02046FFF76FFF08E02046BA
:1025E000FFF76BFF04E02046FFF767FF0020206441
:1025F00088E7FFE7206B012879D105F0100000285B
:1026000075D006F01000002871D000BF00200090A7
:1026100020680068009020684068009000BF00BFFC
:102620002068406900F04000402839D1A06B006864
:1026300040681FFA80F8B8F1000F30D0A08D4045F7
:102640002DDDA4F82E80A06BC069B0F5807F1FD06F
:102650002068C06820F480702168C86020684069E4
:1026600020F00100216848612068406920F04000A6
:1026700021684861202084F83E0000202063206803
:10268000C06820F010002168C860A06BFEF700FB56
:10269000A08DE28D801A81B22046FFF70DFF31E751
:1026A000A08DE18D401A1FFA80F8E08DE8B1B8F1F5
:1026B000000F1AD02068C06820F490702168C860AC
:1026C0002068406920F0010021684861202084F8DA
:1026D0003E00002020632068C06820F010002168C0
:1026E000C86041462046FFF7E7FE0BE7FFE705F02D
:1026F000800030B106F0800018B1204600F08BFB5E
:1027000000E705F0400030B106F0400018B1204667
:1027100000F0D9F9F6E600BFF4E600007D2A0008D3
:1027200010B504460CB9012010BDA06900B100E04D
:1027300000BF94F83D0028B9002084F83C002046F2
:1027400000F028F8242084F83D002068C06820F4B8
:1027500000502168C860204600F024FA2068006913
:1027600020F49040216808612068406920F02A0028
:10277000216848612068C06840F400502168C86042
:1027800000202064202084F83D0084F83E000020D2
:10279000CAE7000010B586B004462E49206888427A
:1027A00055D100BF00BF002000902B48006840F0CA
:1027B0001000294908600846006800F010000090E9
:1027C00000BF00BF00BF00BF00BF00200090224834
:1027D0001438006840F001001F49143908600846A9
:1027E000006800F00100009000BF00BF00BF00BF04
:1027F00000BF002000900846006840F0010008601B
:102800000846006800F00100009000BF00BF00BF54
:1028100048150190022002900120039002200490AC
:102820000720059001A90D48FEF7B2FF4FF4806024
:1028300001900720059001A90848FEF7A9FF25206F
:10284000FFF715F9032211462520FFF720F906B0FE
:1028500010BD00000010014044380240000002405A
:1028600070B504460D46164694F83E00202816D151
:1028700005B10EB9012070BD00BF94F83C000128DD
:1028800001D10220F7E7012084F83C0000BF0020BE
:10289000206332462946204600F09AFAEBE70220F0
:1028A000E9E700001D4A0168914236D11C490988B8
:1028B00001F4004189BB1A49098801F4804171B1D2
:1028C000184909780A2903D00021154A118024E00B
:1028D0001349098841F40041114A11801DE0114952
:1028E00009780D2906D10E49098841F480410C4A26
:1028F000118012E00B490978094A1288C2F30D02CF
:10290000094B995406490988491C054A118011460A
:102910000988C72901DD002111807047001001409E
:10292000180000201A00002034030020704700BF68
:10293000FEE700BFFEE7704710B5FFF747F817F056
:102940007BFC012801D016F04DFF10BD0348006844
:1029500040F47000014908607047000088ED00E015
:1029600010B50E480068C06800F0010078B10C494D
:1029700008698047002009490968486200BF64204F
:1029800006490968C86264210448C16000BF6FF04D
:10299000010002490968086110BD000038050020E7
:1029A0008C00002010B50268294B98420ED0B0F17F
:1029B000804F0BD0274B984208D0274B984205D028
:1029C000264B984202D0264B984203D122F0700247
:1029D0004B681A431E4B984220D0B0F1804F1DD057
:1029E0001C4B98421AD01C4B984217D01B4B984254
:1029F00014D01B4B984211D01A4B98420ED01A4B50
:102A000098420BD0194B984208D0194B984205D0E8
:102A1000184B984202D0184B984203D122F44072CE
:102A2000CB681A4322F080034C6943EA0402026037
:102A30008B68C3620B688362054B984202D0084BD7
:102A4000984201D10B6903630123436110BD00006B
:102A5000000001400004004000080040000C00405D
:102A60000004014000400140004401400048014092
:102A700000180040001C00400020004070B50546D2
:102A8000AC6B0020E085E0842046FFF716FD70BDAA
:102A90000168C96821F490710268D16001684969D0
:102AA00021F0010102685161016B012905D1016822
:102AB000C96821F010010268D160202180F83E1021
:102AC00000210163704710B504462068C06820F0FB
:102AD00040002168C860202084F83D002046FFF7B0
:102AE00025FF002010BD70B5044694F83E00222852
:102AF00056D1A068B0F5805F0CD1206950B900258F
:102B0000A66A20684068C0F308003080A06A801C74
:102B1000A06215E0A56A0026A068B0F5805F03D02A
:102B2000A06828B9206918B920684068287004E0B6
:102B30002068406800F07F002870A06A401CA062F6
:102B4000E08D401E80B2E08540BB2068C06820F068
:102B500020002168C8602068C06820F48070216867
:102B6000C8602068406920F0010021684861202089
:102B700084F83E00206B01280AD12068C06820F04C
:102B800010002168C860A18D2046FFF795FC02E087
:102B90002046FFF787FE0020206370BD0020FCE781
:102BA0000220FAE72DE9F84F04462068006920F476
:102BB0004050E1680843216808612169A068084322
:102BC00061690843E169084300902068C06849F2E0
:102BD0000C618843009908432168C86020684069F7
:102BE00020F44070A1690843216848617649206853
:102BF000884203D075492068884203D1FFF772F8F4
:102C0000814602E0FFF75EF88146E069B0F5004FCB
:102C10006CD102206168A0FB015003461920A9FB7A
:102C2000007001462A463846FDF734FB6421B0FBAC
:102C3000F1F04FEA001A02206168A0FB01510B4637
:102C40001920A9FB00712A463846FDF723FB83466D
:102C500002206168A0FB015003461920A9FB007106
:102C60002A463846FDF716FB6421B0FBF1F000EB75
:102C7000C00101EB0010ABEB8000322101EBC00082
:102C80006421B0FBF1F000F0F8000AEB400A0220EA
:102C90006168A0FB015003461920A9FB00700146A2
:102CA0002A463846FDF7F6FA834602206168A0FB03
:102CB000015003461920A9FB00712A463846FDF74A
:102CC000E9FA6421B0FBF1F000EBC00101EB001068
:102CD000ABEB8000322101EBC0006421B0FBF1F0CE
:102CE00000F007005044216888606AE004206168B1
:102CF000A0FB015003461920A9FB007001462A469B
:102D00003846FDF7C7FA824604206168A0FB0150EF
:102D100003461920A9FB007001462A463846FDF7F4
:102D2000B9FA6421B0FBF1F000EBC00101EB001037
:102D3000AAEB8000322101EB00106421B0FBF1F01E
:102D400000F0F00A04206168A0FB0170034619201E
:102D5000A9FB00513A462846FDF79CFA6421B0FBD6
:102D6000F1F00AEB001A04206168A0FB01510B4648
:102D70001920A9FB00712A463846FDF78BFA8346D5
:102D800004206168A0FB015003461920A9FB0070D4
:102D900001462A463846FDF77DFA6421B0FBF1F082
:102DA00000EBC00101EB0010ABEB8000322101EB26
:102DB00000106421B0FBF1F000F00F0050442168D6
:102DC0008860BDE8F88F0000001001400014014049
:102DD00010B5034699629A85DA850020186422208E
:102DE00083F83E0000BF002083F83C0000BF186855
:102DF000C06840F480701C68E0601868406940F06A
:102E000001001C6860611868C06840F020001C6800
:102E1000E060002010BD014691F83D00212828D136
:102E20008868B0F5805F0BD1086948B90A6A1088D4
:102E3000C0F308000B685860086A801C086205E04F
:102E40000B6A581C086218780B685860C88C401EC2
:102E500080B2C88458B90868C06820F080000B6848
:102E6000D8600868C06840F040000B68D860002057
:102E700070470220FCE7000070B500240F4D104899
:102E8000FFF726FB00BF03E0641CAC4200D904E05E
:102E90000B48FFF713FB2028F6D100BF002403E006
:102EA000641CAC4200D906E0012206490448FFF741
:102EB000D7FC0028F4D100BF70BD0000FFFF010067
:102EC000FC0300201A00002000BFFEE70FB4054BF2
:102ED00010B503A9044A029800F04CF810BC5DF844
:102EE00014FB0000E5640008140000200FB4084B38
:102EF00010B504A902AA039800F03CF8044602A900
:102F0000002000F062FA204610BC5DF814FB0000BF
:102F1000CB33000802480068C0F30220704700006D
:102F20000CED00E010B5002804DB0A07130E054A7B
:102F3000135406E00A07140E034A00F00F031B1F88
:102F4000D45410BD00E400E018ED00E000487047E4
:102F50003003002002E008C8121F08C1002AFAD17D
:102F600070477047002001E001C1121F002AFBD109
:102F7000704700002DE9FF4F8DB00F460546002633
:102F800006E025280BD0DDE90F1290476D1C761C5A
:102F900028780028F5D111B03046BDE8F08F002424
:102FA000A246A1460122E94900E0044315F8013F89
:102FB000203B02FA03F00842F7D128782A2810D0E3
:102FC0006FF02F022878A0F13001092914D80AEBFC
:102FD0008A0102EB410144F0020400EB010A6D1C7E
:102FE000F0E701CF5FEA000A03D544F40054CAF1C8
:102FF000000A44F002046D1C28782E2817D115F819
:10300000010F44F004042A280ED06FF02F02287814
:10301000A0F1300109290AD809EB890102EB41012D
:1030200000EB01096D1CF2E757F8049B6D1C287832
:103030006C280FD006DC4C2817D068280DD06A28E1
:1030400014D104E0742810D07A280FD10DE044F494
:1030500000140AE044F4801401E044F44014697858
:10306000814202D104F580146D1C6D1C28786E28F5
:103070001ED00CDC632830D004DC00288BD058280C
:1030800011D19FE0642867D069280CD164E07328CF
:103090002DD004DC6F2872D0702804D194E07528FC
:1030A0006ED078286DD0DDE90F129047761C4BE189
:1030B000C4F30250022806D0032809D0042801CF07
:1030C00009D0066040E101CFF117C0E900613BE1A2
:1030D00001CF068038E1067036E117F8040B8DF851
:1030E000000000208DF80100EB46012003E057F8B6
:1030F00004BB4FF0FF3061074FF0000102D40DE038
:1031000008F10101884649450FDA8045F8DB1BF8D4
:1031100008100029F4D108E008F101018846814235
:10312000FADB1BF808100029F6D1DDE90F23AAEB22
:1031300008008146214600F031F9304400EB0806D2
:1031400004E0DDE90F121BF8010B9047B8F101080C
:10315000F7D221464846F2E00A21C4F302524FF06A
:10316000000B0891022A04D001CFC117032A09D00D
:103170000AE0FF1D27F00707F7E8020108E02CE04E
:103180001EE01FE000B2C117042A01D140B2C117EE
:10319000021E71F1000206DA0023D0EB030063EB9C
:1031A00001012D2202E0220504D52B228DF82420D6
:1031B000012203E0E20701D02022F7E7904653E026
:1031C0000A210BE0102109E010214FF0000B44F020
:1031D00004044FF00809089103E008214FF0000BA8
:1031E0000891C4F30252022A04D001CF0021032A1D
:1031F00006D006E0FF1D27F00707F7E8020103E00D
:1032000080B2042A00D1C0B24FF0000822072BD5AB
:103210002A78702A07D0DDF820C08CF0100C5CEA08
:103220000B0C05D00EE040228DF82420012208E08E
:1032300050EA010306D030238DF824308DF8252084
:1032400002229046089B83F0080353EA0B030BD13C
:1032500050EA010201D1620706D530228DF8242000
:103260004FF00108A9F101092A78582A04D038A2A0
:103270000B9208AA0A920BE03AA2F9E75B46089A79
:10328000FDF708F80B9B9B5C0A9A521E0A9213707A
:1032900050EA0102F2D10A98ADEB000000F1200BD8
:1032A000600702D524F4803401E04FF00109D945CC
:1032B00002DDA9EB0B0000E0002000EB0B01414414
:1032C0000890AAEB010AE00306D4DDE90F232146AA
:1032D000504600F063F806444FF0000908E009A9E1
:1032E00011F80900DDE90F12904709F10109761C78
:1032F000C145F4DBE0030CD5DDE90F232146504640
:1033000000F04CF8064404E0DDE90F12302090474D
:10331000761C0899481E08900029F5DC08E00A98F8
:103320000A990078491C0A91DDE90F129047761C32
:10333000BBF10001ABF1010BF1DC21465046DDE9A8
:103340000F2300F019F806446D1C21E6092801003E
:10335000303132333435363738396162636465660B
:1033600000000000303132333435363738394142CD
:1033700043444546000000002DE9F0410446002585
:103380001E461746880404D405E039462020B0477D
:103390006D1C641EF9D52846BDE8F0812DE9F04189
:1033A000044600251E469046C80301D5302700E09C
:1033B0002027880404D505E041463846B0476D1CF7
:1033C000641EF9D52846BDE8F0810A68531C0B60DD
:1033D000107070472DE9F04105460E46002440E08C
:1033E0000EF06AF80746214800EB04100068002838
:1033F00033D11E4800EB0410056038460EF0BAF8D1
:1034000000201A4901EB0411486000BF174800EB87
:103410000410807B20B100BF15A0FFF757FD00BF4F
:1034200000BF0020114901EB04110881287800F049
:10343000F000102804D10EB1012002E0002000E0CD
:1034400001200A4901EB041148810020074901EBE2
:10345000041188812046BDE8F08138460EF08AF8D4
:10346000641C042CBCDB4FF0FF30F4E7805A0020D2
:10347000736F636B6574735B695D2E73656C6563F5
:10348000745F77616974696E67203D3D203000008C
:1034900070B504460420FEF759FF0A48046025462B
:1034A0004FF47A7045434FF0E020006940F002008D
:1034B0004FF0E021086108464561006940F00100D5
:1034C000086170BD1000002030B50446002504E0FE
:1034D0004FF47A7000F004F86D1CA542F8D330BDAB
:1034E00070B5034600224FF0E02675690D4E366830
:1034F00003FB06F44FF0E026B16910E04FF0E02640
:10350000B06988420BD0884202D20E1A324402E0DF
:103510002E1A0E4432440146A24200D300E0EDE7E9
:1035200000BF70BD1000002070B505460E4600BFFC
:103530002DB900BF0CA0FFF7C9FC00BF70BD00BFD4
:103540006C6A00BF00BF6CB1607908280AD100BF67
:1035500000BF3068E169884204D100BF00BF28463F
:1035600000F01CFA00BFE9E76E6574696620213D32
:10357000204E554C4C0000007CB5064600BF2EB9CD
:1035800000BF44A0FFF7A2FC00BF7CBD00BF746A6F
:1035900000BF2CB900BF46A0FFF798FC00BFF4E7BE
:1035A00000BF00BF00BF00206082A06A401C90B135
:1035B00000BF00BFA06A1E303C21B0FBF1F5B5F59D
:1035C000803F01D34FF6FF75A582A08A08B901207C
:1035D000A08200BF00BFE06A401CA0B100BF00BFD6
:1035E000E06A1E303C21B0FBF1F5B5F5803F01D318
:1035F0004FF6FF756581608908B90120608100BFC1
:1036000000BF6089E081206B401CA0B100BF00BFFB
:10361000206B1E303C21B0FBF1F5B5F5803F01D3A6
:103620004FF6FF75A581A08908B90120A08100BFD0
:1036300000BFA08920826089A189884204DBA0891B
:10364000002801DD00206081E07910B1206A01903E
:103650000FE0207F7F2802DCFF21019108E0C028D5
:1036600003DB6FF07F41019102E04FF6FF710191A2
:1036700000BF606A009000BF00BF0A21204601F031
:103680000FFA6B4601AA04F11C0130460BF07CFADC
:1036900000BF7AE7646863705F62696E643A206EA7
:1036A0006574696620213D204E554C4C0000000099
:1036B000646863705F62696E643A20646863702056
:1036C000213D204E554C4C002DE9F0410646746AD0
:1036D00000BF00BF0821204601F0E2F9002204F1FA
:1036E0001C01304602F0E0F905460DB100BF00BFF5
:1036F000A079FF2802DAA079401CA0714FF4FA7774
:1037000007F2F310394690FBF1F0208100BF00BFB3
:10371000BDE8F08170B500BF00BF1B4805682FE011
:103720006C6AFCB16079E8B1A08A78B1608A401C0B
:1037300080B26082A18A884208D100BF00BF2846BB
:1037400000F0D8FF284601F0B3F918E0208A50B104
:10375000218A481E2082012905D100BF00BF2846CA
:1037600001F05DFA0BE0E08948B1E189481EE08193
:10377000012904D100BF00BF284601F02BFA2D68B3
:10378000002DCDD170BD00000C0200202DE9F05FAE
:1037900007460D4616469A4600BF3FB900BF44A0F3
:1037A000FFF794FB00BF0020BDE8F09F00BF00BF03
:1037B00035B900BF46A0FFF789FB00BF0020F3E743
:1037C00000BF4FF420724FF49A7136200BF036FB95
:1037D0008146B9F1000F03D100BF00BF0020E3E72D
:1037E00000BFB9F80A00B0F59A7F04D200BF40A02C
:1037F000FFF76CFB00BF00BF032E02D168790328DE
:1038000008D1A87918B9FCF77BFD494908604848F8
:103810000068286000BF00BFD9F804404FF49A71D7
:103820002046FCF7A6FD01202070607097F830005C
:10383000A070286807F038FC6060082E0BD0042EBA
:1038400009D0072E07D0032E07D16879052802D0AA
:103850006879042801D17868E0604FF000080BE037
:1038600007F12A0010F8081004F11C0000F80810F5
:1038700008F101001FFA80F8B8F1060FF0D32D48C7
:10388000C4F8EC000123352204F1F001002000F01F
:10389000B1FA8346324604F1F001584600F0C8FA06
:1038A0008346BAF1000F01D0AAF800B048467BE782
:1038B000646863705F6372656174655F6D73673AB6
:1038C000206E6574696620213D204E554C4C0000E9
:1038D000646863705F6372656174655F6D73673A96
:1038E000206468637020213D204E554C4C00000040
:1038F000646863705F6372656174655F6D73673A76
:1039000020636865636B20746861742066697273F4
:103910007420706275662063616E20686F6C64202D
:1039200073747275637420646863705F6D7367008D
:10393000800200206382536310B500BF0C480078FA
:10394000002804DC00BF0BA0FFF7C0FA00BF00BFD7
:1039500007480078401E064908700846007830B9CC
:103960000D48006813F0CAFE00200B49086010BD26
:103970007C020020646863705F7063625F726566DA
:10398000636F756E7428293A20726566636F756E71
:1039900074206572726F7200780200202DE9FE4F6C
:1039A0000646746A00BF00BF0C21204601F078F87B
:1039B00002AB042221463046FFF7E8FE054675B308
:1039C000D5F804800423322208F1F001BDF8080084
:1039D00000F010FA0290E06907F066FB824652465A
:1039E00008F1F001BDF8080000F052FA02902A46F2
:1039F00008F1F001BDF8080000F0C6FA14484323AE
:103A0000144A2946CDE900601348006813F0E4FF2A
:103A1000074628460BF0E8FD00BF00BF04E0FFE7C3
:103A200000BF00BF4FF0FF37A079FF2802DAA0796E
:103A3000401CA07142F2107909F2F3104FF4FA71B0
:103A400090FBF1F0208100BF00BF3846BDE8FE8F3B
:103A500054DB010858DB0108780200202DE9FE4FF5
:103A600007467C6A4FF0000A00BF00BF0020E061FB
:103A70000621204601F014F802AB01222146384607
:103A8000FFF784FE0546002D4AD06E6800BF00BFD8
:103A90000223392206F1F001BDF8080000F0AAF96E
:103AA00002903A8D06F1F001BDF8080000F034FAFA
:103AB00002900423372206F1F001BDF8080000F05F
:103AC00099F90290D0460DE0274810F8082006F139
:103AD000F001BDF8080000F0ABF9029008F1010018
:103AE00000F0FF08B8F1040FEED32A4606F1F0010A
:103AF000BDF8080000F048FA00BF00BF1B48432390
:103B00001B4A2946CDE900701A48006813F064FF8B
:103B100000BF00BF28460BF067FD00BF00BF01E0FB
:103B200000BF00BFA079FF2802DAA079401CA07175
:103B3000A079062803DAA1790120884000E03C2022
:103B400000EB4001C1EBC0104FF6FF7101EAC00964
:103B500009F2F3104FF4FA7190FBF1F0208100BFED
:103B600000BF5046BDE8FE8F7402002054DB010800
:103B700058DB01087802002070B50D48056814E094
:103B80006C6A8CB12089012803DD2089401E2081C8
:103B90000AE02089012807D12089401E208100BF2A
:103BA00000BF284601F063F82D68002DE8D170BDF4
:103BB0000C020020F8B506460F46746A0020206209
:103BC00060622648C07810B12548C068A0622348CA
:103BD000007918B122480069E06202E0A06A40085A
:103BE000E0621E48407918B11D484069206304E036
:103BF000A06AC0EBC000C00820633869E0611748C4
:103C0000807938B11649886907F04EFA20620120A0
:103C1000E07101E00020E0711048C07920B1104946
:103C2000C86907F041FA606200250DE005F108015E
:103C30000B4A52F8210007F037FA009069462846EF
:103C400001F076FA681CC5B2022D05DA05F108000C
:103C50000249085C0028E9D1F8BD0000584E012057
:103C6000304E012070B50446656A00BF00BF0C21CC
:103C7000284600F015FF054B1A46114620460AF06B
:103C800083FF2046FFF7EAFE70BD000054DB010809
:103C900070B505460E466C6A00BF00BF0B488078C1
:103CA00080B1002020810A49886807F0FDF9A061F1
:103CB00000BF00BF3069E06100BF00BF284600F0D0
:103CC00009FE01E000BF00BF70BD0000584E01209A
:103CD000304E012010B51C48007800282DD100BFBF
:103CE0001A48006820B100BF19A0FFF7EFF800BF25
:103CF00000BF13F0A3FC154908600846006810B91E
:103D00004FF0FF3010BD11480068407A40F02000AD
:103D10000E4909684872442217490C48006813F09C
:103D20000FFA432214490948006813F087FA002269
:103D300012490648006813F0C3FC03480078401C91
:103D4000014908700020DDE77C0200207802002095
:103D5000646863705F696E635F7063625F726566FB
:103D6000636F756E7428293A206D656D6F727920C6
:103D70006C65616B0000000054DB01089945000888
:103D800070B505466C6A04B970BD6079042809D025
:103D900003DC80B103280FD107E0052803D00A28EF
:103DA0000AD101E000BF00BF00BF0020A07128467B
:103DB00000F05EFB10E00FE000BF60790C2804DD2E
:103DC00000BF07A0FFF782F800BF00BF0020A0716E
:103DD0002846FFF743FE00BF00BF00BFD4E7000046
:103DE000696E76616C696420646863702D3E7374DB
:103DF000617465002DE9F04104460D4617461E46E4
:103E000000BFA01C3044442804D900BF0748FFF776
:103E10005DF800BF00BF2046611C8CB22F542046C5
:103E2000611C8CB22E542046BDE8F081A4E201084A
:103E300070B504460D46164600BF442C04D300BF9F
:103E400005A0FFF743F800BF00BF2046611C8CB2FD
:103E50002E54204670BD0000646863705F6F7074FC
:103E6000696F6E5F627974653A206F7074696F6E06
:103E7000735F6F75745F6C656E203C2044484350DF
:103E80005F4F5054494F4E535F4C454E0000000069
:103E900070B504460D46164600BF201D442804D9BF
:103EA00000BF0EA0FFF712F800BF00BF320E204681
:103EB000611C8CB22A54C6F307422046611C8CB2A6
:103EC0002A54C6F307222046611C8CB22A5420468D
:103ED000611C8CB22E54204670BD00006468637073
:103EE0005F6F7074696F6E5F6C6F6E673A206F7092
:103EF00074696F6E735F6F75745F6C656E202B20D5
:103F000034203C3D20444843505F4F5054494F4E6D
:103F1000535F4C454E00000070B504460D461646F2
:103F200000BFA01C442804D900BF08A0FEF7CEFFA4
:103F300000BF00BF320A2046611C8CB22A542046C2
:103F4000611C8CB22E54204670BD00006468637002
:103F50005F6F7074696F6E5F73686F72743A206F11
:103F60007074696F6E735F6F75745F6C656E202B14
:103F70002032203C3D20444843505F4F5054494F2D
:103F80004E535F4C454E000070B504460D46164634
:103F9000FF222046611C8CB22A5404E000222046F5
:103FA000611C8CB22A54442C02D304F0030008B1E3
:103FB000442CF3D304F1F00081B230460BF00EFC38
:103FC00070BD00002DE9F04F8BB0814600200690B7
:103FD00005900A21DE48FCF7CCF9B9F80A002C2834
:103FE00004D26FF001000BB0BDE8F08FD9F80400E7
:103FF00004904FF0F00AB9F80800079000BF4C4653
:10400000CDF820A00AE06089AAEB00001FFA80FA30
:1040100061890798401A80B20790246814B16089BA
:104020005045F0DD14B96FF00100DCE75646079803
:10403000099060680A9050E10A98805D039000271B
:104040004FF0FF38B01C1FFA80FBB34501DAB81EF1
:10405000C9E76189701C814203DD711C0A98455CC7
:1040600007E0206818B120684068007800E0002070
:1040700005462F460398342854D00BDC032820D063
:1040800003DC80B101286FD111E0062824D0332849
:104090006AD13DE0352857D036285FD03A2868D01D
:1040A0003B287AD16FE00020054607467BE000BF41
:1040B000042D02D06FF0050095E700BF4FF0060811
:1040C00071E0042700BFBD4202DA6FF005008AE705
:1040D00000BF4FF0070866E000BFE91705EB9171DC
:1040E0008910A5EB810111B16FF005007BE700BFDE
:1040F000082D01DA284600E00820074600BFBD422F
:1041000002DA6FF005006EE700BF4FF008084AE0E2
:1041100000BF042D02D06FF0050064E700BF4FF030
:10412000030840E000BF012D02D06FF005005AE700
:1041300000BF00BF0898F02802D06FF0050052E7DA
:1041400000BF4FF000082EE000BF012D02D06FF03D
:10415000050048E700BF4FF0010824E000BF042D30
:1041600003D06FF005003EE717E000BF4FF00208F4
:1041700019E000BF042D02D06FF0050033E700BF47
:104180004FF004080FE000BF042D02D06FF00500CF
:1041900029E700BF4FF0050805E0002700BF00BF7A
:1041A00000BF00BF00BF00BF039810B9701C86B2EB
:1041B00077E07019801CB0F5803F02DB6FF00100E2
:1041C00011E77019801C86B2002F6ADD0020029072
:1041D00000BF00BFB8F1000F02DBB8F10A0F04DB2B
:1041E00000BF5CA0FEF772FE00BF00BF584810F889
:1041F0000800B0BB042F01DA384600E0042001902B
:104200005B4602A92046019A0BF05EF80146019830
:10421000814202D06FF00100E5E6042F27DD00BFE8
:10422000F91707EB91718910A7EB810111B16FF0BC
:104230000500D8E600BF0120454901F808000298B2
:1042400006F032FF484941F82800381FC7B20BF189
:10425000040080B200900098584503DA6FF0010026
:10426000C1E61DE0DDF800B008F10108B1E7042F58
:1042700004D1029806F018FF029009E000BF012F58
:1042800002D06FF00500AEE600BF9DF80800029076
:1042900001202F4901F808003349029841F828000D
:1042A00000BF6089B04217DC6089301A86B261892C
:1042B0000998401A80B209900998864209DA246860
:1042C00000BF14B96FF005008DE600BF60680A906A
:1042D00002E06FF0010086E600BF3CB1099886421B
:1042E00004DA0A98805DFF287FF4A6AE18480078AB
:1042F000D0B11D4908680021154A1170012803D169
:104300000121069100BF0EE0022803D10121059191
:1043100000BF08E0032804D101210591069100BFE8
:1043200001E000BF00BF00BF069830B1002006903A
:104330004FF06C0AEC20079061E6059830B1002040
:1043400005904FF02C0A6C20079058E600204AE6B2
:10435000584E0120636865636B206465636F646514
:104360005F69647800000000304E01202DE9FC47B1
:1043700007467C6A00BF00BF0421204600F090FB86
:1043800001AB032221463846FFF700FA0546002D0F
:1043900044D06E680223392206F1F001BDF8040012
:1043A000FFF728FD01903A8D06F1F001BDF80400F9
:1043B000FFF7B2FD01900423372206F1F001BDF8AA
:1043C0000400FFF717FD01904FF000080DE02548AD
:1043D00010F8082006F1F001BDF80400FFF728FDF1
:1043E000019008F1010000F0FF08B8F1040FEED3CE
:1043F0002A4606F1F001BDF80400FFF7C5FD43238E
:10440000194A294619480097006813F057FA81465F
:1044100028460BF0E9F800BF00BF03E000BF00BF73
:104420004FF0FF39A079FF2802DAA079401CA07173
:10443000A0790A2805DAA0794FF47A7110FB01F00F
:1044400001E042F210701FFA80FA0AF2F3104FF402
:10445000FA7190FBF1F0208100BF00BF4846BDE833
:10446000FC8700007402002058DB0108780200205D
:104470002DE9FC5F8046D8F8244000BF00BF03212F
:10448000204600F00DFB01AB032221464046FFF71A
:104490007DF90646002E56D075680223392205F1B3
:1044A000F001BDF80400FFF7A5FC01904FF4107275
:1044B00005F1F001BDF80400FFF72EFD0190042383
:1044C000322205F1F001BDF80400FFF793FC0190E2
:1044D000E06906F0E9FD83465A4605F1F001BDF8B2
:1044E0000400FFF7D5FC01900423372205F1F00109
:1044F000BDF80400FFF77EFC019000270AE0234886
:10450000C25D05F1F001BDF80400FFF791FC0190D8
:10451000781CC7B2042FF2D3324605F1F001BDF882
:104520000400FFF731FD4323194A31461948CDF8FD
:104530000080006813F0C2F9814630460BF054F851
:1045400000BF00BF03E000BF00BF4FF0FF39A079FC
:10455000FF2802DAA079401CA071A0790A2805DAA8
:10456000A0794FF47A7110FB01F001E042F2107073
:104570001FFA80FA0AF2F3104FF4FA7190FBF1F08F
:10458000208100BF00BF4846BDE8FC9F74020020A8
:1045900058DB0108780200202DE9F05F1646DDF8AF
:1045A00028B0514847687C6AD6F804900CB120794D
:1045B00000B994E000BF00BF00BF00BF00BF00BF54
:1045C00000BF00BF70892C2802DA00BF00BF86E060
:1045D00099F80000022802D000BF00BF7FE000254C
:1045E0000CE007F12A00415D09F11C00405D8142A9
:1045F00002D000BF00BF72E0681CC5B297F830005F
:10460000A84201DD062DECD3D9F8040006F04CFDDC
:104610002168884202D000BF00BF60E021463046DA
:10462000FFF7D0FC10B100BF00BF58E000BF00BFD3
:104630002E48407810B900BF00BF50E0D6F804A063
:104640002B4890F80480B8F1050F26D100BF00BFB9
:104650006079012810D151463846FFF7ABFA97F838
:10466000310000F0080018B13846FFF72DF835E0AA
:104670003846FEF781FF31E06079032805D0607984
:10468000042802D06079052828D151463846FFF722
:1046900091FA3846FEF770FF20E0B8F1060F11D10D
:1046A0006079032808D06079012805D06079042852
:1046B00002D06079052805D100BF00BF3846FFF75A
:1046C000D1FA0BE0B8F1020F08D16079062805D1C4
:1046D00000BF00BF51463846FFF7DAFA00BF304648
:1046E0000AF082FFBDE8F09F405F0020584E012095
:1046F000304E01202DE9FE430646746A00BF00BF1C
:104700000CB9BDE8FE83607900B9FAE7A0690290B0
:104710000020A061E061206260622063E062A0622C
:10472000A08260822082E081304600F03FFA0028BB
:104730003FD00021204600F0B3F901AB072221460B
:104740003046FFF723F8054655B36F680423362239
:1047500007F1F001BDF80400FFF74CFB019002984F
:1047600006F0A2FC8046424607F1F001BDF80400C5
:10477000FFF78EFB01902A4607F1F001BDF8040017
:10478000FFF702FC432302AA29461048009600685E
:1047900013F094F828460AF027FF00BF00BF01E09D
:1047A00000BF00BF0A4B1A46114630460AF0ECF92A
:1047B00003E00021204600F073F9207918B1FFF7DB
:1047C000BBF80020207100BF9BE7000078020020AA
:1047D00054DB01082DE9FC4707467C6A00BF00BF97
:1047E0000521204600F05CF901AB03222146384642
:1047F000FEF7CCFF0546002D45D06E680223392216
:1048000006F1F001BDF80400FFF7F4FA01903A8DCB
:1048100006F1F001BDF80400FFF77EFB01900423D0
:10482000372206F1F001BDF80400FFF7E3FA01902A
:104830004FF000080DE0254810F8082006F1F001BF
:10484000BDF80400FFF7F4FA019008F1010000F050
:10485000FF08B8F1040FEED32A4606F1F001BDF8C7
:104860000400FFF791FB432304F11802294618487E
:104870000097006813F022F8814628460AF0B4FE3B
:1048800000BF00BF03E000BF00BF4FF0FF39A079B9
:10489000FF2802DAA079401CA071A0790A2805DA65
:1048A000A0794FF4FA6110FB01F001E044F62060BA
:1048B0001FFA80FA0AF2F3104FF4FA7190FBF1F04C
:1048C000208100BF00BF4846BDE8FC87740200207D
:1048D000780200202DE9FE4F074600BF47B900BF10
:1048E0005DA0FEF7F3FA00BF6FF00F00BDE8FE8F8A
:1048F00000BF7C6A00BF3CB900BF5EA0FEF7E6FACD
:1049000000BF6FF00500F1E700BF00BF00BF01214D
:10491000204600F0C5F802AB032221463846FEF7D8
:1049200035FF0646002E71D075680223392205F145
:10493000F001BDF80800FFF75DFA02903A8D05F12D
:10494000F001BDF80800FFF7E7FA029004233222D5
:1049500005F1F001BDF80800FFF74CFA0290E0699C
:1049600006F0A2FB83465A4605F1F001BDF80800A7
:10497000FFF78EFA02900423362205F1F001BDF80C
:104980000800FFF737FA0290A06906F08DFB834616
:104990005A4605F1F001BDF80800FFF779FA0290D8
:1049A0000423372205F1F001BDF80800FFF722FAD1
:1049B00002904FF000080DE0354810F8082005F18E
:1049C000F001BDF80800FFF733FA029008F101008A
:1049D00000F0FF08B8F1040FEED3324605F1F00104
:1049E000BDF80800FFF7D0FA2A4843232A4A314687
:1049F000CDE900702948006812F0EEFF814630468C
:104A00000AF0F2FD00BF00BF04E0FFE700BF00BFF7
:104A10004FF0FF39A079FF2802DAA079401CA0717D
:104A2000A079062803DAA1790120884000E03C2023
:104A300000EB4001C1EBC0104FF6FF7101EAC00A64
:104A40000AF2F3104FF4FA7190FBF1F0208100BFED
:104A500000BF48464AE70000646863705F73656C96
:104A60006563743A206E6574696620213D204E5559
:104A70004C4C0000646863705F73656C6563743AE6
:104A8000206468637020213D204E554C4C0000008E
:104A90007402002054DB010858DB01087802002072
:104AA00042798A4203D041710022827102817047AB
:104AB00070B5044600BF3CB900BF2FA0FEF706FA50
:104AC00000BF6FF00F0070BD00BF00BF94F8310051
:104AD00000F0010038B900BF2BA0FEF7F7F900BFC6
:104AE0006FF00F00EFE700BF656A00BF00BF208DC9
:104AF000B0F5107F04DA00BF00BF4FF0FF30E2E7EF
:104B000075B900BF00BF342008F0FCFC054625B98C
:104B100000BF00BF4FF0FF30D5E7656200BF05E082
:104B200000BF00BF287908B1FEF706FF34212846F0
:104B3000FBF71FFC00BF00BFFFF7CCF810B14FF030
:104B4000FF30C0E70120287194F83100C0F38000E5
:104B500028B902212846FFF7A3FF0020B3E720462B
:104B6000FEF77CFF06462EB12046FFF7C3FD4FF04F
:104B7000FF30A8E73046A6E76E6574696620213DE0
:104B8000204E554C4C0000006E65746966206973B8
:104B9000206E6F742075702C206F6C642073747994
:104BA0006C6520706F72743F00000000014679B19F
:104BB000486A68B14A6A50790A2805D050790528B0
:104BC00002D05079042801D1012070470020FCE771
:104BD0000020FAE770B505466C6A00BF00BF607937
:104BE000012805D060790A2802D06079052815D1FE
:104BF00000BF00BF2846FFF7EDFDA189628A881A31
:104C000000EBD0710122B2EB610F07DCA189628A4F
:104C1000881A00EBD071C1F34F01E18170BD70B50E
:104C200005466C6A00BF00BF6079012808D0607932
:104C30000A2805D06079052802D06079042815D1AA
:104C400000BF00BF2846FFF791FBA18A628A881A3D
:104C500000EBD0710122B2EB610F07DCA18A628AFE
:104C6000881A00EBD071C1F34F01218270BD70B57D
:104C700005466C6A00BF00BF60790C2802D06079DD
:104C8000062805D100BF00BF2846FEF7E7FE31E049
:104C90006079012811D100BF00BFA079052803DC8D
:104CA0002846FFF717FE25E000BF00BF2846FFF7A4
:104CB00021FD2846FFF7FCFE1CE0607908280CD196
:104CC00000BF00BFA079012803DC2846FEF7FCFCEA
:104CD00010E02846FEF750FC0CE06079032809D16B
:104CE000A079022803DA2846FFF7C2FB02E0284633
:104CF000FEF7B4FE70BD00000146002051B1CA7A33
:104D0000521C022A06DACA7A521C034B53F822209C
:104D100002B1012070470000BC0100202DE9F041E4
:104D200005460E46002428E004EB44003A4951F8B9
:104D3000200000B304EB440001EB8000007AA8429D
:104D400019D104EB4401344F07EB81014A6805EBAC
:104D50000511324F07EB011101F1100004EB440182
:104D60002D4F57F8213031469847002004EB44017D
:104D70003A4642F82100601CC4B2042CD4DB002463
:104D800021E0AC4200D11CE004EB0410234901EB0C
:104D90000010807A022813D104EB041001EB0010FC
:104DA000C07B05EB05111D4A02EB0111C97B88424E
:104DB00006D1042005EB051102EB0111C87304E0D4
:104DC00000BF601CC4B2042CDBDB00BF05EB051088
:104DD000124901EB0010C07B04281BDA05EB05111A
:104DE0000E4A02EB0111C97B0D4A52F8210012F064
:104DF00085FC002005EB0511084A02EB0111C97B77
:104E0000074A42F82100042005EB0511034A02EB92
:104E10000111C873BDE8F081105F0020D05A002056
:104E2000C05A002010B5002404E0204600F006F827
:104E3000601CC4B2042CF8DB10BD000070B506463F
:104E400006EB0610344901EB001400BF042E04DB0E
:104E500000BF32A0FEF73AF800BF00BFA07A0028DA
:104E60004ED0012804D0022815D0032849D13CE0B7
:104E700000F072F820810220A0720020E072012070
:104E8000207300206073304600F08EF805460DB1A7
:104E900000BF00BF3DE0207B401EC0B2207318BBA6
:104EA000607B401CC0B26073042814D12046FFF719
:104EB00023FF38B1E07A401CE0720120207300200B
:104EC00060730AE000BF00BF00213046FFF726FFF5
:104ED0000020A0721DE0607B2073304600F064F873
:104EE00005460DB100BF00BF13E0206818B120686F
:104EF000401E206018B900BF00BF0020A07208E06B
:104F000007E000BF00BF0CA0FDF7E0FF00BF00BF3F
:104F100000BF00BF70BD0000D05A002061727261F6
:104F20007920696E646578206F7574206F662062E1
:104F30006F756E6473000000756E6B6E6F776E2018
:104F4000646E735F7461626C6520656E7472792043
:104F500073746174653A000070B500BFFBF7D0F957
:104F600085B2002411E004EB04100A4901EB0010A3
:104F7000807A022807D104EB041001EB00100089AD
:104F8000A84200D1EAE7601CC4B2042CEBDB28463F
:104F900070BD0000D05A002000BF00BF00BF00BF9E
:104FA00000BF00BF704700002DE9F04F89B0834675
:104FB0000BEB0B10554901EB001500BF00BF00BF04
:104FC000E87A022804DB00BF51A0FDF77FFF00BF95
:104FD00000BFE87A544951F8200040B900215846F2
:104FE000FFF79CFE0020A87209B0BDE8F08F05F124
:104FF0001000FBF7C9F9123080B24FF4207201465D
:105000000290362009F01AFF0746002F73D00020C7
:10501000069007900890288906F053F8ADF818001C
:1050200001208DF81A000002ADF81C000C2206A920
:1050300038460AF0D7FC05F11004641E0C2600BFA8
:10504000641CA0464FF0000904E009F1010000F0E3
:10505000FF09641C20782E2802D020780028F4D183
:10506000A4EB080080B2049006EB0900401CB0F5E8
:10507000803F00DB43E04A46314638460AF099FB60
:10508000701C83B241463846049A0AF04DFD06EB87
:105090000900401C86B220780028D1D10022314678
:1050A00038460AF086FB701C86B24FF48070ADF86B
:1050B0001400ADF816003346042205A938460AF05C
:1050C00033FDE87B039000BF00BF35200190E97AF3
:1050D000154800EB81000290144A039952F8210010
:1050E0003946DDE9013212F079FB824638460AF092
:1050F0007BFA02E0FFE74FF0FF3A504674E738468C
:105100000AF072FA6FF005006EE70000D05A002036
:10511000646E7320736572766572206F7574206F8C
:105120006620617272617900BC010020C05A0020C3
:1051300002280ADA21B1054A0B6842F8203004E05F
:10514000024A034B1B6842F820307047BC01002024
:1051500054DB010810B500BF00BFFFF763FE10BDB0
:105160002DE9F04104460D4600BF05F0030020B1D3
:1051700000BF09A0FDF7AAFE00BF00BF2E460CF03D
:105180009BF90746E06800683060E06806603846D2
:105190000CF0F0F9BDE8F0816D656D705F667265C9
:1051A000653A206D656D2070726F7065726C792044
:1051B000616C69676E65640070B505460CF07CF93A
:1051C0000646E86804688CB12068E968086000BF9A
:1051D00004F0030020B100BF08A0FDF777FE00BF78
:1051E00000BF30460CF0C6F9204670BD30460CF0CA
:1051F000C1F900BF00BF0020F7E700006D656D70CA
:105200005F6D616C6C6F633A206D656D70207072BC
:105210006F7065726C7920616C69676E65640000FF
:105220002DE9F05F80460E46444600BF24B900BF1A
:1052300045A0FDF74BFE00BF00BF0CF03DF98346D3
:1052400000206060267294F8200040F0010084F88D
:10525000200065780020607058460CF08BF9A06A39
:1052600020B1002204212046A36A9847A06A20B1F9
:10527000002211462046A36A9847A06A20B1002266
:1052800002212046A36A9847304606F06FFD824609
:1052900004F1100030B1206920B1514604F1100032
:1052A0000CF0F4F904F1140030B1606920B15146FA
:1052B00004F114000CF0EAF9012D03D0042D01D003
:1052C000032D36D194F82000C0F3800900BF00BF41
:1052D00094F8200000F0FB0084F8200000BF00BF1D
:1052E000B9F1000F24D100BF606A20B900BF1AA035
:1052F000FDF7ECFD00BF00BF042D03D10020616A63
:10530000087101E0606A0671606A006800F10C07CC
:1053100000BF0FB1386820B900BF16A0FDF7D6FD59
:1053200000BF00BF0020606238460CF027FB00BFC2
:1053300008E000BF606A20B100BF15A0FDF7C6FD00
:1053400000BF00BFBDE8F09F636F6E6E20213D205F
:105350004E554C4C00000000636F6E6E2D3E637521
:105360007272656E745F6D736720213D204E554CDF
:105370004C000000696E61766C6964206F705F6339
:105380006F6D706C657465645F73656D000000001F
:10539000636F6E6E2D3E63757272656E745F6D73B2
:1053A00067203D3D204E554C4C0000000146002931
:1053B00002DC4842112801DB0520704702484A42BE
:1053C00050F82200F9E7000074D9010870B50546CD
:1053D000002411E004EB4400094901EBC000067D04
:1053E0004EB104EB440001EBC0008068A84202D13A
:1053F000204600F04FF9641C0A2CEBDB70BD000066
:10540000644E01202DE9FF5F0646894617464FF09E
:105410000A0AD346D04600240A20039000200290B6
:105420000190009000BF73E004EB4400724901EB6F
:10543000C000057DB8F10A0F04D11DB900BF00BF3F
:10544000A04663E0002D61D000BF012D06D0022DE3
:1054500004DA00BF69A0FDF739FD00BF00BFBEB18F
:1054600004EB4401644A02EBC10130684968884298
:105470000ED13FB104EB4400114601EBC00080683F
:10548000B84205D100BF00BF204604B0BDE8F09F80
:10549000012D28D104EB4400574951F8300080B168
:1054A00004EB440001EBC000418A029881422DDBED
:1054B000039404EB4400504901EBC000408A029081
:1054C00024E004EB44004C4901EBC000418A019800
:1054D00081421BDBA24604EB4400474901EBC000BC
:1054E000408A019012E0022D10DB04EB4400424997
:1054F00001EBC000418A0098814207DBA34604EB20
:1055000044003D4901EBC000408A0090601C04B299
:105510000A2C89DB09F0020028B9B8F10A0F07D17B
:1055200009F0010020B900BF00BF4FF0FF30ACE729
:10553000B8F10A0F02DA444600BF2FE0BBF10A0FB0
:105540000FDA5C4600BF00BF00BF04EB44002A49ED
:1055500051F8300020B100BF38A0FDF7B7FC00BF04
:1055600010E0BAF10A0F02DA544600BF0AE00398CD
:105570000A2802DA039C00BF04E000BF00BF4FF01E
:10558000FF3082E700BF0A2C04DB00BF31A0FDF72B
:105590009DFC00BF00BF204600F07CF800BF0A2C35
:1055A00004DB00BF2BA0FDF791FC00BF00BF00BFD4
:1055B00004EB4400104901EBC000007D20B100BFA6
:1055C00029A0FDF783FC00BF00BF36B104EB440106
:1055D000094A02EBC10130684860002004EB440135
:1055E000054A02EBC101488204EB4400114601EB7D
:1055F000C0008760204648E7644E012073746174E0
:1056000065203D3D204554484152505F535441541C
:10561000455F50454E44494E47207C7C2073746161
:105620007465203E3D204554484152505F535441DB
:1056300054455F535441424C450000006172705F15
:105640007461626C655B695D2E71203D3D204E5535
:105650004C4C000069203C204152505F5441424C68
:10566000455F53495A4500006172705F7461626C16
:10567000655B695D2E7374617465203D3D20455402
:10568000484152505F53544154455F454D50545921
:105690000000000010B5044604EB4400194951F81D
:1056A000300070B100BF00BF04EB4401154A52F84E
:1056B000310009F099FF002004EB4401114A42F83F
:1056C0003100002004EB44010E4A02EBC1010875D1
:1056D00004EB440102EBC101488204EB440102EBFC
:1056E000C101886004EB440102EBC101486004EB96
:1056F0004400114601EBC00003490A68C260898872
:10570000018210BD644E012062DB0108F0B587B054
:1057100007460D4600BF35B900BF35A0FDF7D6FBE3
:1057200000BF07B0F0BD00BF7C682088B0F5807F67
:1057300008D12079062805D16079042802D1608833
:10574000082805D000BF00BF384609F04DFFE8E744
:10575000D4F80E000690A0690590686808B9002684
:1057600007E005986968884201D1012000E0002027
:1057700006460EB1012000E00220034604F10802B3
:1057800006A9284600F0E6FBE088B0F5807F03D04C
:10579000B0F5007F22D11AE000BF00BF86B102221F
:1057A00006AB04F10800291DCDE90232CDE9001055
:1057B00005F12A0302462631284600F0A9FA05E041
:1057C000686808B900BF01E000BF00BF09E000BF82
:1057D00000BF06A92846FDF7A7FE02E000BF00BFF4
:1057E00000BF00BF384609F0FFFE00BF99E7000088
:1057F0006E6574696620213D204E554C4C000000BA
:105800002DE9FE4304460F461546A94600BF24B9BC
:1058100000BF57A0FDF75AFB00BF00BF00BF27B96C
:1058200000BF57A0FDF752FB00BF00BF00BF25B966
:1058300000BF56A0FDF74AFB00BF00BF2146286805
:1058400001F068F810B1DFF8548186E0287800F0A4
:10585000F000E02816D101208DF8040000208DF81A
:1058600005005E208DF80600687800F07F008DF856
:105870000700A8788DF80800E8788DF809000DF188
:10588000040869E02868A1680840D4E901121140C1
:1058900088420ED0288880B24FF6A961884208D08D
:1058A000E06810B104F10C0903E06FF00300BDE8FB
:1058B000FE833B48007800EB40003A4901EBC00012
:1058C000007D02281BDB3648007800EB400001EB2E
:1058D000C0008068A04212D13149097801EB410132
:1058E000304A02EBC101D9F800004968884206D16C
:1058F0002B4802783946204600F056F8D7E70026B4
:1059000022E006EB4600274901EBC000007D02289B
:1059100018DB06EB460001EBC0008068A04211D105
:1059200006EB46011F4A02EBC101D9F800004968A5
:10593000884207D11A48067032463946204600F0A0
:1059400033F8B4E7701CC6B20A2EDADB3A46494691
:10595000204600F0A9F8AAE700BF4FF400604346D4
:1059600004F12A0239460090204600F06FFC9EE7C1
:105970006E6574696620213D204E554C4C00000038
:105980007120213D204E554C4C000000697061642F
:10599000647220213D204E554C4C00005CDB010818
:1059A00084020020644E0120F8B505460E461446D8
:1059B00000BF04EB44002F4901EBC000007D02282A
:1059C00004DA00BF2CA0FDF781FA00BF00BF04EB92
:1059D0004400284901EBC000007D022839D104EBC6
:1059E000440001EBC000408AB0F58E7F11DD04EB6E
:1059F00044000A4602EBC000011D284600F014FADC
:105A000038BB032004EB44011A4A02EBC1010875BC
:105A10001FE004EB4400174901EBC000408AB0F5D9
:105A2000877F16DB04EB44000B4603EBC00000F15C
:105A30000C0204EB440003EBC000011D284600F0FB
:105A400001FA30B9032004EB44010A4A02EBC10118
:105A500008754FF40060009004EB4400054901EB29
:105A6000C00000F10C0305F12A023146284600F07F
:105A7000EDFBF8BD644E01206172705F7461626C71
:105A8000655B6172705F6964785D2E7374617465C3
:105A9000203E3D204554484152505F5354415445A7
:105AA0005F535441424C45002DE9FC5F81460F464F
:105AB000164609F12A0001904FF0FF3A4FF0000B13
:105AC0004946386800F026FF38B9387800F0F00011
:105AD000E02802D00FB1386828B900BF00BF6FF0CE
:105AE0000F00BDE8FC9F4A4601213846FFF78AFCBB
:105AF0008046B8F1000F07DA00BF00BF0EB100BF4B
:105B000000BF4FFA88F0ECE700BFB8F17F0F04D375
:105B100000BF65A0FDF7DAF900BF00BF08F0FF0481
:105B200004EB4400644901EBC000007D78B94FF0FC
:105B3000010B012004EB44015F4A02EBC10108752F
:105B400004EB4400114601EBC000C0F8089000BF10
:105B500004EB4400584901EBC000007D01280BD044
:105B600004EB440001EBC000007D022804DA00BF12
:105B700052A0FDF7ABF900BF00BFBBF1000F00D191
:105B8000F6B93946484600F04FF98246BAF1000F9F
:105B900013D104EB4400484901EBC000007D01280B
:105BA0000BD1BBF1000F08D100BF00BF002004EBF8
:105BB0004401414A02EBC10148820EB9504690E7C8
:105BC00000BF26B900BF47A0FDF780F900BF00BFA6
:105BD00004EB4400384901EBC000007D022811DBD2
:105BE000434804704FF40060009004EB440001EB64
:105BF000C00000F10C0331464846019A00F026FB34
:105C000082464FE004EB44002B4901EBC000007DCD
:105C1000012847D100200090354614E000BF688974
:105C20002989884206D1286820B100BF31A0FDF73C
:105C30004DF900BF00BF287B00F0400010B10120EB
:105C4000009002E02D68002DE8D100BF009838B127
:105C500032464FF420710E2009F0E8FA054603E0C1
:105C60003546284609F032FEBDB104EB4400124926
:105C700051F8300040B100BF00BF04EB44010E4AB0
:105C800052F8310009F0B0FC04EB44000A4941F835
:105C900030504FF0000A00BF03E000BF00BF4FF0DC
:105CA000FF3A00BF50461CE774797065206F766537
:105CB00072666C6F77000000644E01206172705F45
:105CC0007461626C655B695D2E7374617465203DFF
:105CD0003D2050454E44494E47206F722053544159
:105CE000424C45007120213D204E554C4C00000097
:105CF000840200206E6F207061636B657420717583
:105D00006575657320616C6C6F77656421000000B8
:105D10002DE9FC5F06460F4690469946DDE90CAB3F
:105D20000020019000BF26B900BF2DA0FDF7CEF8DE
:105D300000BF00BF4FF420721C210E2009F07EF836
:105D400005462DB900BF00BF4FF0FF30BDE8FC9FF6
:105D500000BF68891C2804DA00BF25A0FDF7B6F84B
:105D600000BF00BF6C6800BF00BF0F9805F0A9F925
:105D7000E08000BF96F83000062804D000BF294814
:105D8000FDF7A4F800BF00BFD9F80000A060B9F883
:105D90000400A081DBF80000C4F81200BBF8040086
:105DA000E082DAF80000C4F80E000E980068A061E6
:105DB0004FF480702080082060800620207104202D
:105DC000607140F6060043463A4629460090304648
:105DD00000F03CFA284609F007FC00250198B5E7D9
:105DE0006E6574696620213D204E554C4C000000C4
:105DF000636865636B20746861742066697273748C
:105E000020706275662063616E20686F6C64207319
:105E10007472756374206574686172705F6864720F
:105E200000000000E8E2010870B504460D4600BF1E
:105E300000BF034A2946204600F004F870BD000068
:105E40005CDB01087FB504460D4616460121074A72
:105E5000201D04F12A038DE82500039132461946DE
:105E60002046FFF755FF04B070BD000062DB01085B
:105E700070B500BF00BF002466E004EB4400344965
:105E800001EBC000057D002D5DD004EB440001EB6B
:105E9000C000408A401C04EB44012D4A02EBC101C2
:105EA000488204EB4400114601EBC000408AB0F583
:105EB000967F0DDA04EB440001EBC000007D012861
:105EC0000CD104EB440001EBC000408A052805DB3F
:105ED00000BF00BF2046FFF7DDFB34E004EB4400C9
:105EE0001B4901EBC000007D032807D1042004EB0F
:105EF0004401174A02EBC101087524E004EB440099
:105F0000134901EBC000007D042807D1022004EBF7
:105F100044010F4A02EBC101087514E004EB440090
:105F20000B4901EBC000007D01280CD104EB4402B9
:105F30000B4603EBC202111D04EB440203EBC20249
:105F40009068FFF771FF641C0A2C96DB70BD00009F
:105F5000644E01202DE9F84305460E461746984643
:105F600000BF95F83000062804D000BF2FA0FCF732
:105F7000ADFF00BF00BF00BF00BF5EB1306848B1D9
:105F80002946306800F0C6FC20B9307800F0F000F7
:105F9000E02805D100BF00BF6FF00F00BDE8F88317
:105FA0002A4641463046FFF72DFA0446002C01DA16
:105FB00060B2F3E7022004EB4401254A02EBC10181
:105FC000087504EB4400114601EBC000856000BF7A
:105FD00000BF04EB440001EBC0003968C160B98820
:105FE0000182002004EB440102EBC101488204EB72
:105FF0004400114651F83000B0B104EB440051F8B0
:106000003090002004EB440142F831004FF400606E
:106010003B4605F12A0249460090284600F016F951
:10602000484609F0E1FA00BF0020B7E76E657469E1
:10603000662D3E6877616464725F6C656E203D3DDD
:10604000204554485F4857414444525F4C454E00F8
:10605000644E012010B5112000F04AF9C0F38034DD
:10606000204610BD014600200A6802F0004252B9E5
:106070000A6802F4004232B90A6802F4807212B16E
:106080000A68C2F30D4070471CB51A4800788DF8B5
:106090000000184840788DF80100164880788DF887
:1060A00002001448C0788DF80300124800798DF87A
:1060B0000400104840798DF805000F480F4908602A
:1060C0000120486081030D488160C910C160002132
:1060D0000182C0F814D0012181610021C1614FF417
:1060E00000010162FAF734FF08B900201CBD01204D
:1060F000FCE70000644F012000800240F004002013
:106100002DE9F04104460E464FF00E0860890E2836
:1061100000DC59E0E07B18B996F83400401CE073CD
:10612000656800BF00BFAF89287800F00100B0B1FA
:106130002878012809D1687888B9A8785E280ED116
:10614000607B40F01000607309E006222149284678
:10615000FAF721F918B9607B40F008006073082F46
:1061600003D0B7F5C16F2AD114E096F8310000F0E2
:10617000080000B928E04146204609F0CBFB20B1D9
:1061800000BF00BF00BF00BF1EE03146204600F048
:1061900011FD15E096F8310000F0080000B913E099
:1061A0004146204609F0B6FB20B100BF00BF00BF4A
:1061B00000BF09E031462046FFF7A8FA00E003E0FF
:1061C00000BF0020BDE8F081204609F00DFA002054
:1061D000F8E700005CDB010810B51848006840B91A
:1061E0001748006828B91748006810B916480068B1
:1061F00008B1012000E00020E8B98021002007F06C
:10620000EBFC0E4908608021002007F0E5FC0C49FA
:10621000086041F2D071002007F0DEFC09490860F7
:1062200041F2D071002007F0D7FC0749086000BF99
:1062300000BF00BF00BF002010BD000030000020E4
:1062400034000020380000203C0000202DE9F047F9
:1062500005460E4617469846DDF82090484604F05D
:1062600030FF82460E21304608F096FD00B120E056
:106270007468A4F80CA0D8F800002060B8F80400F6
:10628000A0803868C4F80600B888608100BF95F81F
:106290003000062804D000BF08A0FCF717FE00BF9E
:1062A00000BF00BF00BF31462846AA699047BDE83D
:1062B000F08700BF00BF6FF00100F8E76E657469FA
:1062C000662D3E6877616464725F6C656E206D75E3
:1062D0007374206265203620666F7220657468656D
:1062E000726E65745F6F75747075742100000000C4
:1062F00038B504466A4621460248FBF7C7F80098BD
:1063000038BD0000F004002070B5044600BF24B979
:1063100000BF11A0FCF7DAFD00BF00BF042007F0AA
:10632000F1F8054625B900BF00BF4FF0FF3070BD42
:106330002562652084F832006E21332001550A4819
:1063400060610A48A06104F12A002860204604F038
:1063500025FC0020EBE700006E6574696620213D96
:10636000204E554C4C0000000158000855AD000867
:10637000054600262C4600BF00BF27E04FF0FF3146
:106380001348006813F09EFD01281FD112F05CFC39
:1063900000BF204604F060FC064612F0A1FCAEB13E
:1063A00012F052FC214630462269904730B100BFBE
:1063B00000BF304609F018F9002605E00021044826
:1063C000006813F07FFDE4E712F08AFCD6E70000D6
:1063D000900200202DE9F84F05460E46DDB1AF6969
:1063E000002F12DA0BF068F88146A869002808DA55
:1063F00016B9A869401EA86148460BF0BBF8BDE875
:10640000F88FAF6948460BF0B5F8384600F090F8C1
:1064100004460CB9F3E7F2E74FF001080BF04CF833
:106420008146052E24D2DFE806F0030E151C20005D
:106430002089401C00B22081B4F90800012801DD48
:106440004FF000081CE02089401E00B220814FF070
:10645000000815E0608908B14FF000080120608154
:106460000EE00020608180460AE00120A08107E064
:1064700000BF00BF17A0FCF729FD00BF00BF00BF91
:1064800000BFA07B00B3B8F1000F1DD0B4F9080025
:10649000002801DD012000E000208246608908B16B
:1064A000012000E000208346A08908B1012000E01F
:1064B0000020009048460BF05DF85A465146384699
:1064C000009B0AF0C7FC02E048460BF053F800BFFF
:1064D00095E70000756E6B6E6F776E206576656E62
:1064E0007400000000BF054A126802F04002002A52
:1064F000F9D0C2B2014B5A60704700000010014051
:106500001CB50648052100238022CDE9001004A116
:10651000064813F05BFE12F0C7FF1CBD040000200C
:1065200073746172745F7461736B00001D120108F3
:1065300070B50446204610F0DDFD054665B9002C17
:1065400001DB042C01DB00BF00BF00BF09200349B1
:10655000086000BF002070BD2846FCE798020020BC
:1065600070B505460C4622460321284600F02EF958
:1065700070BD00002DE9F04F85B004468A4677488B
:1065800080680390039800780007860E142E02DAC4
:1065900000BF00BFD9E06089042802D200BF00BF5D
:1065A000D3E06068057860684078049015B1082DE4
:1065B00072D100E0C4E0DFF8A49109F11409674842
:1065C000007D00F0F000E02802D100BF00BFC0E075
:1065D000624A1168506900F09DF910B100BF00BF18
:1065E000B7E000BF00BF2089082802D200BF00BF6B
:1065F000ABE0204600F063F938B100BF00BF204691
:1066000008F0F2FF05B0BDE8F08F06F10E0120465C
:1066100008F0C2FB002845D0208930441FFA80FBD7
:106620002089584502DD00BF00BF92E04FF4207280
:1066300059460E2008F002FC074617B900BF00BFFC
:1066400087E0798906F10800814205D200BF00BFCA
:10665000384608F0C9FF7CE0324678680399F9F7BC
:1066600061FE3146384609F055F950B100BF00BF10
:106670003BA0FCF72BFC00BF00BF384608F0B4FF7E
:1066800067E02146384608F0F9FD30B100BF00BF91
:10669000384608F0A9FF5CE03EE0204608F0A4FF81
:1066A0003C460DE006F10E01204609F033F938B101
:1066B00000BF00BF38A0FCF709FC00BF00BF48E0E6
:1066C000D4F804803146204608F066FB08B100BFCC
:1066D00021E06768D9F80000F86020480069386157
:1066E000002088F80000A8F80200FF20387200207F
:1066F000788101200021FF230A46CDE9010A00919B
:106700004946204600F078FB8346BBF1000F01D0DC
:1067100000BF00BF00BF13E0032D0ED00B2D0CD027
:106720000C2D0AD0042D08D0052D06D00D2D04D037
:106730000E2D02D0112D00D000BF00BF00BF00BF42
:1067400000BF204608F050FF5CE7204608F04CFFF1
:1067500058E7204608F048FF00BF53E7405F00209D
:1067600069636D705F696E7075743A206D6F7669DC
:106770006E6720722D3E7061796C6F616420746F5A
:106780002069636D70206865616465722066616967
:106790006C65640A0000000069636D705F696E706B
:1067A00075743A20726573746F72696E67206F72C8
:1067B0006967696E616C20702D3E7061796C6F61E4
:1067C00064206661696C65640A0000002DE9FF5F62
:1067D0000646894692464FF01C083089404501DA4A
:1067E000B6F8088008F1080081B24FF42072222028
:1067F00008F024FB04461CB900BF00BFBDE8FF9FA2
:1068000000BF618908F10800814204D200BF1CA0CA
:10681000FCF75CFB00BF00BFD6F804B000BF00BFB0
:1068200000BF00BF00BF00BF00BF00BF00BF00BF70
:10683000656885F8009085F801A00020A880E880B0
:106840007168626802F108004246F9F76BFDDBF8F7
:106850000C00039003A800F0D7FC07465FB10020AE
:10686000688001200021FF2303AACDE901070091E0
:10687000204600F0C1FA204608F0B6FE00BFBDE792
:10688000636865636B2074686174206669727374F1
:1068900020706275662063616E20686F6C64206989
:1068A000636D70206D6573736167650070B5054633
:1068B0000C4622460B212846FFF788FF70BDF0B535
:1068C000064600270024354619E06989686806F005
:1068D00087FB0444A0B200EB1444688900EBD0713C
:1068E0004910A0EB410149B10FB9012000E000209F
:1068F0000746E0B2C4F3072141EA00242D68002DC9
:10690000E3D127B1E0B2C4F3072141EA0024E04318
:1069100080B2F0BD18B502460092D04300B10AB96A
:10692000012018BD91F8310000F0020008B90020E4
:10693000F7E74868904201D10020F2E700988B68A1
:106940001840D1E901342340984208D1886822EAEE
:1069500000008C68E343984201D10120E1E7002068
:10696000DFE700002DE9F74F8CB004460F464FF0EB
:106970000008398DA1F11400C11700EB5171C1F36A
:10698000CF0A1420059060680990DDF8249099F8EA
:10699000000000F00F001421B1EB800F04D06FF065
:1069A00005000FB0BDE8F08F00BF6089142807DA3A
:1069B00000BF6CA0FCF78AFA00BF6FF00500F0E79B
:1069C00000BFB9F8060004F07CFB04900498C0F303
:1069D0000C000790049800F40050039020891438AC
:1069E0001FFA80FBB5E04FF6FF7000EACA00584579
:1069F00001DD584603E04FF6FF7000EACA00089038
:106A00004FF4207214210E2008F018FA054605B93B
:106A1000A5E000BF6889142804DA00BF58A0FCF77D
:106A200055FA00BF00BF142268680999F9F77AFC8B
:106A3000D5F8049008980A9050E061890598081AE2
:106A400080B2029000BF61890598814204DA00BFDC
:106A500053A0FCF73BFA00BF00BF02990A98884296
:106A600001DA0A9800E002988046B8F1000F03D1DD
:106A700000200590246831E000F04AFD06461EB96A
:106A8000284608F0B1FD6AE061680598084433467D
:106A900041224146CDE90008002008F015FB0B908B
:106AA0000B9830B9304600F039FD284608F09CFDBF
:106AB00055E0204608F00AFF74613D4830612846E1
:106AC0000B9908F02FFB0A98A0EB080080B20A90FF
:106AD0000A9810B100200590246800BF0A98002889
:106AE000ABD10598404480B20590388D1438584594
:106AF00001DB012000E0002006900798C0F30C00A5
:106B00000490069808B1039818B1049840F4005016
:106B10000490049804F0D5FAA9F8060008991431F5
:106B200088B204F0CEFAA9F802000020A9F80A0001
:106B30007B69294638460E9A9847284608F054FD46
:106B40000898ABEB00001FFA80FB0798504480B216
:106B50000790BBF1000F7FF446AF002021E74FF014
:106B6000FF301EE76970345F6672616728293A203A
:106B70007062756620746F6F2073686F72740000A6
:106B800074686973206E6565647320612070627536
:106B90006620696E206F6E652070696563652100EF
:106BA000702D3E6C656E203E3D20706F6666000065
:106BB000A17A00082DE9F04706460F464FF0010A7A
:106BC000756828780421B1EB201F07D000BF00BFF3
:106BD000304608F009FD0020BDE8F087287800075E
:106BE0004FEA9068688804F06CFA8146318949451B
:106BF00003DD4946304608F0F1FD7089404505DB6C
:106C00003089484502DBB8F1140F13DAB8F1140FDC
:106C100001DA00BF00BF7089404501DA00BF00BF44
:106C20003089484501DA00BF00BF304608F0DCFC7F
:106C30000020D1E728695F494861E8680861084693
:106C4000007D00F0F000E0280AD197F8310000F054
:106C5000010018B1786808B13C461CE000241AE035
:106C6000384600F0ABF808B13C4614E00024514827
:106C7000007D7F280FD05048046809E0BC4200D155
:106C800005E0204600F09AF800B103E000BF246858
:106C9000002CF3D100BF84B9687A11280DD105EB1F
:106CA000080000BF00BF4188B1F5884F04D100BF84
:106CB00000BF3C464FF0000A00BFBAF1000F15D0EC
:106CC0003C48006990B13B4908693946FFF722FE0C
:106CD00028B93848007C00F0F000E02806D100BF59
:106CE00000BF304608F080FC002075E734B900BFD3
:106CF00000BF304608F078FC00206DE7E8884FF6CA
:106D00003F71084048B100BF00BF304600F030F985
:106D100006460EB900205FE7756800BF00BF00BFE0
:106D200000BF244804604760856028780007800E13
:106D3000204988814146304608F0ECFD687A0128F8
:106D40000DD0062806D011280ED13946304610F055
:106D5000EBFA24E0394630460BF0F0FD1FE03946EF
:106D60003046FFF707FC1AE0124948692146FFF751
:106D7000D1FD70B90F48007D00F0F000E02808D088
:106D80000FFA88F1304608F0EBFC02213046FFF79D
:106D9000E7FB00BF00BF304608F026FC00BF00BF85
:106DA0000020044908604860886088810861486163
:106DB00000BF11E7405F00200C02002010B5044620
:106DC00000BF00BF94F8310000F0010080B160689E
:106DD00070B1084840696168884205D00549486932
:106DE0002146FFF797FD18B100BF00BF012010BD7D
:106DF0000020FCE7405F00202DE9FE4F07460C46CF
:106E000015469846DDE90C9A0E9EA34625B10CB1B5
:106E1000206808B906F1040B43462A46594638460D
:106E2000CDE9009A029600F003F8BDE8FE8F00005D
:106E30002DE9F84F05460F4690469A46DDF828B0F2
:106E40000C9E00BFA87B012804D000BF37A0FCF730
:106E50003DF800BF00BFB8F1000F44D04FF0140957
:106E60001421284607F098FF28B100BF00BF6FF03B
:106E70000100BDE8F88F6C6800BF6889142804D24F
:106E800000BF2DA0FCF722F800BF00BF84F808A0C7
:106E90000B986072D8F80000206148464FEAE9710B
:106EA00009EB9171C1F3870141F04001217084F831
:106EB00001B0288904F005F960800020E0802A48AC
:106EC000008804F0FEF8A08027480088401C26496E
:106ED00008801FB925480068E06001E03868E0607C
:106EE000002060810BE06889142804DA00BF00BF2D
:106EF0006FF00100BDE76C6820690090E84600BFB4
:106F000000BF308D48B12889318D884205DD424669
:106F100031462846FFF726FDABE700BF00BF4246DB
:106F20002946304673699847A3E70000702D3E72EA
:106F30006566203D3D203100636865636B207468A1
:106F40006174206669727374207062756620636173
:106F50006E20686F6C64207374727563742069703E
:106F60005F686472000000008602002054DB0108A4
:106F70002DE9F14F84B004984568287800F00F009F
:106F80001421B1EB800F02D000BF00BF0DE1E888F3
:106F900004F097F8C0F30C004FF6FF7101EAC00A45
:106FA000688804F08EF8074628780007810E029161
:106FB0000299B94200DDF8E00298381A87B20498C5
:106FC00008F02BF906467C48018888190A280CDD50
:106FD0003146284600F0F6FC20B17748008830445E
:106FE0000A2802DD00BF00BFDFE07448046813E038
:106FF0006069E968884209D1A0692969884205D198
:10700000A089A988884201D1012000E0002010B1A8
:1070100000BF00BF02E02468002CE9D100BF34B9F2
:107020003146284600F0F4FB044694B9BDE0E888F8
:1070300004F047F8C0F30C0058B9E08904F041F8B7
:10704000C0F30C0028B11422294604F10800F9F716
:1070500069F9E888012121EA50100190019850B1A6
:107060000AEB070188B2504503DB4FF6EB7188420B
:1070700000DD80E000BF2046019A049900F064FA28
:1070800083460BF1010000B975E04B48008830449D
:1070900049490880019850B10AEB070188B2A083E2
:1070A000A17F41F00101A17700BF00BF00BFBBF18C
:1070B000010F5CD1A08B143080B2009060684068F2
:1070C000D0F8009060684568142204F10801284651
:1070D000F9F728F9009803F0F4FF68800020E880B1
:1070E0006881606804900DE0D9F8040003901421D1
:1070F000484608F00FFC4946049808F013F8039836
:10710000D0F80090B9F1000FEED12C48006884420D
:1071100002D14FF000080EE02848D0F8008006E0C9
:10712000D8F80000A04200D104E0D8F80080B8F1FF
:10713000000FF5D100BF4146204600F03FFB049808
:1071400008F06BF8064600BF1B480088B04204DA1E
:1071500000BF1BA0FBF7BAFE00BF00BF16480088A7
:10716000801B15490880049805B0BDE8F08F00BF6A
:1071700000BF0020F8E700BF24B900BF17A0FBF74D
:10718000A5FE00BF00BF606870B900BF0B48006873
:10719000844204D000BF14A0FBF798FE00BF00BFDC
:1071A0000021204600F00AFB00BF00BF00BF04988A
:1071B00008F01AFA0020D7E78C020020880200208D
:1071C00069705F72656173735F70627566636F7516
:1071D0006E74203E3D20636C656E00006970722005
:1071E000213D204E554C4C006E6F742066697273C1
:1071F00074616C74686F756768206A757374206554
:107200006E7175657565640010B5024622480168A7
:1072100021E091F8310000F00100D8B191F831007F
:10722000C0F38000B0B14868A0B110688B68184006
:10723000D1E901342340984201D1084610BD91F8AC
:10724000310000F0020028B91068CB68984201D1E3
:107250000846F3E709680029DBD110480068A0B1AF
:107260000E48006890F8310000F0010068B10B484A
:10727000006890F83100C0F3800030B10748006822
:10728000406810B110787F2803D100BF00BF0020F4
:10729000D4E702480068D1E70C0200201002002069
:1072A0002DE9FF47064688466F46347800BFF9F758
:1072B00023F80068005D202803D0002004B0BDE85A
:1072C000F08700254FF00A09302C0ED1701C0646BD
:1072D0000478782C01D0582C05D14FF01009701C7F
:1072E0000646047801E04FF0080900BFF9F704F8FA
:1072F0000068005D20280FD1B9F1080F04D1A4F176
:107300003000082800D328E0A4F1300005FB09056F
:10731000701C06460478E9E7B9F1100F1CD1F8F7A4
:10732000EBFF006810F804A08AEA8A0000F08000F1
:1073300090B1F8F7E1FF0068005D00F0080008B1C7
:10734000612100E0412104F10A00401A40EA0515DC
:10735000701C06460478C9E700BF00BF2E2C09D177
:1073600003A8874201D30020A8E720C7701C064667
:1073700004789CE700BF00BF44B1F8F7BDFF006888
:10738000005D00F0010008B9002097E76846381A50
:10739000012101EBA000052842D2DFE800F003053F
:1073A00006142800002089E742E0B5F1807F01D370
:1073B000002083E70098FF2801D900207EE700988D
:1073C00045EA006534E0B5F5803F01D3002075E75C
:1073D0000098FF2802D80198FF2801D900206DE706
:1073E00000980006019940EA0140054320E0FF2D86
:1073F00001D9002062E70098FF2805D80198FF28EE
:1074000002D80298FF2801D9002057E7009800060B
:10741000019940EA0140029940EA0120054307E052
:1074200000BF00BF08A0FBF751FD00BF00BF00BFB9
:1074300000BFB8F1000F04D0284603F035FEC8F8AD
:10744000000001203AE70000756E68616E646C65AB
:107450006400000010B5044610220249204600F0E6
:1074600003F810BD544F01202DE9FC4706460B469A
:1074700014464FF0000C30680190194601AA00270D
:107480003CE0002500BF10784FF00A0990FBF9FAA4
:1074900009FB1A0000F0FF08107890FBF9F010705B
:1074A00008F1300000F0FF0A284605F1010909F053
:1074B000FF050DF800A010780028E4D10BE060462D
:1074C0000CF1010CA04202DB0020BDE8FC871DF896
:1074D000050001F8010B281EA5F1010909F0FF05BF
:1074E000EDD160460CF1010CA04201DB0020ECE77D
:1074F0002E2001F8010B521C781CC7B2042FC0DBF0
:107500004FF00009481E014680F800901846DCE75D
:1075100010B5052006F05AFA10BD000010B504465B
:1075200000BF24B900BF05A0FBF7D0FC00BF00BF1F
:107530002146052006F0FCF910BD00007020213D19
:10754000204E554C4C0000002DE9F74F84B0064604
:107550008846002501200190D8F804000290029985
:10756000488803F0AEFD8346029800780007800E3D
:1075700003900398584503DD681E07B0BDE8F08FFF
:107580000398ABEB00001FFA80FB0299C88803F058
:1075900098FDC0F30C004FF6FF7101EAC00A00BF6E
:1075A00000BFD8F8044000202060A4F804A00AEB33
:1075B0000B00E080E088504502DA4FF0FF30DCE756
:1075C000D6F804903EE0D9F80470A088B9888842C3
:1075D00020DAC4F800909DB1A088E988884203DBD6
:1075E000E088B988884202DD4FF0FF30C5E7C5F872
:1075F0000080E888A18888420BD00020019008E034
:10760000E088B988884202DD4FF0FF30B5E7C6F860
:1076100004801AE0A088B988884202D14FF0FF3078
:10762000ABE7A088F988884202DA4FF0FF30A4E780
:107630002DB1E888B988884201D000200190D7F8A0
:1076400000903D46B9F1000FBDD100BFB9F1000F68
:107650001FD19DB100BFE888A188884204DD00BF2A
:1076600033A0FBF733FC00BF00BFC5F80080E888FB
:10767000A18888420DD0002001900AE000BF706808
:1076800020B100BF32A0FBF721FC00BF00BFC6F84D
:107690000480069820B9B07F00F00100002844D093
:1076A000019800283BD0706818B1706840688088E5
:1076B00010B10020019032E02546D4F800900BE094
:1076C000D9F80440E888A188884202D000200190BF
:1076D00005E02546D4F80090B9F1000FF0D100BFC5
:1076E0000198E0B100BF706820B900BF26A0FBF789
:1076F000EDFB00BF00BF00BF70684068A04204D12E
:1077000000BF21A0FBF7E2FB00BF00BF00BF206865
:1077100020B100BF20A0FBF7D9FB00BF00BF01983C
:1077200008B1012029E7002027E7002025E7000015
:10773000636865636B20667261676D656E74732044
:10774000646F6E2774206F7665726C617000000044
:107750006E6F2070726576696F75732066726167EF
:107760006D656E742C2074686973206D7573742058
:107770006265207468652066697273742066726140
:10778000676D656E7421000073616E6974792063A2
:107790006865636B0000000076616C696461746504
:1077A0005F646174616772616D3A6E6578745F7071
:1077B000627566213D4E554C4C00000070B5044684
:1077C0000D460B480068A04203D1094920680860B3
:1077D00009E000BF25B900BF06A0FBF777FB00BF9B
:1077E00000BF206828602146042006F0A1F870BD83
:1077F0008802002073616E69747920636865636B29
:10780000206C696E6B6564206C6973740000000005
:1078100070B505460E46042006F0D8F8044674B943
:107820003146284600F0CEF8B04203DB042006F0D3
:10783000CDF804461CB900BF00BF002070BD202158
:107840002046F8F796FD0F20E07706480068206094
:10785000044804601422294604F10800F8F762FD88
:107860002046EBE7880200202DE9F04704468846D1
:10787000002500BFA04504D100BF38A0FBF726FBC0
:1078800000BF00BFB8F1000F0AD000BFD8F8000059
:10789000A04204D000BF34A0FBF718FB00BF00BF1C
:1078A0006068D0F80490B9F8040008BB6768D9F89C
:1078B00000006060142204F108017868F8F732FDD6
:1078C00001213846FEF7F2FF384607F0A6FC0646CF
:1078D00000BFA819B0F5803F04DB00BF27A0FBF76D
:1078E000F5FA00BF00BFA81985B2384607F07CFE44
:1078F000676819E0D7F80490BA46D9F80070504686
:1079000007F08BFC064600BFA819B0F5803F04DBEA
:1079100000BF1AA0FBF7DAFA00BF00BFA81985B2B2
:10792000504607F061FE00BF002FE3D141462046DC
:10793000FFF744FF00BF19480088A84204DA00BFDF
:1079400017A0FBF7C3FA00BF00BF14480088401B14
:10795000124908802846BDE8F087000070726576FD
:1079600020213D2069707200707265762D3E6E6533
:107970007874203D3D206970720000007062756669
:10798000735F6672656564202B20636C656E203CB6
:107990003D20307866666666000000008C0200209C
:1079A00069705F72656173735F70627566636F752E
:1079B0006E74203E3D2070627566735F6672656509
:1079C000640000002DE9F84F05468946002700BFF6
:1079D0000026B2460020009083461B48046821E040
:1079E0006069E968884207D1A0692969884203D1A2
:1079F000A089A988884201D0012000E0002068B158
:107A00000BF1010B1EB92646CDF800A006E0E07F81
:107A1000F17F884202DC2646CDF800A0206800B144
:107A2000A2462468002CDBD12EB130460099FFF726
:107A30001BFF804647444F4502DABBF1010FC7DC0C
:107A40003846BDE8F88F00008802002070B5002697
:107A50000C48046813E0E07F002807DDE07F401E4B
:107A6000E07700BF00BF2646246808E000BF00BFE3
:107A70002546246831462846FFF7F6FE00BF002C55
:107A8000E9D170BD8802002038B504466946204619
:107A9000FFF706FC08B1009838BD4FF0FF30FBE758
:107AA00070B505462C4600BF24B900BF0BA0FBF7FC
:107AB0000DFA00BF00BF00BFAC4204D000BF0AA057
:107AC000FBF704FA00BF00BF606910B1606907F0FE
:107AD0008BFD2046FFF722FD70BD00007063722011
:107AE000213D204E554C4C00706372203D3D20706E
:107AF0000000000000B587B000BF00BF002001906B
:107B00003848006840F010003649086008460068B0
:107B100000F01000019000BF00BF00BF00BF00BF19
:107B2000002001900846006840F0100008600846F8
:107B3000006800F01000019000BF00BF00BF00BF50
:107B400000BF002001900846006840F01000086067
:107B50000846006800F01000019000BF00BF00BFA1
:107B600000BF00BF002001900846006840F00100FF
:107B700008600846006800F00100019000BF00BFE7
:107B800000BF1020029000200390012004900220EA
:107B9000059002A91448F9F7FBFD08200290002087
:107BA0000390012004900220059002A90E48F9F7E5
:107BB000EFFD042002900020039001200490022099
:107BC000059002A90848F9F7E3FD01200290002082
:107BD000039002200490059002A90448F9F7D8FD0B
:107BE00007B000BD303802400010024000000240E3
:107BF00070B50446002609480588408845430021A1
:107C0000084602F0ADFD02F059FF00BF02E0044853
:107C10000480761CAE42FAD370BD000090040020B0
:107C20008000006C10B5044649488471002C45D191
:107C3000F020474908804FF4A070488008468088AB
:107C400045F21051884210D14FF43050404908811C
:107C50004FF4285048814FF42C5088814FF4F07035
:107C600008804FF4487048801AE03948808841F60F
:107C7000631188420DD12C20354908812B20488181
:107C80002A2088814FF4F07008804FF448704880B3
:107C900006E02C202E4908812A2048812B2088814B
:107CA0002B48808845F2103188424CD14FF4A070A7
:107CB000274908804FF4F070488044E04FF4A070EA
:107CC00023490880F02048800846808845F21051FA
:107CD000884210D14FF430501D4908814FF428508C
:107CE00048814FF42C5088814FF4487008804FF43D
:107CF000F07048801AE01648808841F66311884287
:107D00000DD12C20124908812A2048812B208881FE
:107D10004FF4487008804FF4F070488006E02C2043
:107D20000B4908812A2048812B20888108488088B7
:107D300045F21031884206D14FF4F07004490880B2
:107D40004FF4A0704880002002F0F2FB10BD00004C
:107D50009004002070B505460E461446314628466C
:107D600002F0FEFC02F0AAFE01490C8070BD00008A
:107D70008000006C10B5CF2002F094FE002002F0CD
:107D800085FEC12002F082FE302002F07FFEED2051
:107D900002F088FE642002F079FE032002F076FEF5
:107DA000122002F073FE812002F070FEE82002F043
:107DB00079FE852002F06AFE102002F067FE7A202C
:107DC00002F064FECB2002F06DFE392002F05EFE70
:107DD0002C2002F05BFE002002F058FE342002F05E
:107DE00055FE022002F052FEF72002F05BFE20203A
:107DF00002F04CFEEA2002F055FE002002F046FEA2
:107E0000002002F043FEC02002F04CFE1B2002F0D6
:107E10003DFEC12002F046FE012002F037FEC520E3
:107E200002F040FE302002F031FE302002F02EFE43
:107E3000C72002F037FEB72002F028FE362002F0FD
:107E400031FE482002F022FE3A2002F02BFE55209F
:107E500002F01CFEB12002F025FE002002F016FE0A
:107E60001A2002F013FEB62002F01CFE0A2002F0D7
:107E70000DFEA22002F00AFEF22002F013FE002006
:107E800002F004FE262002F00DFE012002F0FEFDAD
:107E9000E02002F007FE0F2002F0F8FD2A2002F099
:107EA000F5FD282002F0F2FD082002F0EFFD0E2083
:107EB00002F0ECFD082002F0E9FD542002F0E6FD9E
:107EC000A92002F0E3FD432002F0E0FD0A2002F0C9
:107ED000DDFD0F2002F0DAFD002002F0D7FD0020CA
:107EE00002F0D4FD002002F0D1FD002002F0CEFD12
:107EF000E12002F0D7FD002002F0C8FD152002F0BD
:107F0000C5FD172002F0C2FD072002F0BFFD1120C1
:107F100002F0BCFD062002F0B9FD2B2002F0B6FDF8
:107F2000562002F0B3FD3C2002F0B0FD052002F027
:107F3000ADFD102002F0AAFD0F2002F0A7FD3F20AA
:107F400002F0A4FD3F2002F0A1FD0F2002F09EFDF3
:107F50002B2002F0A7FD002002F098FD002002F087
:107F600095FD012002F092FD3F2002F08FFD2A20B6
:107F700002F098FD002002F089FD002002F086FD4D
:107F8000002002F083FDEF2002F080FD112002F0BE
:107F900089FD7820FBF798FA292002F083FD10BDB7
:107FA00010B5ED2002F07EFD012002F06FFDFE20F5
:107FB00002F06CFDEE2002F075FDDE2002F066FDA1
:107FC000212002F063FDF12002F06CFD012002F09F
:107FD0005DFDDF2002F066FD102002F057FDC42099
:107FE00002F060FD8F2002F051FDC62002F05AFD24
:107FF000002002F04BFDE22002F048FDE22002F0FA
:1080000045FDE22002F042FDBF2002F04BFDAA2018
:1080100002F03CFDB02002F045FD0D2002F036FDDF
:10802000002002F033FD0D2002F030FD002002F0B0
:108030002DFD112002F02AFD002002F027FD19205D
:1080400002F024FD002002F021FD212002F01EFD9F
:10805000002002F01BFD2D2002F018FD002002F090
:1080600015FD3D2002F012FD002002F00FFD5D2005
:1080700002F00CFD002002F009FD5D2002F006FD7B
:10808000002002F003FDB12002F00CFD802002F080
:10809000FDFC002002F0FAFC8B2002F0F7FC00202F
:1080A00002F0F4FC962002F0F1FC002002F0EEFC5D
:1080B000B22002F0F7FC002002F0E8FC002002F001
:1080C000E5FC022002F0E2FC002002F0DFFC0320CD
:1080D00002F0DCFC002002F0D9FCB32002F0E2FC4C
:1080E000002002F0D3FC002002F0D0FC002002F0BF
:1080F000CDFC002002F0CAFC002002F0C7FC0020EA
:1081000002F0C4FC002002F0C1FC002002F0BEFC22
:10811000002002F0BBFC002002F0B8FC002002F0BE
:10812000B5FC002002F0B2FC002002F0AFFC002001
:1081300002F0ACFC002002F0A9FC002002F0A6FC3A
:10814000002002F0A3FC002002F0A0FC002002F0BE
:108150009DFC002002F09AFC002002F097FC002019
:1081600002F094FC002002F091FC002002F08EFC52
:10817000B42002F097FC8B2002F088FC002002F073
:1081800085FC962002F082FC002002F07FFCA120FA
:1081900002F07CFC002002F079FCB52002F082FCA9
:1081A000022002F073FC002002F070FC032002F0B9
:1081B0006DFC002002F06AFC042002F067FC002045
:1081C00002F064FCB62002F06DFC002002F05EFCC0
:1081D000002002F05BFCB72002F064FC002002F0FB
:1081E00055FC002002F052FC3F2002F04FFC002022
:1081F00002F04CFC5E2002F049FC002002F046FC3C
:10820000642002F043FC002002F040FC8C2002F0CD
:108210003DFC002002F03AFCAC2002F037FC0020CC
:1082200002F034FCDC2002F031FC002002F02EFCD5
:10823000702002F02BFC002002F028FC902002F0BD
:1082400025FC002002F022FCEB2002F01FFC0020A5
:1082500002F01CFCDC2002F019FC002002F016FCED
:10826000B82002F01FFC002002F010FC002002F0F9
:108270000DFC002002F00AFC002002F007FC0020A8
:1082800002F004FC002002F001FC002002F0FEFBE2
:10829000002002F0FBFBBA2002F004FC242002F0D4
:1082A000F5FB002002F0F2FB002002F0EFFB0020C3
:1082B00002F0ECFBC12002F0F5FB202002F0E6FB0F
:1082C000002002F0E3FB542002F0E0FB002002F06B
:1082D000DDFBFF2002F0DAFB002002F0D7FBC2201A
:1082E00002F0E0FB0A2002F0D1FB002002F0CEFBFE
:1082F000042002F0CBFB002002F0C8FBC32002F0F8
:10830000D1FB3C2002F0C2FB002002F0BFFB3A2070
:1083100002F0BCFB002002F0B9FB392002F0B6FBF2
:10832000002002F0B3FB372002F0B0FB002002F087
:10833000ADFB3C2002F0AAFB002002F0A7FB362098
:1083400002F0A4FB002002F0A1FB322002F09EFB11
:10835000002002F09BFB2F2002F098FB002002F08F
:1083600095FB2C2002F092FB002002F08FFB2920CD
:1083700002F08CFB002002F089FB262002F086FB35
:10838000002002F083FB242002F080FB002002F09A
:108390007DFB242002F07AFB002002F077FB2320F3
:1083A00002F074FB002002F071FB3C2002F06EFB37
:1083B000002002F06BFB362002F068FB002002F088
:1083C00065FB322002F062FB002002F05FFB2F20F1
:1083D00002F05CFB002002F059FB2C2002F056FB5F
:1083E000002002F053FB292002F050FB002002F095
:1083F0004DFB262002F04AFB002002F047FB242020
:1084000002F044FB002002F041FB242002F03EFB7E
:10841000002002F03BFB232002F038FB002002F09A
:1084200035FBC42002F03EFB622002F02FFB00204F
:1084300002F02CFB052002F029FB002002F026FBB5
:10844000842002F023FB002002F020FBF02002F049
:108450001DFB002002F01AFB182002F017FB002081
:1084600002F014FBA42002F011FB002002F00EFB2E
:10847000182002F00BFB002002F008FB502002F055
:1084800005FB002002F002FB0C2002F0FFFA0020A6
:1084900002F0FCFA172002F0F9FA002002F0F6FAD6
:1084A000952002F0F3FA002002F0F0FAF32002F037
:1084B000EDFA002002F0EAFAE62002F0E7FA0020E6
:1084C00002F0E4FAC52002F0EDFA322002F0DEFA02
:1084D000002002F0DBFA442002F0D8FA002002F07B
:1084E000D5FA652002F0D2FA002002F0CFFA762009
:1084F00002F0CCFA002002F0C9FA882002F0C6FA95
:10850000002002F0C3FAC62002F0CCFA202002F0CC
:10851000BDFA002002F0BAFA172002F0B7FA0020E4
:1085200002F0B4FA012002F0B1FA002002F0AEFA33
:10853000C72002F0B7FA002002F0A8FA002002F0EB
:10854000A5FA002002F0A2FA002002F09FFAC8204B
:1085500002F0A8FA002002F099FA002002F096FA40
:10856000002002F093FA002002F090FAC92002F0F5
:1085700099FA002002F08AFA002002F087FA00201F
:1085800002F084FA002002F081FA002002F07EFA64
:10859000002002F07BFA002002F078FA002002F0BE
:1085A00075FA002002F072FA002002F06FFA002043
:1085B00002F06CFA002002F069FA002002F066FA7C
:1085C000002002F063FA002002F060FA002002F0BE
:1085D0005DFAE02002F066FA162002F057FA002059
:1085E00002F054FA1C2002F051FA002002F04EFA78
:1085F000212002F04BFA002002F048FA362002F067
:1086000045FA002002F042FA462002F03FFA00202C
:1086100002F03CFA522002F039FA002002F036FA59
:10862000642002F033FA002002F030FA7A2002F0DF
:108630002DFA002002F02AFA8B2002F027FA0020FF
:1086400002F024FA992002F021FA002002F01EFA2A
:10865000A82002F01BFA002002F018FAB92002F05C
:1086600015FA002002F012FAC42002F00FFA0020DE
:1086700002F00CFACA2002F009FA002002F006FA11
:10868000D22002F003FA002002F000FAD92002F012
:10869000FDF9002002F0FAF9E02002F0F7F90020DD
:1086A00002F0F4F9F32002F0F1F9002002F0EEF903
:1086B000E12002F0F7F9162002F0E8F9002002F0BC
:1086C000E5F91C2002F0E2F9002002F0DFF9222097
:1086D00002F0DCF9002002F0D9F9362002F0D6F9D8
:1086E000002002F0D3F9452002F0D0F9002002F07A
:1086F000CDF9522002F0CAF9002002F0C7F9642037
:1087000002F0C4F9002002F0C1F97A2002F0BEF9AB
:10871000002002F0BBF98B2002F0B8F9002002F033
:10872000B5F9992002F0B2F9002002F0AFF9A820C3
:1087300002F0ACF9002002F0A9F9B92002F0A6F984
:10874000002002F0A3F9C42002F0A0F9002002F0FA
:108750009DF9CA2002F09AF9002002F097F9D22080
:1087600002F094F9002002F091F9D82002F08EF97D
:10877000002002F08BF9E02002F088F9002002F0DE
:1087800085F9F32002F082F9002002F07FF9E2205F
:1087900002F088F9052002F079F9002002F076F95C
:1087A0000B2002F073F9002002F070F91B2002F098
:1087B0006DF9002002F06AF9342002F067F9002018
:1087C00002F064F9442002F061F9002002F05EF941
:1087D0004F2002F05BF9002002F058F9612002F00E
:1087E00055F9002002F052F9792002F04FF90020EB
:1087F00002F04CF9882002F049F9002002F046F915
:10880000972002F043F9002002F040F9A62002F080
:108810003DF9002002F03AF9B72002F037F90020C4
:1088200002F034F9C22002F031F9002002F02EF9F2
:10883000C72002F02BF9002002F028F9D12002F025
:1088400025F9002002F022F9D62002F01FF90020BD
:1088500002F01CF9DD2002F019F9002002F016F9EF
:10886000F32002F013F9002002F010F9E32002F0E7
:1088700019F9052002F00AF9002002F007F90A2090
:1088800002F004F9002002F001F91C2002F0FEF8C9
:10889000002002F0FBF8332002F0F8F8002002F08C
:1088A000F5F8442002F0F2F8002002F0EFF8502032
:1088B00002F0ECF8002002F0E9F8622002F0E6F89D
:1088C000002002F0E3F8782002F0E0F8002002F047
:1088D000DDF8882002F0DAF8002002F0D7F89720BF
:1088E00002F0D4F8002002F0D1F8A62002F0CEF871
:1088F000002002F0CBF8B72002F0C8F8002002F008
:10890000C5F8C22002F0C2F8002002F0BFF8C7206C
:1089100002F0BCF8002002F0B9F8D12002F0B6F85D
:10892000002002F0B3F8D52002F0B0F8002002F0E9
:10893000ADF8DD2002F0AAF8002002F0A7F8F3203D
:1089400002F0A4F8002002F0A1F8E42002F0AAF856
:10895000012002F09BF8002002F098F8012002F0BC
:1089600095F8002002F092F8022002F08FF8002023
:1089700002F08CF82A2002F089F8002002F086F834
:108980003C2002F083F8002002F080F84B2002F037
:108990007DF8002002F07AF85D2002F077F80020E0
:1089A00002F074F8742002F071F8002002F06EF802
:1089B000842002F06BF8002002F068F8932002F0A7
:1089C00065F8002002F062F8A22002F05FF80020B3
:1089D00002F05CF8B32002F059F8002002F056F8DB
:1089E000BE2002F053F8002002F050F8C42002F03C
:1089F0004DF8002002F04AF8CD2002F047F80020A0
:108A000002F044F8D32002F041F8002002F03EF8D2
:108A1000DD2002F03BF8002002F038F8F32002F0ED
:108A200035F8002002F032F8E52002F03BF8002093
:108A300002F02CF8002002F029F8002002F026F8BD
:108A4000002002F023F8022002F020F8002002F0BB
:108A50001DF8292002F01AF8002002F017F83C2037
:108A600002F014F8002002F011F84B2002F00EF88A
:108A7000002002F00BF85D2002F008F8002002F060
:108A800005F8742002F002F8002001F0FFFF8420B6
:108A900001F0FCFF002001F0F9FF932001F0F6FF48
:108AA000002001F0F3FFA22001F0F0FF002001F010
:108AB000EDFFB32001F0EAFF002001F0E7FFBE2048
:108AC00001F0E4FF002001F0E1FFC42001F0DEFF2F
:108AD000002001F0DBFFCD2001F0D8FF002001F0E5
:108AE000D5FFD32001F0D2FF002001F0CFFFDC2022
:108AF00001F0CCFF002001F0C9FFF32001F0C6FF18
:108B0000002001F0C3FFE62001F0CCFF112001F0AE
:108B1000BDFF002001F0BAFF342001F0B7FF0020B4
:108B200001F0B4FF562001F0B1FF002001F0AEFFCC
:108B3000762001F0ABFF002001F0A8FF772001F0C4
:108B4000A5FF002001F0A2FF662001F09FFF00209A
:108B500001F09CFF882001F099FF002001F096FFB2
:108B6000992001F093FF002001F090FFBB2001F05D
:108B70008DFF002001F08AFF992001F087FF00207F
:108B800001F084FF662001F081FF002001F07EFFEC
:108B9000552001F07BFF002001F078FF552001F007
:108BA00075FF002001F072FF452001F06FFF0020EB
:108BB00001F06CFF432001F069FF002001F066FF27
:108BC000442001F063FF002001F060FFE72001F086
:108BD00069FF322001F05AFF002001F057FF5520B5
:108BE00001F054FF002001F051FF762001F04EFF0C
:108BF000002001F04BFF662001F048FF002001F04B
:108C000045FF672001F042FF002001F03FFF672091
:108C100001F03CFF002001F039FF872001F036FF12
:108C2000002001F033FF992001F030FF002001F017
:108C30002DFFBB2001F02AFF002001F027FF992023
:108C400001F024FF002001F021FF772001F01EFF3A
:108C5000002001F01BFF442001F018FF002001F06C
:108C600015FF562001F012FF002001F00FFF232016
:108C700001F00CFF002001F009FF332001F006FF96
:108C8000002001F003FF452001F000FF002001F06B
:108C9000FDFEE82001F006FF002001F0F7FE0020B5
:108CA00001F0F4FE992001F0F1FE002001F0EEFE4B
:108CB000872001F0EBFE002001F0E8FE882001F0A3
:108CC000E5FE002001F0E2FE772001F0DFFE00204B
:108CD00001F0DCFE662001F0D9FE002001F0D6FE96
:108CE000882001F0D3FE002001F0D0FEAA2001F080
:108CF000CDFE002001F0CAFEBB2001F0C7FE00201F
:108D000001F0C4FE992001F0C1FE002001F0BEFE7A
:108D1000662001F0BBFE002001F0B8FE552001F0F6
:108D2000B5FE002001F0B2FE552001F0AFFE00209C
:108D300001F0ACFE442001F0A9FE002001F0A6FEE7
:108D4000442001F0A3FE002001F0A0FE552001F018
:108D50009DFE002001F09AFEE92001F0A3FEAA206A
:108D600001F094FE002001F091FE002001F08EFE43
:108D7000002001F08BFE002001F094FEAA2001F0FB
:108D800085FECF2001F08EFE002001F07FFE002046
:108D900001F07CFE002001F079FE002001F076FE5B
:108DA000002001F073FE002001F070FE002001F0B1
:108DB0006DFE002001F06AFE002001F067FE002039
:108DC00001F064FE002001F061FE002001F05EFE73
:108DD000002001F05BFE002001F058FE002001F0B1
:108DE00055FE002001F052FE002001F04FFEF02061
:108DF00001F058FE002001F049FE502001F046FE2F
:108E0000002001F043FE002001F040FE002001F0B0
:108E10003DFEF32001F046FE002001F037FEF92070
:108E200001F040FE062001F031FE102001F02EFE80
:108E3000292001F02BFE002001F028FE3A2001F04D
:108E400031FE552001F022FE112001F02BFE64209E
:108E5000FAF73AFB292001F025FE352001F022FE29
:108E6000002001F013FE512001F01CFEFF2001F054
:108E70000DFE532001F016FE2C2001F007FE5520B8
:108E800001F010FE822001F001FE2C2001F00AFE0C
:108E900010BD10B555214FF4704001F019FEAA2104
:108EA0004FF2010001F014FE52214FF2020001F0D6
:108EB0000FFE08214FF2030001F00AFE01214FF2DC
:108EC000040001F005FE0D214FF4304001F000FEDA
:108ED0000D214BF2010001F0FBFD0D214BF20200D0
:108EE00001F0F6FD34214FF4364001F0F1FD34215C
:108EF0004BF2016001F0ECFD34214BF2026001F015
:108F0000E7FD0D214FF4314001F0E2FD0D214BF260
:108F1000011001F0DDFD0D214BF2021001F0D8FD32
:108F200034214FF4374001F0D3FD34214BF201706E
:108F300001F0CEFD34214BF2027001F0C9FD002199
:108F40004FF4324001F0C4FD00214BF2012001F04A
:108F5000BFFD00214BF2022001F0BAFD24214FF4A5
:108F6000384001F0B5FD24214BF6010001F0B0FDC1
:108F700024214BF6020001F0ABFD01214FF43F40EC
:108F800001F0A6FD0F214FF4334001F0A1FD0F21A8
:108F90004BF2013001F09CFD0F214BF2023001F049
:108FA00097FD34214FF4394001F092FD34214BF606
:108FB000011001F08DFD34214BF6021001F088FD07
:108FC00008214FF4354001F083FD08214BF2015098
:108FD00001F07EFD08214BF2025001F079FD0321E2
:108FE0004FF4424001F074FD24214FF43A4001F067
:108FF0006FFD24214BF6012001F06AFD24214BF680
:10900000022001F065FD00214FF43C4001F060FDBD
:1090100078214BF6014001F05BFD00214BF6024048
:1090200001F056FD00214FF43D4001F051FD782143
:109030004BF6015001F04CFD00214BF6025001F0BF
:1090400047FD00214FF43E4001F042FD64214BF604
:10905000016001F03DFD00214FF4514001F038FD69
:1090600033214DF2011001F033FD00214DF20210C9
:1090700001F02EFD34214DF2031001F029FD0021F5
:109080004DF2041001F024FD3A214DF2051001F0DB
:109090001FFD00214DF2061001F01AFD4A214DF28C
:1090A000071001F015FD00214DF2081001F010FD30
:1090B0005C214DF2091001F00BFD00214DF20A1068
:1090C00001F006FD81214DF20B1001F001FD0021A0
:1090D0004DF20C1001F0FCFCA6214DF20D1001F038
:1090E000F7FC00214DF20E1001F0F2FCE5214DF2EB
:1090F0000F1001F0EDFC01214DF2101001F0E8FC21
:1091000013214DF2111001F0E3FC01214DF2121078
:1091100001F0DEFC54214DF2131001F0D9FC0121C5
:109120004DF2141001F0D4FC82214DF2151001F023
:10913000CFFC01214DF2161001F0CAFCCA214DF2FC
:10914000171001F0C5FC02214DF2181001F0C0FC0F
:1091500000214DF2191001F0BBFC02214DF21A1052
:1091600001F0B6FC01214DF21B1001F0B1FC02210F
:109170004DF21C1001F0ACFC34214DF21D1001F039
:10918000A7FC02214DF21E1001F0A2FC67214DF256
:109190001F1001F09DFC02214DF2201001F098FCFF
:1091A00084214DF2211001F093FC02214DF2221096
:1091B00001F08EFCA4214DF2231001F089FC022164
:1091C0004DF2241001F084FCB7214DF2251001F07E
:1091D0007FFC02214DF2261001F07AFCCF214DF2E6
:1091E000271001F075FC02214DF2281001F070FCEF
:1091F000DE214DF2291001F06BFC02214DF22A1004
:1092000001F066FCF2214DF22B1001F061FC02210D
:109210004DF22C1001F05CFCFE214DF22D1001F0FE
:1092200057FC03214DF22E1001F052FC10214DF29B
:109230002F1001F04DFC03214DF2301001F048FCDD
:1092400033214DF2311001F043FC03214DF2321075
:1092500001F03EFC6D214DF2331001F039FC00218C
:109260004FF4524001F034FC33214DF2012001F063
:109270002FFC00214DF2022001F02AFC34214DF296
:10928000032001F025FC00214DF2042001F020FC18
:109290003A214DF2052001F01BFC00214DF2062081
:1092A00001F016FC4A214DF2072001F011FC0021CB
:1092B0004DF2082001F00CFC5C214DF2092001F078
:1092C00007FC00214DF20A2001F002FC81214DF241
:1092D0000B2001F0FDFB00214DF20C2001F0F8FB0A
:1092E000A6214DF20D2001F0F3FB00214DF20E20DE
:1092F00001F0EEFBE5214DF20F2001F0E9FB012129
:109300004DF2102001F0E4FB13214DF2112001F089
:10931000DFFB01214DF2122001F0DAFB54214DF266
:10932000132001F0D5FB01214DF2142001F0D0FBF8
:1093300082214DF2152001F0CBFB01214DF21620C8
:1093400001F0C6FBCA214DF2172001F0C1FB02213A
:109350004DF2182001F0BCFB00214DF2192001F064
:10936000B7FB02214DF21A2001F0B2FB01214DF2B0
:109370001B2001F0ADFB02214DF21C2001F0A8FBE7
:1093800034214DF21D2001F0A3FB02214DF21E20DD
:1093900001F09EFB67214DF21F2001F099FB022195
:1093A0004DF2202001F094FB84214DF2212001F0A8
:1093B0008FFB02214DF2222001F08AFBA4214DF205
:1093C000232001F085FB02214DF2242001F080FBD7
:1093D000B7214DF2252001F07BFB02214DF2262022
:1093E00001F076FBCF214DF2272001F071FB022125
:1093F0004DF2282001F06CFBDE214DF2292001F016
:1094000067FB02214DF22A2001F062FBF2214DF2AE
:109410002B2001F05DFB02214DF22C2001F058FBC6
:10942000FE214DF22D2001F053FB03214DF22E20A1
:1094300001F04EFB10214DF22F2001F049FB0321DA
:109440004DF2302001F044FB33214DF2312001F088
:109450003FFB03214DF2322001F03AFB6D214DF22A
:10946000332001F035FB00214FF4534001F030FB75
:1094700033214DF2013001F02BFB00214DF202307F
:1094800001F026FB34214DF2033001F021FB0021D5
:109490004DF2043001F01CFB3A214DF2053001F091
:1094A00017FB00214DF2063001F012FB4A214DF26C
:1094B000073001F00DFB00214DF2083001F008FBF0
:1094C0005C214DF2093001F003FB00214DF20A301E
:1094D00001F0FEFA81214DF20B3001F0F9FA002182
:1094E0004DF20C3001F0F4FAA6214DF20D3001F0EE
:1094F000EFFA00214DF20E3001F0EAFAE5214DF2CB
:109500000F3001F0E5FA01214DF2103001F0E0FAE0
:1095100013214DF2113001F0DBFA01214DF212302E
:1095200001F0D6FA54214DF2133001F0D1FA0121A5
:109530004DF2143001F0CCFA82214DF2153001F0D9
:10954000C7FA01214DF2163001F0C2FACA214DF2DC
:10955000173001F0BDFA02214DF2183001F0B8FACF
:1095600000214DF2193001F0B3FA02214DF21A3008
:1095700001F0AEFA01214DF21B3001F0A9FA0221EF
:109580004DF21C3001F0A4FA34214DF21D3001F0EF
:109590009FFA02214DF21E3001F09AFA67214DF236
:1095A0001F3001F095FA02214DF2203001F090FABF
:1095B00084214DF2213001F08BFA02214DF222304C
:1095C00001F086FAA4214DF2233001F081FA022144
:1095D0004DF2243001F07CFAB7214DF2253001F034
:1095E00077FA02214DF2263001F072FACF214DF2C6
:1095F000273001F06DFA02214DF2283001F068FAAF
:10960000DE214DF2293001F063FA02214DF22A30B9
:1096100001F05EFAF2214DF22B3001F059FA0221ED
:109620004DF22C3001F054FAFE214DF22D3001F0B4
:109630004FFA03214DF22E3001F04AFA10214DF27B
:109640002F3001F045FA03214DF2303001F040FA9D
:1096500033214DF2313001F03BFA03214DF232302B
:1096600001F036FA6D214DF2333001F031FA00216C
:109670004FF4544001F02CFA33214DF2014001F037
:1096800027FA00214DF2024001F022FA34214DF276
:10969000034001F01DFA00214DF2044001F018FAD8
:1096A0003A214DF2054001F013FA00214DF2064037
:1096B00001F00EFA4A214DF2074001F009FA0021AB
:1096C0004DF2084001F004FA5C214DF2094001F02E
:1096D000FFF900214DF20A4001F0FAF981214DF223
:1096E0000B4001F0F5F900214DF20C4001F0F0F9CA
:1096F000A6214DF20D4001F0EBF900214DF20E4094
:1097000001F0E6F9E5214DF20F4001F0E1F9012108
:109710004DF2104001F0DCF913214DF2114001F03F
:10972000D7F901214DF2124001F0D2F954214DF246
:10973000134001F0CDF901214DF2144001F0C8F9B8
:1097400082214DF2154001F0C3F901214DF216407E
:1097500001F0BEF9CA214DF2174001F0B9F902211A
:109760004DF2184001F0B4F900214DF2194001F01A
:10977000AFF902214DF21A4001F0AAF901214DF290
:109780001B4001F0A5F902214DF21C4001F0A0F9A7
:1097900034214DF21D4001F09BF902214DF21E4093
:1097A00001F096F967214DF21F4001F091F9022175
:1097B0004DF2204001F08CF984214DF2214001F05E
:1097C00087F902214DF2224001F082F9A4214DF2E5
:1097D000234001F07DF902214DF2244001F078F997
:1097E000B7214DF2254001F073F902214DF22640D8
:1097F00001F06EF9CF214DF2274001F069F9022105
:109800004DF2284001F064F9DE214DF2294001F0CB
:109810005FF902214DF22A4001F05AF9F2214DF28E
:109820002B4001F055F902214DF22C4001F050F986
:10983000FE214DF22D4001F04BF903214DF22E4057
:1098400001F046F910214DF22F4001F041F90321BA
:109850004DF2304001F03CF933214DF2314001F03E
:1098600037F903214DF2324001F032F96D214DF20A
:10987000334001F02DF900214FF4554001F028F953
:1098800033214DF2015001F023F900214DF2025035
:1098900001F01EF934214DF2035001F019F90021B5
:1098A0004DF2045001F014F93A214DF2055001F047
:1098B0000FF900214DF2065001F00AF94A214DF24C
:1098C000075001F005F900214DF2085001F000F9B0
:1098D0005C214DF2095001F0FBF800214DF20A50D5
:1098E00001F0F6F881214DF20B5001F0F1F8002162
:1098F0004DF20C5001F0ECF8A6214DF20D5001F0A4
:10990000E7F800214DF20E5001F0E2F8E5214DF2AA
:109910000F5001F0DDF801214DF2105001F0D8F8A0
:1099200013214DF2115001F0D3F801214DF21250E4
:1099300001F0CEF854214DF2135001F0C9F8012185
:109940004DF2145001F0C4F882214DF2155001F08F
:10995000BFF801214DF2165001F0BAF8CA214DF2BC
:10996000175001F0B5F802214DF2185001F0B0F88F
:1099700000214DF2195001F0ABF802214DF21A50BE
:1099800001F0A6F801214DF21B5001F0A1F80221CF
:109990004DF21C5001F09CF834214DF21D5001F0A5
:1099A00097F802214DF21E5001F092F867214DF216
:1099B0001F5001F08DF802214DF2205001F088F87F
:1099C00084214DF2215001F083F802214DF2225002
:1099D00001F07EF8A4214DF2235001F079F8022124
:1099E0004DF2245001F074F8B7214DF2255001F0EA
:1099F0006FF802214DF2265001F06AF8CF214DF2A6
:109A0000275001F065F802214DF2285001F060F86E
:109A1000DE214DF2295001F05BF802214DF22A506F
:109A200001F056F8F2214DF22B5001F051F80221CD
:109A30004DF22C5001F04CF8FE214DF22D5001F06A
:109A400047F803214DF22E5001F042F810214DF25B
:109A50002F5001F03DF803214DF2305001F038F85D
:109A600033214DF2315001F033F803214DF23250E1
:109A700001F02EF86D214DF2335001F029F800214C
:109A80004FF4564001F024F833214DF2016001F00B
:109A90001FF800214DF2026001F01AF834214DF256
:109AA000036001F015F800214DF2046001F010F898
:109AB0003A214DF2056001F00BF800214DF20660ED
:109AC00001F006F84A214DF2076001F001F800218B
:109AD0004DF2086000F0FCFF5C214DF2096000F0DF
:109AE000F7FF00214DF20A6000F0F2FF81214DF2F4
:109AF0000B6000F0EDFF00214DF20C6000F0E8FF7C
:109B0000A6214DF20D6000F0E3FF00214DF20E6042
:109B100000F0DEFFE5214DF20F6000F0D9FF0121DA
:109B20004DF2106000F0D4FF13214DF2116000F0EF
:109B3000CFFF01214DF2126000F0CAFF54214DF217
:109B4000136000F0C5FF01214DF2146000F0C0FF6A
:109B500082214DF2156000F0BBFF01214DF216602D
:109B600000F0B6FFCA214DF2176000F0B1FF0221EC
:109B70004DF2186000F0ACFF00214DF2196000F0CA
:109B8000A7FF02214DF21A6000F0A2FF01214DF261
:109B90001B6000F09DFF02214DF21C6000F098FF59
:109BA00034214DF21D6000F093FF02214DF21E6042
:109BB00000F08EFF67214DF21F6000F089FF022147
:109BC0004DF2206000F084FF84214DF2216000F00E
:109BD0007FFF02214DF2226000F07AFFA4214DF2B6
:109BE000236000F075FF02214DF2246000F070FF49
:109BF000B7214DF2256000F06BFF02214DF2266087
:109C000000F066FFCF214DF2276000F061FF0221D6
:109C10004DF2286000F05CFFDE214DF2296000F07B
:109C200057FF02214DF22A6000F052FFF2214DF25F
:109C30002B6000F04DFF02214DF22C6000F048FF38
:109C4000FE214DF22D6000F043FF03214DF22E6006
:109C500000F03EFF10214DF22F6000F039FF03218C
:109C60004DF2306000F034FF33214DF2316000F0EE
:109C70002FFF03214DF2326000F02AFF6D214DF2DB
:109C8000336000F025FF55214FF4704000F020FFB5
:109C9000AA214FF2010000F01BFF52214FF20200F7
:109CA00000F016FF08214FF2030000F011FF002121
:109CB0004FF2040000F00CFFCC214FF4314000F0D3
:109CC00007FF00214BF2011000F002FF05214FF4C5
:109CD000364000F0FDFE70214FF4374000F0F8FEF2
:109CE00070214BF2017000F0F3FE01214FF4384077
:109CF00000F0EEFE03214BF6010000F0E9FE032127
:109D00004BF6020000F0E4FE03214BF6030000F0E6
:109D1000DFFE02214FF43C4000F0DAFE00214BF65A
:109D2000014000F0D5FE00214BF6024000F0D0FECD
:109D3000D0214FF4494000F0CBFE02214CF6011037
:109D400000F0C6FE50214CF6021000F0C1FE50217A
:109D50004CF6031000F0BCFE50214CF6041000F04D
:109D6000B7FE00214FF4545000F0B2FE55214FF4DD
:109D7000685000F0ADFE4FF4885000F093FE78205C
:109D8000F9F7AEFB4FF4245000F08CFE10BD10B577
:109D9000E22000F087FE1D2000F078FE022000F097
:109DA00075FE042000F072FE6420F9F799FBE020B4
:109DB00000F078FE012000F069FE0A20F9F784FB2C
:109DC000E02000F06FFE032000F060FE0C20F9F7A9
:109DD0007BFB012000F066FE0A20F9F775FBE62008
:109DE00000F060FE2F2000F051FEFF2000F04EFE3C
:109DF000FF2000F04BFEB02000F054FE202000F0C9
:109E000045FE002000F042FE032000F03FFE40F23D
:109E10001F3000F03BFE012000F038FE40F2DF1062
:109E200000F034FE002000F031FEB42000F03AFED5
:109E3000042000F02BFE40F21F4000F027FE00201F
:109E400000F024FE2E2000F021FE002000F01EFE77
:109E5000002000F01BFE002000F018FE002000F0A3
:109E600015FEB62000F01EFE022000F00FFE4FF49B
:109E7000037000F00BFE002000F008FE172000F039
:109E800005FE152000F002FE002000F0FFFD00207E
:109E900000F0FCFDF02000F005FE032000F0F6FDD0
:109EA000292000F0FFFDD02000F0FCFD002000F094
:109EB000EDFDBE2000F0F6FD052000F0E7FDFE20E0
:109EC00000F0E4FD012000F0E1FD002000F0DEFDE7
:109ED000002000F0DBFD002000F0D8FDB82000F0ED
:109EE000E1FD032000F0D2FD012000F0CFFDBA20FB
:109EF00000F0D8FD012000F0C9FD10BD10B5112003
:109F000000F0D0FD7820F9F7DFFA362000F0CAFD26
:109F1000002000F0BBFD3A2000F0C4FD052000F059
:109F2000B5FDB22000F0BEFD0C2000F0AFFD0C200E
:109F300000F0ACFD002000F0A9FD332000F0A6FDEC
:109F4000332000F0A3FDB72000F0ACFD352000F079
:109F50009DFDBB2000F0A6FD322000F097FDC02043
:109F600000F0A0FD0C2000F091FDC22000F09AFD51
:109F7000012000F08BFDC32000F094FD102000F0C4
:109F800085FDC42000F08EFD202000F07FFDC6205E
:109F900000F088FD0F2000F079FDD02000F082FD58
:109FA000A42000F073FDA12000F070FDE02000F07F
:109FB00079FDD02000F06AFD002000F067FD02204E
:109FC00000F064FD072000F061FD0A2000F05EFD56
:109FD000282000F05BFD322000F058FD442000F006
:109FE00055FD422000F052FD062000F04FFD0E20EE
:109FF00000F04CFD122000F049FD142000F046FD59
:10A00000172000F043FDE12000F04CFDD02000F0CF
:10A010003DFD002000F03AFD022000F037FD072052
:10A0200000F034FD0A2000F031FD282000F02EFD64
:10A03000312000F02BFD542000F028FD472000F0D7
:10A0400025FD0E2000F022FD1C2000F01FFD172032
:10A0500000F01CFD1B2000F019FD1E2000F016FD75
:10A060002A2000F01FFD002000F010FD002000F06D
:10A070000DFD002000F00AFDEF2000F007FD2B2071
:10A0800000F010FD002000F001FD002000F0FEFCBB
:10A09000012000F0FBFC3F2000F0F8FC292000F03C
:10A0A00001FD10BD2DE9F04F05460E4617469846B6
:10A0B000DDF824A04FF0000B781B401C1FFA80FB3A
:10A0C000344613E02146284600F04AFB00F0F6FC37
:10A0D0004FF0000906E00749A1F800A009F10100CE
:10A0E0001FFA80F9D945F6DB601C84B24445E9DDEE
:10A0F000BDE8F08F8000006C00B595B000BF00BFD8
:10A1000000200190FD48006840F04000FB490860D5
:10A110000846006800F04000019000BF00BF00BF8B
:10A1200000BF00BF002001900846006840F0080012
:10A1300008600846006800F00800019000BF00BFFA
:10A1400000BF00BF00BF002001900846006840F03B
:10A15000080008600846006800F00800019000BF91
:10A1600000BF00BF00BF00BF00200190084600688C
:10A1700040F0400008600846006800F04000019090
:10A1800000BF00BF00BF00BF00BF00200190084615
:10A19000006840F0020008600846006800F0020015
:10A1A000019000BF00BF00BF8814109002201190E2
:10A1B00001201290022013900C20149010A9D04876
:10A1C000F7F7E6FA2020109010A9CE48F7F7E0FA4A
:10A1D0001020109010A9CB48F7F7DAFA4FF480500E
:10A1E000109010A9C848F7F7D3FA4FF40040109028
:10A1F0000120119010A9C548F7F7CAFA4FF0204086
:10A20000C3490860C3484860062088600021C048F0
:10A21000C1601021416100218161C16141624FF43F
:10A22000805181620021C1624FF4804101630021AD
:10A23000416381630F20099000200A903C200B901D
:10A2400000200F9005900920029000200390082024
:10A2500004900020089002AA09A9AD48F7F7F8FF7A
:10A260003220F9F731F9D32000F01CFC00F056F948
:10A27000A949888000F052F9A749888000F04EF97A
:10A28000A5498880084680884FF6FF7101EA0020C2
:10A29000A149888000F042F99F49898808439E4976
:10A2A00088800846808849F2413188427DD0042068
:10A2B00000F0F8FB00F032F99749888000F02EF9A1
:10A2C0009549888000F02AF993498880084680885B
:10A2D0004FF6FF7101EA00208F49888000F01EF9D7
:10A2E0008D49898808438C4988800846808848F2CF
:10A2F0005251884203D147F2897087498880864845
:10A30000808847F289718842D0D0D42000F0CAFBFF
:10A3100000F004F98049888000F000F97E498880C7
:10A3200000F0FCF87C498880084680884FF6FF7171
:10A3300001EA00207849888000F0F0F876498988A1
:10A340000843754988800846808845F21031884264
:10A3500062D055214FF4704000F0BAFBAA214FF2B1
:10A36000010000F0B5FB52214FF2020000F0B0FBFB
:10A3700008214FF2030000F0ABFB01214FF2040073
:10A3800000F0A6FB4FF4454000F08CFB00F0C6F84F
:10A3900061498880084680884FF6FF7101EA0020F5
:10A3A0005D4988804CF2015000E035E000F07AFB16
:10A3B00000F0B4F858498988084357498880052037
:10A3C000F9F782F85448808845F21051884223D02A
:10A3D000A12000F067FB00F0A1F84F49888000F051
:10A3E0009DF84D498880084680884FF6FF7101EA44
:10A3F00000204949888000F091F84749898808433E
:10A40000454988800846808845F26171884203D1B9
:10A4100041F66310404988803F48808847F289713F
:10A42000884202D1FFF76AFD25E03B48808849F267
:10A430004131884202D1FDF79DFC1CE036488088FE
:10A4400045F21031884202D1FDF7AAFD13E03248EF
:10A45000808845F21051884202D1FEF71AFD0AE0C9
:10A460002D48808841F66311884204D1FFF78FFCA4
:10A47000642000F0DBFA2848808849F241318842A4
:10A480000BD02548808841F66311884205D02248C8
:10A49000808847F28971884209D103200290049094
:10A4A0001B490B6B8A68486802A9F6F77DFB1A48BE
:10A4B000808845F21031884205D01748808845F2DF
:10A4C0001051884209D102200290049010490B6B70
:10A4D0008A68486802A9F6F767FB0020FDF7A2FB2F
:10A4E00000BF0122D1030948F7F75EFA00BF4FF61B
:10A4F000FF70FDF77DFB15B000BD00003038024055
:10A5000000180240000C0240001402400004024007
:10A5100040040020040100A09004002008B5034876
:10A5200000880090BDF8000008BD00008000006CAD
:10A53000F0B505460024002788488079012805D118
:10A540008648808841F66311884208D18348807923
:10A55000F0B98248808841F66311884218D1082DED
:10A5600015D2DFE805F00406080A0C0E10120625C5
:10A570000DE007250BE0042509E0052507E001258E
:10A5800005E0002503E0032501E0022500BF00BF30
:10A59000082D1CD2DFE805F00406090C0F1215186F
:10A5A00000BF14E044F0800411E044F040040EE0E9
:10A5B00044F0C0040BE044F0200408E044F06004E0
:10A5C00005E044F0A00402E044F0E00400BF00BF56
:10A5D00036276248808845F21051884200D13F02F8
:10A5E0005E48808849F24131884205D05B488088C6
:10A5F00047F28971884201D144F008042146384667
:10A6000000F066FA5548808841F6631188421DD0F3
:10A6100004F0200068B151480088504949888842B8
:10A6200014DA4E48068840884C490880084646801F
:10A630000CE04A48008849494988884206DD474875
:10A6400006884088454908800846468043488088F7
:10A6500045F21051884252D14049488900F022FA0F
:10A66000002000F013FA3D494989491C88B200F0E6
:10A6700019FA002000F00AFA38494989891C88B281
:10A6800000F010FA35490988491EC1F30F2000F087
:10A69000FDF932494989C91C88B200F003FA2F49F3
:10A6A0000978491EC8B200F0F1F92C49888900F0F8
:10A6B000F9F9002000F0EAF928498989491C88B293
:10A6C00000F0F0F9002000F0E1F924498989891CA3
:10A6D00088B200F0E7F921494988491EC1F30F20EB
:10A6E00000F0D4F91D498989C91C88B200F0DAF953
:10A6F0001A498978491EC8B200F0C8F92DE01749F7
:10A70000488900F0CFF9002000F0C0F9002000F0E7
:10A71000BDF912490988491EC1F30F2000F0B6F9AE
:10A720000E490978491EC8B200F0B0F90B49888972
:10A7300000F0B8F9002000F0A9F9002000F0A6F917
:10A7400006494988491EC1F30F2000F09FF90349CB
:10A750008978491EC8B200F099F9F0BD9004002034
:10A7600010B502460C464548808841F66311884280
:10A7700047D142488079A8B940480088401E801AD5
:10A7800082B23E49488900F08DF9002000F07EF940
:10A79000002000F07BF9101200F078F9D0B200F040
:10A7A00075F916E03549488900F07CF9101200F07F
:10A7B0006DF9D0B200F06AF930490988491EC1F339
:10A7C0000F2000F063F92D490978491EC8B200F046
:10A7D0005DF92A49888900F065F9201200F056F9E0
:10A7E000E0B200F053F925494988491EC1F30F2012
:10A7F00000F04CF921498978491EC8B200F046F9A9
:10A800003AE01E48808845F21051884220D11B4909
:10A81000488900F047F9101200F038F917494989C2
:10A82000491C88B200F03EF9D0B200F02FF913496C
:10A83000888900F037F9201200F028F90F4989893A
:10A84000491C88B200F02EF9E0B200F01FF913E0C5
:10A850000A49488900F026F9101200F017F9D0B221
:10A8600000F014F90549888900F01CF9201200F065
:10A870000DF9E0B200F00AF910BD000090040020CC
:10A880002DE9FC4F80460E4615461C46B346002077
:10A89000019000902046E31704EB5373DB10214630
:10A8A0004FEAE47C04EB5C7C4FEAEC0CA4EBCC0CB0
:10A8B000BCF1000F02D04FF0010C01E04FF0000C92
:10A8C0006344224604EBD27C4FEA6C0C03FB0CF38E
:10A8D000DBB20193A5F12000C5B20C2C06D0102CE0
:10A8E0000BD0182C0ED0202C18D112E005EB45000F
:10A8F0002D4901EB8000009012E02C4800EB051080
:10A9000000900DE005EBC500294901EB80000090A7
:10A9100006E0284800EB8510009001E0BDE8FC8FC0
:10A9200000BF00273AE0009810F807904FF0000AA7
:10A930002EE009F0800028B1314640460C9AFDF720
:10A9400009FA07E00B9828B91B48314602684046CF
:10A95000FDF700FA4FEA49604FEA1069701C86B2B1
:10A9600016484088B04200DCD8E7A6EB0B00A042B6
:10A970000AD15E4608F101001FFA80F80F480088EE
:10A98000404500DCCAE706E00AF1010000F0FF0ADA
:10A99000BAF1080FCDDB00BF781CC7B2019887421F
:10A9A000C1DB00BFBAE70000CCA9010840AE010836
:10A9B00030B401088CC101082C0000209004002054
:10A9C0002DE9FC4F04460D4690469946DDE90C7A88
:10A9D0000B9E04F0FF0B08EB04001FFA80F809EB54
:10A9E00005001FFA80F917E0444502DB5C46A81910
:10A9F00085B24D4500DB15E00020CDE9000A3A782C
:10AA0000334629462046FFF73BFF304606EBD07120
:10AA100004EB61018CB27F1C38787E2802DC387828
:10AA20002028E1DA00BFBDE8FC8F000070B52DEDF5
:10AA3000048B0446BE2000F035F8052000F026F80F
:10AA40002046F5F734FD41EC190B9FED0E0B53EC4E
:10AA5000102BF5F7BAFC41EC180BF5F735FD85B274
:10AA6000284600F013F8012000F010F8FF2000F055
:10AA70000DF8002000F00AF8002000F007F8BDEC07
:10AA8000048B70BD666666666666044001B5BDF8F7
:10AA900000000090BDF800000149088008BD0000DA
:10AAA0008000006C01B5BDF800000090BDF800000A
:10AAB0000149088008BD00007E00006C0248008942
:10AAC0000249088070470000900400207E00006C5E
:10AAD000034A10804FF0D842A2F88010704700005F
:10AAE0007E00006C00B587B000BF00BF0020019061
:10AAF0002048006840F020001E49086008460068B1
:10AB000000F02000019000BF00BF00BF00BF00BFE9
:10AB1000002001900846006840F0200008600846C8
:10AB2000006800F02000019000BF00BF00BF481582
:10AB300002900120039004900220059002A90E4883
:10AB4000F6F726FE4FF48060029002A90A48F6F755
:10AB50001FFE00BF012251020748F6F725FF00BF84
:10AB600000BF012291020448F6F71EFF00BF07B0A4
:10AB700000BD0000303802400014024000BF09E070
:10AB800000BF4FF480610448F6F704FF00BF642063
:10AB90000EF090FAF4E70000001402401CB50446E1
:10ABA000062084F830002148007884F82A001F48E5
:10ABB00041782B2001551D4881782C2001551B48D8
:10ABC000C1782D200155194801792E2001551748CB
:10ABD00041792F20015540F2DC50208503220021CD
:10ABE00001200EF02BFE124908600220430222468B
:10ABF0001049009010A006F06FFF01900E2084F81D
:10AC0000310004230F4802680F4801680F48F6F727
:10AC100003F904230E4802680E4801680B48F6F752
:10AC2000B5F80A48F6F77BFC1CBD0000644F012014
:10AC300090020020716300086574685F7468726533
:10AC4000616400003C00002034000020F00400207B
:10AC500038000020300000202DE9F84F0024A246E3
:10AC6000A046002000903A48F6F718F910B10020ED
:10AC7000BDE8F88F3648808F1FFA80FB3448D0F843
:10AC800040904FF4C1725946002004F0D7F80746AF
:10AC9000002F32D02E48066B00243D462BE0B5F83D
:10ACA0000A804FF0000A16E040F2F4531A1B09EB39
:10ACB00004016B6803EB0A00F5F734FBF668D6F87D
:10ACC000089040F2F450001BA8EB000840F2F4504A
:10ACD000001B8244002408EB040040F2F451884237
:10ACE000E2D809EB04016A6802EB0A004246F5F774
:10ACF00019FB44442D68002DD1D11548066B002066
:10AD0000009007E0306840F000403060F66800983E
:10AD1000401C00900E48816B00988142F2D80021BF
:10AD20000B488163006800F58050406900F08000A6
:10AD300058B180210648006800F58050416100212B
:10AD40000348006800F580508160384690E70000B5
:10AD5000F00400202DE9F84F8B463748C06A806820
:10AD600000904FF0000900240026A2463248D0F897
:10AD70002C8000BF5D463FE0D8F8000000F00040A6
:10AD800010B16FF007073FE06E894FF0000A23E033
:10AD900040F2F4531A1B6B6803EB0A01009B18196D
:10ADA000F5F7C0FAD8F80C80D8F8000000F00040A1
:10ADB00010B16FF0070727E0D8F80800009040F2C4
:10ADC000F450001B361A40F2F450001B824440F24B
:10ADD000F450001B81440024301940F2F4518842A1
:10ADE000D6D86A6802EB0A01009A10193246F5F7C4
:10ADF00099FA3444B1442D68002DBDD149460E481E
:10AE0000F6F7DFFB002700BF0B48006800F5805015
:10AE1000406900F0200058B120210748006800F583
:10AE20008050416100210448006800F58050416075
:10AE30003846BDE8F88F0000F0040020C021817181
:10AE4000A822C271012202721B224272B821017033
:10AE5000AE2141701D2181700021C1700721017157
:10AE600000214171C0218172A822C27201220273A5
:10AE70001E224273FF218173FF22C27302740022DB
:10AE80004274C0218174A822C274012202754275E5
:10AE9000002181757047000030B587B00025002182
:10AEA00008460BF09FFFFBF797F910B1012007B0A0
:10AEB00030BD2948FFF7C2FF06E0681CC5B2052D6A
:10AEC00002DD00250320F2E7FBF7DEF80028F4D1CD
:10AED00006900590049021482149002204ABCDE959
:10AEE0000021029005AA06A91E4803F06FFC044643
:10AEF0000CB90420DBE71B4803F076FE194890F8F4
:10AF00003100C0F3800018B1164803F019FF02E0C9
:10AF1000144803F071FE134800F0FCF81249114880
:10AF200003F09CFE03204FF480730E4A0F490090FB
:10AF30000FA006F0D1FD039000200749C875887561
:10AF400004208301074A0D4900900DA006F0C4FDBE
:10AF500003900020ABE70000644F0120116F01084F
:10AF600009630008804F012015B1000891B1000865
:10AF70006574685F6C696E6B000000001DBE0008A0
:10AF80006574685F64686370000000002DE9F0413B
:10AF9000044625466868804706F062FC06460D496F
:10AFA000286809684718B81BB0F1004F01D3012089
:10AFB00000E0002030B1296888192246064906F0D1
:10AFC00003FE04E022460449384606F0FDFDBDE8D4
:10AFD000F0810000640200208DAF00081CB52C2019
:10AFE00002F090FA04460120606100220221084626
:10AFF00001F074FFA0610420009004F114032022EA
:10B0000040F6FF71A06901F021FD0220607042F25C
:10B01000823000F056F8608013A0FCF735FD6060C8
:10B0200010202061144860624FF48061A1621348CF
:10B03000E0611021216203204B012246104900905B
:10B0400010A006F049FD01900CE02069CDE9004018
:10B050000023D4E90712A06901F054FC4FF47A7080
:10B060000EF028F8F1E700003235352E3235352E56
:10B070003235352E32353500B84F01209C02002084
:10B08000ADC500086C7769705F73656E645F746846
:10B09000726561640000000000BFFFF79FFF02E0DF
:10B0A00005200EF007F8FBE70146080601F47F4291
:10B0B00040EA022001F47F0240EA122040EA1160D7
:10B0C000704701460806000C40EA11207047000056
:10B0D00008B50020009000BF6846804204D000BF41
:10B0E0000B48F7F7F3FE00BF00BF00BF00BF06F03C
:10B0F00071FA02F091F902F043FC03F007FD0CF045
:10B1000007F907F00FFCF9F747FF06F0CBFD08BD84
:10B11000F8E0010810B5044694F8310000F0010091
:10B1200030B101200649087006A0F7F7CFFE05E010
:10B130000520034908700CA0F7F7C8FE10BD0000F9
:10B1400094020020546865206E6574776F726B20DE
:10B150006361626C6520697320636F6E6E656374F2
:10B160006564200D0A000000546865206E657477E0
:10B170006F726B206361626C65206973206E6F74FF
:10B1800020636F6E6E6563746564200D0A000000B5
:10B1900008B50446002000902646002530E06A46A7
:10B1A00001211848F6F772F9009800F0040098B9E8
:10B1B00000201549C8756D1C022D00DB20E005201C
:10B1C000124908700F48F6F7D3F9304603F014FD22
:10B1D000304603F047FD0FE000250B48C07D58B90D
:10B1E00001200949C8750748F6F799F9304603F078
:10B1F000A7FD304603F06AFD64200DF05BFF00BF41
:10B20000CDE70000F0040020644F012094020020EC
:10B2100070B505462C4620684678206840680028AE
:10B2200051D02068007800F0F00010284BD1207A2F
:10B23000032801D0022E46D0032E02D1F520207122
:10B2400043E0012E02D1FB2020713EE0207A00F085
:10B25000010010B1206802F0ECFD00BF2068406AD8
:10B2600020B100BF1AA0F7F731FE00BF00BF0420D5
:10B2700021684870206844620021206800F03CF892
:10B2800000B300BF20684078042804D000BF17A096
:10B29000F7F71CFE00BF00BF164806F09FFA2168B2
:10B2A00001F10C00002106F00DF9124806F034FA05
:10B2B00000BF2068407820B100BF0CA0F7F706FE61
:10B2C00000BF00BF70BDF520207100BFFAE700008D
:10B2D000616C72656164792077726974696E672048
:10B2E0006F7220636C6F73696E67000073746174B2
:10B2F00065210000B40100202DE9FC5F04468B4667
:10B300000020019000BF24B900BF7BA0F7F7DEFD4D
:10B3100000BF00BF00BF207800F0F000102804D06C
:10B3200000BF79A0F7F7D2FD00BF00BF00BF607873
:10B33000042804D000BF7CA0F7F7C8FD00BF00BF01
:10B3400000BF606820B900BF80A0F7F7BFFD00BF55
:10B3500000BF00BF606A20B900BF81A0F7F7B6FD4B
:10B3600000BF00BF6768606A90F808A00AF0010992
:10B370000AF00208BAF1030F01D1012517E0B9F173
:10B38000000F0AD0387D052805D0387D062802D068
:10B39000387D082801D1012509E0B8F1000F05D05A
:10B3A000B87E00F0100008B1012500E000251DB1B5
:10B3B0000021384606F0E8FD387D012804D100213F
:10B3C000384606F070FD1BE0B9F1000F07D00021F0
:10B3D000384609F07FFE0021384606F064FDB8F1DA
:10B3E000000F03D0002138460AF0DEF945B10022F3
:10B3F0001146384608F0B8FE0021384607F020F91B
:10B4000025B1384606F0CCFD064605E042464946E1
:10B4100038460AF0EDF9064616B9012001900EE013
:10B42000701C50B9606A407A48B90120019035B16A
:10B43000384606F031FD002601E001200190019818
:10B4400078B3606A00680C300090606A0671002072
:10B4500060626070E6B93DB16060A06A20B1002210
:10B4600004212046A36A9847B9F1000F06D0A06ACC
:10B4700020B1002211462046A36A9847B8F1000F78
:10B4800006D0A06A20B1002202212046A36A984774
:10B49000BBF1000F02D0009806F070FA0020BDE862
:10B4A000FC9FFFE70198E8B900BF387D012804D16F
:10B4B00000BF32A0F7F70AFD00BF00BFB8F1000FD0
:10B4C00003D0374938460AF06FF90122354938462A
:10B4D00008F04AFE3449384607F0B2F821463846AB
:10B4E00006F052FD00BF26B900BF30A0F7F7EEFC12
:10B4F00000BF00BF3046D2E7696E76616C69642098
:10B50000636F6E6E000000007468697320697320B9
:10B51000666F7220746370206E6574636F6E6E73F5
:10B52000206F6E6C79000000636F6E6E206D757316
:10B530007420626520696E207374617465204E45C5
:10B5400054434F4E4E5F434C4F534500706362204F
:10B55000616C726561647920636C6F73656400006F
:10B56000636F6E6E2D3E63757272656E745F6D7380
:10B570006720213D204E554C4C000000436C6F73FA
:10B58000696E672061206C697374656E20706362F8
:10B59000206D6179206E6F74206661696C210000F6
:10B5A0005D0F0108D9FD0008215200086572722064
:10B5B000213D204552525F4F4B00000070B50646BA
:10B5C00034462068457800BF55B12068007800F007
:10B5D000F000102804D000BF46A0F7F777FC00BFAA
:10B5E00000BF1DB1022D01D0032D07D1032D08D1BD
:10B5F000206890F8200000F0040010B9FB202071B2
:10B6000075E000BF032D0AD1206890F8200000F0FB
:10B61000040020B900BF3CA0F7F758FC00BF00BFF2
:10B6200000202071206802F004FC20684068002897
:10B630004DD02068007800F0F00010280AD02028B3
:10B6400040D1002021684968C861216848680CF031
:10B6500055F838E000BF2068406A20B100BF32A032
:10B66000F7F734FC00BF00BF0420216848700320B6
:10B6700020722068446200212068FFF73DFE00B37D
:10B6800000BF20684078042804D000BF2DA0F7F741
:10B690001DFC00BF00BF2D4806F0A0F8216801F195
:10B6A0000C00002105F00EFF284806F035F800BF19
:10B6B0002068407820B100BF22A0F7F707FC00BF48
:10B6C00000BF70BD00BF00BF002021684860206837
:10B6D000806A20B1206800221146836A984720685A
:10B6E000806A20B1206800220221836A984700BF47
:10B6F000E7E700006E6574636F6E6E2073746174AB
:10B7000065206572726F7200626C6F636B696E6741
:10B7100020636F6E6E65637420696E2070726F6750
:10B720007265737300000000616C7265616479205A
:10B7300077726974696E67206F7220636C6F7369CA
:10B740006E6700007374617465210000B40100200D
:10B7500070B505462C4620684068002850D0207CF3
:10B7600028B1206840680068A168086004E020688B
:10B7700040684068A1680860002020712068007857
:10B7800000F0F000102818D0202830D1207C28B1FB
:10B7900020684068418AE06801800DE020684068C8
:10B7A000007C00F0040010B9F520207104E020684E
:10B7B0004068818AE068018021E0207C58B92068D7
:10B7C0004068007D20B120684068007D012802D1DA
:10B7D000F52020710AE0207C18B120684068C08AFA
:10B7E00002E020684068008BE168088007E000BF45
:10B7F00000BF05A0F7F76AFB00BF00BF00BF01E074
:10B80000F520207170BD0000696E76616C6964205E
:10B810006E6574636F6E6E5F747970650000000012
:10B8200070B504462546002028712868406810B984
:10B83000284604F0CDF970BD2DE9F04105462C46AF
:10B840000020207120684068C0B12068007800F0B6
:10B85000F000102812D1A66800BFB6F5803F02D3D1
:10B860004FF6FF7000E0304687B2216848683946DD
:10B8700009F086FCF61B002EEFD100BFBDE8F08179
:10B880002DE9F04105462C46206802F023FB0646D0
:10B8900016BB2068406800B32068007800F0F00014
:10B8A000202816D1A068806800B107E0A26811685E
:10B8B000226850680BF05AFF064609E0A768BB896A
:10B8C00007F108023968276878680BF087FF064699
:10B8D00002E06FF00A0600BF01E06FF00A06267171
:10B8E000BDE8F08170B505462C46206802F0F2FAFA
:10B8F0000646002E53D12068007800F0F000102892
:10B900004BD12068407808B1761F48E02068406835
:10B9100000283FD001202168487000BF2068406A9D
:10B9200020B100BF1FA0F7F7D1FA00BF00BF00BFD2
:10B93000606920B900BF22A0F7F7C8FA00BF00BFB6
:10B94000206844620021206800F04AF808B300BF74
:10B9500020684078012804D000BF1EA0F7F7B6FA8F
:10B9600000BF00BF1D4805F039FF216801F10C0040
:10B97000002105F0A7FD194805F0CEFE00BF2068A4
:10B980004078012804D100BF12A0F7F79FFA00BF4A
:10B9900000BF70BD6FF00A0601E06FF0050626716A
:10B9A00000BFF6E7616C7265616479207772697433
:10B9B000696E67206F7220636C6F73696E67000039
:10B9C0006D73672D3E6D73672E772E6C656E20212B
:10B9D0003D2030007374617465210000B4010020C3
:10B9E0002DE9F34F83B004460020019000BF24B935
:10B9F00000BFA0A0F7F76AFA00BF00BF00BF6078E1
:10BA0000012804D000BF9FA0F7F760FA00BF00BF75
:10BA100000BF606A20B900BFA2A0F7F757FA00BFC5
:10BA200000BF00BF606820B900BFA5A0F7F74EFABD
:10BA300000BF00BF00BF606A81694069814204D3D2
:10BA400000BFA5A0F7F742FA00BF00BF00BF606AC1
:10BA50008089002804DC00BFAFA0F7F737FA00BFE9
:10BA600000BF606A077F94F8200000F0020010B960
:10BA700007F0040008B1012000E00020814600BF6B
:10BA8000606A80680168606A006908440290606AC0
:10BA900080684168606A0069A1EB0008B8F5803FE2
:10BAA00004D34FF6FF7647F0020701E01FFA88F64D
:10BAB0006068B0F864B0B3450FDA5E46B9F1000FC4
:10BAC00009D056B9606A806910B96FF0060000E0CD
:10BAD000002005465AE047F0020700BF606A00698F
:10BAE0003044616A89684968884204D900BF94A0DB
:10BAF000F7F7ECF900BF00BF4FF6FF70864202D1A6
:10BB0000B8F5803F07D21FFA88F0B04208D1606ACA
:10BB10008089012804DD0120009047F0020701E040
:10BB2000002000903B463246606802990AF01EFCF5
:10BB3000054615BB606A80698119606A8161606A27
:10BB400000698119606A0161606A0069616A8968D7
:10BB50004968884211D1606A8089401E81B2606A5A
:10BB60008181606A8089002807DD606A806808300A
:10BB7000616A88600021606A0161009810B1002D3F
:10BB80003FF47EAF0DB1681C48BB00BFB9F1000F98
:10BB900012D0606A8169406981420DD2A06A20B1E9
:10BBA000002203212046A36A984794F8200040F021
:10BBB000100084F8200012E06068B0F8640041F6DC
:10BBC0005E71884204DD6068B0F866002C2806DBF0
:10BBD000A06A20B1002203212046A36A9847A5B994
:10BBE000606A81694069814202D0B9F1000F01D0D9
:10BBF00001200190606807F019FD82460AF10400F7
:10BC000010B95546012001901CE0681CC0B960685D
:10BC100007F00CFD82460AF1040018B955460120D0
:10BC200001900CE0B9F1000F09D0606A806910B989
:10BC30006FF0060000E0002005460120019001E0C1
:10BC400001200190019870B1606A006800F10C0A4F
:10BC5000606A0571002060626070049810B15046FF
:10BC600005F08CFE04E04FF0FF3005B0BDE8F08F2A
:10BC70000020FAE7636F6E6E20213D204E554C4C3C
:10BC800000000000636F6E6E2D3E7374617465205A
:10BC90003D3D204E4554434F4E4E5F57524954450B
:10BCA00000000000636F6E6E2D3E63757272656EEC
:10BCB000745F6D736720213D204E554C4C00000091
:10BCC000636F6E6E2D3E7063622E74637020213D33
:10BCD000204E554C4C000000636F6E6E2D3E637518
:10BCE0007272656E745F6D73672D3E6D73672E772C
:10BCF0002E6F6666736574203C20636F6E6E2D3EFA
:10BD000063757272656E745F6D73672D3E6D7367D8
:10BD10002E772E6C656E0000636F6E6E2D3E637520
:10BD20007272656E745F6D73672D3E6D73672E77EB
:10BD30002E766563746F725F636E74203E203000F0
:10BD40006C7769705F6E6574636F6E6E5F646F5F52
:10BD500077726974656D6F72653A20696E76616C91
:10BD60006964206C656E67746821000010B5044634
:10BD700014F10F0F09D014F10E0F04D014F10D0FB0
:10BD800005D1084810BD0848FCE70848FAE700BF9D
:10BD900024B100BF06A0F7F799F800BF00BF00204C
:10BDA000F0E7000070D9010871D9010872D90108C3
:10BDB000756E68616E646C6564206572726F720086
:10BDC00070B505460C4600BF24B900BF0DA0F7F7BB
:10BDD0007DF800BF00BF0E48854203D1F3202070DC
:10BDE000012070BD0B48854203D1F2202070012054
:10BDF000F7E70948854203D1F12020700120F0E7E0
:10BE00000020EEE765727220213D204E554C4C001B
:10BE100070D9010871D9010872D9010888B080462B
:10BE2000444600250026002784E1C3480078012805
:10BE300004D0022813D0052872D171E1002060607F
:10BE4000A060E0606060A060E0600220BA49087015
:10BE5000BAA0F7F73BF82046F8F72AFE65E120463E
:10BE6000F8F7A4FE002864D00320B3490870BD4849
:10BE700045688668C768201DFBF7ECFA8246524683
:10BE8000B9A103A8F7F732F803A9B8A0F7F71EF88D
:10BE9000002D4DD00220C0498875084640790979A7
:10BEA000BD4AD278CDE900210290BB488378427820
:10BEB0000178BAA0F7F70AF8290EB7484173290CA0
:10BEC0000173290AC17201468D72407B00900846B9
:10BED000037BC27A817AC0A0F6F7F8FF310EAE4834
:10BEE0004174310C0174310AC17301468E73407C78
:10BEF00000900846037CC27B817BC5A0F6F7E6FF75
:10BF0000390EA5484175390C0175390AC1740146CD
:10BF10008F74407D00900846037DC27C817C00E0E8
:10BF200002E1CAA0F6F7D2FF9B4881690220884748
:10BF3000F5E0D4F8249099F806000428F8DD0420F0
:10BF40007D490870FF20944988750846807A01066B
:10BF50009148C07A41EA00418F48007B41EA0020C5
:10BF60008D49497B084302068B48807A01068A483E
:10BF7000C07A41EA00418848007B41EA00218648B6
:10BF8000407B014301F47F4042EA00228248807AEC
:10BF900001068148C07A41EA00417F48007B41EABE
:10BFA00000207D49497B084300F47F0042EA1022CB
:10BFB0007948807A01067848C07A41EA004176489B
:10BFC000007B41EA00207449497B084342EA106043
:10BFD000644948607048807B01066F48C07B41EA35
:10BFE00000416D48007C41EA00206B49497C0843D0
:10BFF00002066948807B01066748C07B41EA004130
:10C000006548007C41EA00216348407C014301F41B
:10C010007F4042EA00226048807B01065E48C07B88
:10C0200041EA00415C48007C41EA00205A49497CD1
:10C03000084300F47F0042EA10225748807B010643
:10C040005548C07B41EA00415348007C41EA002149
:10C050005148407C014342EA1160424988604E48A1
:10C06000807C01064C48C07C41EA00414A48007D82
:10C0700041EA00204849497D084302064648807C41
:10C0800001064548C07C41EA00414348007D41EA41
:10C0900000204149497D084300F47F4042EA0022E4
:10C0A0003D48807C01063C48C07C41EA00413A485A
:10C0B000007D41EA00213848407D014301F47F00C2
:10C0C00042EA10223448807C01063348C07C41EAB1
:10C0D00000413148007D41EA00212F48407D014365
:10C0E00042EA11601F49C86001F10C031A1F091DC3
:10C0F000204602F049FD201DFBF7ACF9824652466E
:10C1000019A103A8F6F7F2FE5FA0F6F7DFFE03A978
:10C1100062A0F6F7DBFE204881690220884704E030
:10C1200000200549087000E000BF00BF4FF47A709E
:10C130000CF0C0FF79E60000940200205374617493
:10C14000653A204C6F6F6B696E6720666F72204492
:10C1500048435020736572766572202E2E2E0D0A8C
:10C1600000000000804F012025730000495020612D
:10C170006464726573732061737369676E656420AC
:10C18000627920612044484350207365727665725D
:10C190003A2025730D0A0000644F0120E7BD91E5A8
:10C1A0008DA1656EE79A844D4143E59CB0E59D8085
:10C1B000E4B8BA3A2E2E2E2E2E2E2E2E2E2E2E2EC7
:10C1C0002E2E2E2E25642E25642E25642E25642EDB
:10C1D00025642E25640D0A00E9809AE8BF8744484B
:10C1E0004350E88EB7E58F96E588B04950E59CB09E
:10C1F000E59D802E2E2E2E2E2E2E2E2E2E2E2E2EE7
:10C200002E25642E25642E25642E25640D0A00003B
:10C21000E9809AE8BF8744484350E88EB7E58F9697
:10C22000E588B0E5AD90E7BD91E68EA9E7A0812E47
:10C230002E2E2E2E2E2E2E2E2E2E2E25642E2564C4
:10C240002E25642E25640D0A00000000E9809AE87E
:10C25000BF8744484350E88EB7E58F96E588B0E73E
:10C260009A84E9BB98E8AEA4E7BD91E585B32E2E8C
:10C270002E2E2E2E2E2E2E2E25642E25642E256457
:10C280002E25640D0A000000444843502054696D77
:10C29000656F7574202121200D0A000053746174AC
:10C2A000696320495020616464726573733A202584
:10C2B000730D0A0008B56946084800680DF076FC61
:10C2C00000BF009838B14FF0805005490860BFF3B7
:10C2D0004F8FBFF36F8F00BF08BD0000900200209A
:10C2E00004ED00E0F0B504460D461646059F00211A
:10C2F00017E0606900EBC1021068A84210D12EB1AE
:10C30000107900F0010008B10120F0BD2BB11079C7
:10C3100000F0020008B10120F7E70FB10120F4E7B7
:10C32000491CA0698842E4D80020EEE72DE9FC41D1
:10C3300004460D4616461F46002000903B463246F6
:10C3400029460190204600F04BF9BDE8FC81000031
:10C350002DE9FF4F83B004468B461F464FF0080A75
:10C3600000260598B0F1004F01D2059801E06FF06A
:10C370000040804600BF24B900BF59A0F6F7A6FDD3
:10C3800000BF00BF00BF2068007800F0F000102858
:10C3900004D000BF56A0F6F799FD00BF00BF07F01C
:10C3A000080008B14AF0040A00BF00BF00BF60687F
:10C3B00010B16068029031E0524602A9206802F094
:10C3C00053F8814600BF00BFB9F1000F1BD0002E0B
:10C3D00000DD74E000BF00BF00BF4846F8F7E6FF8D
:10C3E000019000BF019810B14A490198086000BF50
:10C3F00000BF09F10F0018B9002007B0BDE8F08FA9
:10C400004FF0FF30F9E700BF029820B900BF42A00B
:10C41000F6F75CFD00BF00BF0298606000BF00BF80
:10C4200002980089404502DA0298058901E01FFA66
:10C4300088F57019B04203DA6FF00040801B85B2B6
:10C440000BEB060100232A46029802F03DFF2E4422
:10C4500000BFA84504DA00BF32A0F6F737FD00BFE1
:10C4600000BFA8EB050807F00100E8B900BF02987B
:10C470000089A84204DA00BF34A0F6F727FD00BF08
:10C4800000BF02980089401B002806DD294602985B
:10C4900003F046F9606000BF06E00020606000BF66
:10C4A00000BF029803F0A0F84AF0140AB8F1000F98
:10C4B00004DD07F0010000283FF477AF00BF002E35
:10C4C00006DD07F0010018B93146206802F054F883
:10C4D00000BF002000BF00BF00BF30468DE7000056
:10C4E0006E6F20736F636B657420676976656E008D
:10C4F000746869732073686F756C6420626520636B
:10C500006865636B656420696E7465726E616C6CDE
:10C5100079000000980200207020213D204E554CEB
:10C520004C000000696E76616C696420636F7079FD
:10C530006C656E2C206C656E20776F756C64207551
:10C540006E646572666C6F7700000000696E7661DC
:10C550006C696420636F70796C656E002DE9FE4331
:10C5600004460D4616469946DDE90A7814B90020BE
:10C57000BDE8FE83C5B1BEB1002302AA01A92068AF
:10C5800001F03CFD00BF00BF00BF00BF00BF00BF07
:10C590004DB146B100962B46BDF8082001A9206890
:10C5A00000F036FCE4E700BF0020E1E705462C463A
:10C5B000002610E00023D4E90912A069FFF7B6FEB7
:10C5C00006460020616A8855034904A0F6F77EFC00
:10C5D00001200CF06FFDEDE7B84F0120257300003E
:10C5E0002DE9FF4F8BB007468A461546DDE918B4A2
:10C5F00000BF00BF3846F9F79BFF064626B94FF04B
:10C60000FF300FB0BDE8F08F3068007800F0F00028
:10C61000102810D12A46514630460E9BFFF798FE4F
:10C6200080462EA3224659463046CDE90078FFF7D2
:10C6300095FF4046E5E700200A90CDF820A0099537
:10C6400005900690079008A8039001200490CDF86B
:10C6500004B00CB1206800E0002002900AAB01AAEF
:10C66000009730460E9900F043F88146B9F1000F6B
:10C6700011D000BF00BF00BF4846F8F797FE0090FA
:10C6800000BF009810B119490098086000BF00BFB2
:10C690004FF0FF30B5E7BDF82800854201D22846AB
:10C6A00001E0BDF828006FF00041884208D2BDF8D3
:10C6B0002800854201D2284604E0BDF8280001E0A8
:10C6C0006FF0004080460CB10298206000BF00BFB0
:10C6D000002000BF00BF00BF404692E76C77697042
:10C6E0005F7265637666726F6D00000098020020CD
:10C6F0002DE9FF5F0546894614469A4600BFA068AB
:10C7000060B9E068002809DD00BF46A0F6F7DEFB4F
:10C7100000BF6FF00F0004B0BDE8F09F00BF09F04C
:10C72000080010B14FF0040B01E04FF0000B00BF08
:10C7300000BF686803900398B0B95A4603A92868F7
:10C7400001F0BEFE029000BF00BF029808B102983F
:10C75000E1E700BF039820B900BF3DA0F6F7B6FBA4
:10C7600000BF00BF0398686003980068B0F80880B5
:10C7700000BF00BF0027002620E0A8EB070080B222
:10C780000090A06800EBC60041680098814202D981
:10C790000098019005E0A06800EBC600808880B298
:10C7A0000190A26852F83610039A3B461068019A2D
:10C7B00002F08AFD0198384487B2761CE068B042E6
:10C7C00001DD4745D9DB2068A0B1606890B100BFAA
:10C7D00000BF00BF00BF00BF00BF206850B160684D
:10C7E00040B1201D0090236803998A890831286888
:10C7F00000F00EFB0020A061206920B1002008B9E4
:10C800000021616100BF09F0010020B900206860CB
:10C81000039801F0F5F9BAF1000F01D0AAF80080F1
:10C82000002078E76C7769705F7265637666726F77
:10C830006D5F7564705F7261773A20696E76616CC6
:10C84000696420617267756D656E74730000000025
:10C8500062756620213D204E554C4C002DE9FE4F5F
:10C8600081468A4693461D4600BF00BF4846F9F7F9
:10C870005FFE04461CB94FF0FF30BDE8FE8F206814
:10C88000007800F0F000102809D0002000902B461E
:10C890005A4651460190484600F034F8EDE705F05D
:10C8A000100008B1022000E0002040F0010005F077
:10C8B000080109B1042100E0002140EA010700203D
:10C8C000029002A800903B465A465146206801F06B
:10C8D000B3FE064600BF00BF00BF3046F8F766FD56
:10C8E000804600BFB8F1000F02D00548C0F80080B4
:10C8F00000BF00BF0EB90298BFE74FF0FF30BCE7A2
:10C90000980200202DE9FF4F85B01746DDE9124956
:10C910000598F9F70DFE8046B8F1000F04D14FF0ED
:10C92000FF3009B0BDE8F08FD8F80000007800F0C3
:10C93000F000102806D13A46089BDDE90501FFF713
:10C940008DFFEEE7B7F5803F0AD300BF5A2000BF46
:10C950005A21354A116000BF00BF4FF0FF30E0E7B9
:10C960001FFA87FA00BF14B9B9F1000F20D0B9F14E
:10C97000100F06D12CB16078022802D104F0030018
:10C98000B0B100BF29A0F6F7A1FA00BF00BF6FF059
:10C990000F00F8F70BFD834600BFBBF1000F02D07C
:10C9A0002148C0F800B000BF00BF4FF0FF30B8E72B
:10C9B00000BF0020029001903CB100BF606803906E
:10C9C0006088FEF77EFB064602E00026002003900A
:10C9D000ADF8106000BF00BF00BF00BF00BF00BFC8
:10C9E000524601A8069901F03FF905462DB901A963
:10C9F000D8F8000001F094FD054601A801F010F9F7
:10CA000000BF2846F8F7D2FC834600BFBBF1000FF9
:10CA100002D00548C0F800B000BF00BF0DB95046B5
:10CA20007FE74FF0FF307CE7980200206C77697059
:10CA30005F73656E64746F3A20696E76616C6964C9
:10CA40002061646472657373000000002DE9F84F83
:10CA500006460F4690461C46DDF8289000253046D5
:10CA6000F9F766FD8246BAF1000F02D1681EBDE8F3
:10CA7000F88F54B900BF0E2000BF0E21114A11607B
:10CA800000BF00BF4FF0FF30F1E70F4804F044FE55
:10CA90002346424639463046CDF8009000F016F85D
:10CAA0000546094804F09AFE00BF284600BF08B1B9
:10CAB0000449086000BF00BF15B14FF0FF30D6E752
:10CAC0000020D4E798020020B40100202DE9F84F9F
:10CAD0008246894616461D460A9F00200090504611
:10CAE0000AF008FB044614B90920BDE8F88FB9F133
:10CAF000000F71D0B9F1060F6FD0B9F1FF0F6DD0F3
:10CB0000A9F6FF7000286AD141F20601701A8E4220
:10CB10003CD004DC082E08D0202E72D104E004287A
:10CB200053D00528F9D185E000BF202E07D1206819
:10CB3000007800F0F000202801D05C20D5E73046D6
:10CB400000F02CFA064600BF00BF042F01D21620C9
:10CB5000CBE700BF206810B12068406808B91620F4
:10CB6000C3E700BF286838B120684068407A304386
:10CB700021684968487206E020684068407AB043FE
:10CB800021684968487200BF00BF93E000BF00BF42
:10CB9000082F01D21620A8E700BF206808B9162088
:10CBA000A3E700BF4FF47A72686890FBF2F02A683E
:10CBB00002EB4203C3EBC21200EBC201002901DA0F
:10CBC000162092E72068C16174E000BF00BF00BF7B
:10CBD000042F05D2162088E76EE0A4E0F1E0F8E02B
:10CBE00000BF206810B12068406808B916207CE7B3
:10CBF00000BF2068007800F0F000202802D05C2000
:10CC000073E752E000BF286848B100BF2068406861
:10CC1000007C40F0010021684968087409E000BF09
:10CC200020684068007C00F0FE00216849680874B4
:10CC300000BF3FE04FF0000B00BF00BF062F01D246
:10CC4000162052E700BF206808B916204DE700BF44
:10CC5000A846454698F8000040B1404601F014FF50
:10CC60008346BBF1000F01D113203EE72068007816
:10CC700000F0F000102802D020280CD105E0216837
:10CC80004868594605F083F90DE02168486859461F
:10CC90000AF0CAFA07E000BF00BF52A0F6F716F983
:10CCA00000BF00BF00BF00BF04E000BF00BF5C20AA
:10CCB000009000BF00BF91E0012E17D0022E2BD1B3
:10CCC00000BF00BF042F01D216200EE700BF20686E
:10CCD00010B12068406808B9162006E700BF287820
:10CCE00021684968C87200BF00BF1AE000BF00BFDA
:10CCF000042F01D21620F8E600BF206810B120688A
:10CD0000406808B91620F0E600BF28782168496815
:10CD1000887200BF00BF04E000BF00BF5C2000902D
:10CD200000BF00BF5AE000BF00BF00BF042F01D208
:10CD30001620DAE600BF206810B12068406808B904
:10CD40001620D2E600BF2068007800F0F00010281E
:10CD500001D05C20C9E600BF20684068007D012842
:10CD600001D11620C1E6012E02D0022E22D119E0F7
:10CD7000286848B100BF20684068408B40F0400000
:10CD80002168496848830AE000BF20684068408BFA
:10CD90004FF6BF71084021684968488300BF00BF53
:10CDA00000BF0CE0286821684968C1F8900000BF06
:10CDB00000BF04E000BF00BF5C20009000BF00BFC8
:10CDC0000CE000BF00BF00BF5C20009000BF00BFB0
:10CDD00004E000BF00BF5C20009000BF00BF0098CF
:10CDE00083E60000556E68616E646C6564206E6554
:10CDF00074636F6E6E207479706520696E20534F76
:10CE00005F42494E44544F44455649434500000053
:10CE10002DE9FF4781460D4617461E460C9C4FF0F4
:10CE2000000800BF25B900BF1FA0F6F74FF800BFEC
:10CE300000BF00BF26B900BF20A0F6F747F800BF2B
:10CE400000BF00BF24B900BF20A0F6F73FF800BF25
:10CE500000BF00BF10208DF8000002208DF80100F7
:10CE60003846FEF72EF9ADF8020028680190002040
:10CE70000290039000BF9DF800102068884202D203
:10CE80004FF0010807E09DF800102068884202D9A1
:10CE90009DF800002060694630462268F3F742FAA8
:10CEA000404604B0BDE8F08766726F6D61646472DD
:10CEB00020213D204E554C4C0000000066726F6DE5
:10CEC00020213D204E554C4C0000000066726F6DD5
:10CED0006C656E20213D204E554C4C002DE9F041F3
:10CEE00080460F461646012F1AD0022F0AD0032F74
:10CEF0001FD1F1B2274A402001F0E8F8044600BFF4
:10CF000000BF21E0882E01D1212100E02021084628
:10CF1000204A002101F0DAF8044600BF00BF13E008
:10CF20001C4A0021102001F0D1F8044600BF00BFC8
:10CF30000AE000BF00BF00BF16201749086000BF0D
:10CF40004FF0FF30BDE8F08100BF4CB900BF00BF1B
:10CF500000BF69201049086000BF4FF0FF30F1E7C3
:10CF600000212046F6F736FA0546681C50B92046DF
:10CF700000F050FF00BF17200749086000BF4FF0C6
:10CF8000FF30DFE7A56100BF00BF00BF00BF28463C
:10CF9000D8E70000D56300089802002010B50446C9
:10CFA000042C06D0082C02D0202C04D110BD08205F
:10CFB000FCE70420FAE700BF00BF03A0F5F786FFF7
:10CFC00000BF00BF0020F1E7556E6B6E6F776E20DB
:10CFD000736F636B6574206F7074696F6E0000000F
:10CFE000F8B505460A462B4600200090002103F0C4
:10CFF000010636B1002A04DD13F8010B8DF801009B
:10D00000521E1C4603E034F8027B3944921E012A6A
:10D01000F9DC002A02DD20788DF80000BDF8000060
:10D02000014488B200EB114188B200EB114126B1F6
:10D03000C8B2C1F3072747EA002188B2F8BD000053
:10D0400030B58BB0044604F00100002831D04FF613
:10D05000FF700090494802886E231E210520FDF7CD
:10D0600021F84FF4784046A110221346CDE9002163
:10D070000290C8221E210520FDF7A2FC4FF4784043
:10D0800041A110221346CDE9002102904FF4C8724D
:10D0900032210520FDF794FC4FF4784040A1102286
:10D0A0001346CDE900210290C82246210520FDF754
:10D0B00087FC04F0020000285DD04FF6FF7000905E
:10D0C0002E48438802886E210520FCF7EBFF1F20C5
:10D0D00037A110221346CDE900210290C8226E210B
:10D0E0000520FDF76DFC3748807D02280DD13548BD
:10D0F000407B3449097BCDE900103248C37A827AFB
:10D1000031A103A8F5F7F2FE0CE02E48407B2D4933
:10D11000097BCDE900102B48C37A827A2FA103A89E
:10D12000F5F7E4FE1F2003A910221346CDE90021E4
:10D130000290C82282210520FDF742FCF8F78AFF01
:10D14000054665B11F202BA110221346CDE9002111
:10D150000290C82296210520FDF732FC0BE01F202B
:10D1600029A110221346CDE900210290C822962160
:10D170000520FDF725FC0BB030BD00009004002019
:10D1800053544D33320000006C77495020554450C1
:10D1900042726F616463617374546573740000005C
:10D1A00041544F4D40414C49454E54454B000000C1
:10D1B0006C77495020496E697420537563636573B9
:10D1C00073656400644F0120444843502049503A3D
:10D1D00025642E25642E25642E2564005374617405
:10D1E00069632049503A25642E25642E25642E2536
:10D1F0006400000045746865726E65742053706544
:10D2000065643A3130304D0045746865726E6574FE
:10D210002053706565643A31304D000010B5F4F765
:10D22000E1FB0723022208214FF4A87004F0EEFB73
:10D23000A820F6F72DF94FF4E1300AF0F1FC0C4884
:10D24000416854208847FDF74DFCFCF755FFFAF77D
:10D2500051FC03F0EBFE002000F016FC022000F071
:10D2600013FC012000F010FCF9F74AF9002010BD72
:10D270008C00002070B5054615B900BF00BF70BD19
:10D2800005F0030088B100BF00BF38A0F5F71EFE0F
:10D2900000BF00BF00BF00BF00BF04F00DF906468D
:10D2A000304604F067F900BFE9E7A5F10804384803
:10D2B0000068844205D305F10C00364909688842AC
:10D2C00011D900BF00BF34A0F5F700FE00BF00BFBA
:10D2D00000BF00BF00BF04F0EFF80646304604F080
:10D2E00049F900BFCBE7334804F016FA2079A0B91A
:10D2F00000BF00BF30A0F5F7E9FD00BF00BF2D481B
:10D3000004F06CFA00BF00BF00BF04F0D5F8064679
:10D31000304604F02FF900BFB1E7204600F0C6F810
:10D32000A0B900BF00BF2EA0F5F7D0FD00BF00BF21
:10D33000204804F053FA00BF00BF00BF04F0BCF85F
:10D340000646304604F016F900BF98E70020207129
:10D3500030480068844201D22E480460204602F022
:10D360008BFC144804F03AFA00BF88E76D656D5FE6
:10D37000667265653A2073616E69747920636865C9
:10D38000636B20616C69676E6D656E7400000000F0
:10D39000C4010020C80100206D656D5F667265657F
:10D3A0003A20696C6C6567616C206D656D6F727990
:10D3B00000000000CC0100206D656D5F6672656540
:10D3C0003A20696C6C6567616C206D656D6F727970
:10D3D0003A20646F75626C652066726565000000B6
:10D3E0006D656D5F667265653A20696C6C65676135
:10D3F0006C206D656D6F72793A206E6F6E2D6C6961
:10D400006E6B65643A20646F75626C652066726548
:10D4100065000000D001002010B500BF00BF174814
:10D4200020F0030016490860084604684FF4C8401D
:10D4300020800020608020714FF4C84003F0E4FA9F
:10D44000104908600120096808714FF4C8400D496F
:10D45000096808800B4909684880094800680A493A
:10D4600008600A4804F09CF930B100BF00BF08A072
:10D47000F5F72CFD00BF00BF10BD00005B5F002072
:10D48000C4010020C8010020D0010020CC010020F0
:10D490006661696C656420746F2063726561746590
:10D4A000206D656D5F6D7574657800002DE9F04144
:10D4B0000446204600F046F90546208803F0A4FA09
:10D4C0000646608803F0A0FA07462088B0F5C84FEA
:10D4D00010D86088B0F5C84F0CD86088A84202D038
:10D4E0003888A84206D106480068864205D0708870
:10D4F000A84202D00020BDE8F0810120FBE7000037
:10D50000C80100202DE9F0478146B9F1000F02D192
:10D510000020BDE8F08709F1030020F0030085B288
:10D520000C2D00D20C25B5F5C84F01D84D4501DAB8
:10D530000020EEE7534804F0EFF85348006800F08D
:10D5400001F9064692E0304603F05EFA044620797F
:10D5500000286AD1218806F10800081AA84264D37D
:10D56000218806F10800091A05F11400814225D32B
:10D5700006F1080028441FFA80F800BFB8F5C84F2C
:10D5800004D100BF41A0F5F7A1FC00BF00BF404699
:10D5900003F03AFA074600213971218839807E80EC
:10D5A000A4F80080012020713888B0F5C84F07D05A
:10D5B000388803F029FAA0F8028001E001202071E8
:10D5C00031480068844223D12F48D0F800A004E0FD
:10D5D000BAF8000003F018FA82469AF8040018B16D
:10D5E0002F4800688245F3D12748C0F800A000BF4B
:10D5F00000682B490968884208D0234800680079F0
:10D6000020B100BF27A0F5F761FC00BF00BF00BF3D
:10D610001C4804F0E3F800BF04F108002844204946
:10D620000968884206D900BF00E01BE024A0F5F796
:10D630004DFC00BF00BF00BF04F0030020B100BFDD
:10D640002BA0F5F743FC00BF00BF00BF04F00300B0
:10D6500020B100BF32A0F5F739FC00BF00BF04F1D4
:10D66000080056E7304603F0CFF90688C5F5C840F4
:10D67000B0423FF668AF034804F0B0F800BF00BF07
:10D68000002046E7CC010020D0010020696E7661C1
:10D690006C6964206E6578742070747200000000FC
:10D6A000C80100206D656D5F6D616C6C6F633A2021
:10D6B000216C667265652D3E75736564000000001F
:10D6C0006D656D5F6D616C6C6F633A20616C6C6F42
:10D6D0006361746564206D656D6F7279206E6F741F
:10D6E0002061626F76652072616D5F656E642E00E9
:10D6F0006D656D5F6D616C6C6F633A20616C6C6F12
:10D700006361746564206D656D6F72792070726FEE
:10D710007065726C7920616C69676E65642E0000BB
:10D720006D656D5F6D616C6C6F633A2073616E69DE
:10D73000747920636865636B20616C69676E6D65E1
:10D740006E740000014602480088081A80B27047D3
:10D75000C40100202DE9F84F81468B460BF10300F0
:10D7600020F0030085B20C2D00D20C25B5F5C84F72
:10D7700001D85D4502DA0020BDE8F88F00BF5548AA
:10D780000068814503D354480068814504D300BF35
:10D7900052A0F5F79BFB00BF00BF4E4800688145D3
:10D7A00003D34D48006881450BD300BF00BF00BFC5
:10D7B00003F082FE0090009803F0DCFE00BF4846B4
:10D7C000DAE7A9F108063046FFF7BCFF07463188C3
:10D7D000C81B08381FFA80FA00BF554504DD00BF9A
:10D7E00044A0F5F773FB00BF00BF554501DD0020E5
:10D7F000C2E7554501D14846BEE7464803F08CFFD5
:10D80000308803F001F90446207978BB00BF3088E6
:10D81000B0F5C84F04D100BF3FA0F5F757FB00BFDC
:10D8200000BF2088009007F1080028441FFA80F804
:10D830003E480068A04204D1404603F0E5F83B4969
:10D840000860404603F0E0F804460020207100988C
:10D8500020806780A6F800802088B0F5C84F04D0EB
:10D86000208803F0D1F8A0F802802EE0FFE705F150
:10D870001400504529D807F1080028441FFA80F801
:10D8800000BF3088B0F5C84F04D100BF22A0F5F723
:10D890001DFB00BF00BF404603F0B6F80446234816
:10D8A0000068844201D22148046000202071308841
:10D8B00020806780A6F800802088B0F5C84F04D08B
:10D8C000208803F0A1F8A0F80280124803F086FF38
:10D8D000484651E7C4010020C80100206D656D5F16
:10D8E0007472696D3A206C6567616C206D656D6F4F
:10D8F000727900006D656D5F7472696D2063616E91
:10D90000206F6E6C7920736872696E6B206D656D27
:10D910006F727900CC010020696E76616C696420B9
:10D920006E6578742070747200000000D0010020D1
:10D9300070B504460D4600BF0E2C05DB00BF08A0E5
:10D94000F5F7C4FA00BF70BD00BF05B9FBE70B498E
:10D9500051F824002946F7F703FC00BFF3E7000065
:10D960006D656D705F667265653A207479706520CB
:10D970003C204D454D505F4D4158000098DA01085C
:10D9800010B5002406E0054951F8240000F008F81D
:10D99000601C84B20E2CF6D310BD000098DA01088A
:10D9A00010B50023C46823608368DB1C23F00301E7
:10D9B000002207E0C3681B680B60C3681960838896
:10D9C0001944521CC3889342F4DC10BD70B5044660
:10D9D00000BF0E2C06DB00BF07A0F5F777FA00BFEB
:10D9E000002070BD00BF0C4951F82400F7F7E4FB9C
:10D9F00005462846F5E700006D656D705F6D616C4A
:10DA00006C6F633A2074797065203C204D454D5011
:10DA10005F4D41580000000098DA01082DE9F041FF
:10DA200004460E461548005D38B914482038016890
:10DA3000204688470120BDE8F081114850F82400B5
:10DA4000B04219D90F4850F82400B6FBF0F10B484A
:10DA50000C3850F8240030F81120002508E000238D
:10DA600006480C3850F824004F1920F817306D1C68
:10DA70009542F4DB0020DEE70220DCE7A001002075
:10DA800064D9010858D9010830B50446022508496F
:10DA900051F8241001FB05F2064951F82400002139
:10DAA00000F07EF8012103480C30015530BD000024
:10DAB0004CD90108940100202DE9F04704460F4697
:10DAC0000025A9462348005D20B922482038016876
:10DAD000204688471FB94FF0FF30BDE8F0871E4849
:10DAE00050F82400B7FBF0F61B4850F82400B7FBB1
:10DAF000F0F100FB117000B1761C184850F82400BA
:10DB0000451E22E013480C3850F8240030F8150068
:10DB100010B909F1010901E04FF00009B14513D135
:10DB20004FF0000809E00B480C3850F8240005EBD2
:10DB3000080220F8126008F10108B045F3D3064846
:10DB400050F824006843C8E76D1E002DDADA4FF064
:10DB5000FF30C2E7A001002058D901084CD90108C4
:10DB600010B501460023002207E00B4850F82100C1
:10DB700030F8120000B15B1C521C084850F821001C
:10DB80009042F2D84FF47A705843044C54F8214034
:10DB9000B0FBF4F080B210BD940100204CD9010814
:10DBA00030B5034601E003F8011B141EA2F1010287
:10DBB000F9D130BD70B505460C4604B970BD0548B5
:10DBC00050F82500261A31462846FFF727FF00BFE8
:10DBD000F4E700008801002070B504460E46314687
:10DBE0002046FFF769FF0546681C08B9002070BD94
:10DBF000024850F824002844F9E70000880100207A
:10DC000010B504465CB1206828B1206801F0ECFC36
:10DC100000206060206021460620FFF789FE10BDCD
:10DC200010B5044600BF2CB900BF08A0F5F74EF9A7
:10DC300000BF10BD00BF206810B1206801F0D4FC07
:10DC400000206060206000BFF3E700006E65746232
:10DC500075665F667265653A20696E76616C6964A7
:10DC6000206275660000000070B504460D46164639
:10DC700000BF3CB900BF11A0F5F728F900BF6FF055
:10DC80000F0070BD00BF206810B1206801F0ACFC2F
:10DC900041220021362001F0D1F82060206818B917
:10DCA00000206060401EECE7206845602068068127
:10DCB00020684681206860600020E2E76E6574623B
:10DCC00075665F7265663A20696E76616C6964207C
:10DCD000627566002DE9F04105460F464FF00008D9
:10DCE0000720FFF773FE044614B90020BDE8F08159
:10DCF000002020722570606005F0F000102803D02D
:10DD0000202803D10A2609E00A2607E000BF00BF49
:10DD100015A0F5F7DBF800BF00BF1FE000BF3146DC
:10DD200004F1100003F082FC00B117E0002104F1BF
:10DD30000C0003F0C3FD20B104F1100003F04CFC13
:10DD40000CE0002060616070401EA061A7620020AE
:10DD50006062E06184F820802046C7E72146072002
:10DD6000FFF7E6FD0020C1E76E6574636F6E6E5FBE
:10DD7000616C6C6F633A20756E646566696E65648C
:10DD8000206E6574636F6E6E5F747970650000005D
:10DD900070B506460C46FA202071206800F10C028E
:10DDA0002146304609F0CCF8054615B994F904002F
:10DDB00070BD2846FCE7000070B588B004460D46EB
:10DDC00000BF44B900BF0BA0F5F780F800BF6FF0AB
:10DDD0000F0008B070BD00BF00948DF808502921D5
:10DDE0008DF8091069460A48FFF7D2FF064630460B
:10DDF000EFE700006E6574636F6E6E5F636C6F7348
:10DE0000653A20696E76616C696420636F6E6E009E
:10DE100011B2000870B505460DB9002070BD284646
:10DE200000F0ECF9044614B9284600F065F82046E5
:10DE3000F4E77CB5044604F1100008B32069F8B19A
:10DE400010E0207800F0F000102808D16946019811
:10DE5000FDF7B6FF10B9019801F0C6FB02E001988A
:10DE6000FFF7CEFE01A904F1100003F0DDFA401C1B
:10DE70000028E6D104F1100003F0AEFB0020206181
:10DE800004F1140028B3606918B314E069460198DE
:10DE9000FDF796FF70B9019D2846FFF7CAFF686835
:10DEA00020B1686803F0F8FF00206860284600F0A1
:10DEB00023F800BF00BF01A904F1140003F0B4FA75
:10DEC000401C0028E2D104F1140003F085FB00207F
:10DED00060617CBD70B504460CB9002070BD03F0D4
:10DEE000EBFA064694F9085000202072304603F001
:10DEF00041FB2846F2E7000010B5044600BF606809
:10DF000020B100BF13A0F4F7E1FF00BF00BF00BFC6
:10DF100004F1100030B1206920B100BF19A0F4F75E
:10DF2000D5FF00BF00BF00BF04F1140030B160692D
:10DF300020B100BF22A0F4F7C9FF00BF00BF04F169
:10DF40000C0003F091FC0020E06021460720FFF761
:10DF5000EFFC10BD504342206D7573742062652044
:10DF60006465616C6C6F6361746564206F75747354
:10DF700069646520746869732066756E6374696F7F
:10DF80006E000000726563766D626F78206D757348
:10DF900074206265206465616C6C6F636174656494
:10DFA000206265666F72652063616C6C696E6720C4
:10DFB000746869732066756E6374696F6E00000023
:10DFC0006163636570746D626F78206D7573742022
:10DFD0006265206465616C6C6F6361746564206266
:10DFE00065666F72652063616C6C696E672074682A
:10DFF00069732066756E6374696F6E002DE9F04178
:10E0000088B004460D4616461F4600BF4CB900BFF7
:10E0100015A0F4F75BFF00BF6FF00F0008B0BDE87C
:10E02000F08100BF00BF3DB900BF17A0F4F74EFF5D
:10E0300000BF6FF00F00F1E700BF00BF3EB900BFA7
:10E0400019A0F4F743FF00BF6FF00F00E6E700BF31
:10E0500000948DF810700295039669461A48FFF7F0
:10E0600097FE80464046D9E76E6574636F6E6E5FBB
:10E07000676574616464723A20696E76616C696484
:10E0800020636F6E6E0000006E6574636F6E6E5F6E
:10E09000676574616464723A20696E76616C696464
:10E0A00020616464720000006E6574636F6E6E5F61
:10E0B000676574616464723A20696E76616C696444
:10E0C00020706F727400000051B700082DE9F04114
:10E0D00088B007460D46164631463846FFF7FAFD2A
:10E0E0000446002C48D08DF8085000946946234817
:10E0F000FFF74EFE8046B8F1000F3CD000BF6068CD
:10E1000020B100BF1EA0F4F7E1FE00BF00BF00BFBA
:10E1100004F1100008B1206920B900BF21A0F4F774
:10E12000D5FE00BF00BF00BF04F1140030B160692C
:10E1300020B100BF21A0F4F7C9FE00BF00BF00BF9F
:10E1400004F10C0008B1E06820B900BF24A0F4F786
:10E15000BDFE00BF00BF04F10C0003F085FB04F11D
:10E16000100003F039FA21460720FFF7E1FB0020F9
:10E1700008B0BDE8F08100BF2046F9E721B80008EB
:10E1800066726565696E6720636F6E6E207769746D
:10E19000686F75742066726565696E67207063626A
:10E1A00000000000636F6E6E20686173206E6F2048
:10E1B000726563766D626F7800000000636F6E6E4B
:10E1C0002D3E6163636570746D626F782073686F54
:10E1D000756C646E277420657869737400000000A4
:10E1E000636F6E6E20686173206E6F206F705F6367
:10E1F0006F6D706C657465640000000030B589B0A7
:10E20000044614B9002009B030BD019429218DF8CD
:10E210000D1001A90448FFF7BBFD05460DB12846C6
:10E22000F1E70020EFE70000BDB500082DE9FC4153
:10E2300004460D4617460020019000BF45B900BFB7
:10E2400045A0F4F743FE00BF6FF00F00BDE8FC816E
:10E2500000BF0020286000BF3CB900BF46A0F4F713
:10E2600035FE00BF6FF00F00F0E700BF04F11000B3
:10E2700008B1206958B92046FFF72CFE8046B8F156
:10E28000000F01D04046E1E76FF00A00DEE794F8A6
:10E29000200000F0020048B907F0040030B994F8FB
:10E2A000200000F0010008B9207AD8B101A904F1DA
:10E2B000100003F0B9F8401C98B92046FFF70AFE99
:10E2C0008046B8F1000F01D04046BFE794F8200027
:10E2D00000F0010010B16FF00A00B7E76FF0060020
:10E2E000B4E70AE001A904F11000E26903F03EF886
:10E2F000401C10B96FF00200A8E7207800F0F00091
:10E30000102810D169460198FDF75AFD40B19DF9DA
:10E3100000000F3008B9002098E79DF9000095E74C
:10E32000019806890BE000BF019820B900BF19A031
:10E33000F4F7CCFD00BF00BF019800680689A06A11
:10E3400020B1324601212046A36A984700BF00BF92
:10E3500001982860002079E76E6574636F6E6E5FC8
:10E36000726563763A20696E76616C696420706FBD
:10E37000696E7465720000006E6574636F6E6E5F27
:10E38000726563763A20696E76616C696420636FAA
:10E390006E6E000062756620213D204E554C4C008B
:10E3A0002DE9F04389B004468846174604F1100071
:10E3B00008B1206920B96FF00A0009B0BDE8F08308
:10E3C00094F8200000F0800040B100BF94F82000D5
:10E3D00000F07F0084F8200000BF28E03A46414664
:10E3E0002046FFF723FF05460DB12846E5E7D8F89C
:10E3F000006007F0080050B90EB1308900E001203C
:10E40000814601AA4946204600F0E6F800BF46BB17
:10E4100007F0100050B100BF94F8200040F08000D9
:10E4200084F8200000BF6FF00600C6E700BFA06AB6
:10E4300020B1002201212046A36A9847606848B9AC
:10E440002046FFF747FD05460DB12846B5E76FF0BA
:10E450000D00B2E701212046FFF7AEFC6FF00E0081
:10E46000ABE72846A9E7000070B504460D461646FE
:10E4700000BF24B1207800F0F000102807D000BFC2
:10E4800006A0F4F723FD00BF6FF00F0070BD00BFC2
:10E49000324629462046FFF783FFF7E76E6574632F
:10E4A0006F6E6E5F726563765F7463705F706275C6
:10E4B000663A20696E76616C696420636F6E6E00E7
:10E4C00070B504460D46164600BF24B1207800F012
:10E4D000F000102807D100BF06A0F4F7F7FC00BF3A
:10E4E0006FF00F0070BD00BF324629462046FFF78F
:10E4F0009DFEF7E76E6574636F6E6E5F726563769F
:10E500005F7564705F7261775F6E65746275663A9D
:10E5100020696E76616C696420636F6E6E00000026
:10E5200070B588B004460D4600BF44B900BF0AA0CC
:10E53000F4F7CCFC00BF6FF00F0008B070BD00BF57
:10E5400000BF00BF0094029569460A48FFF720FC0F
:10E5500006463046F1E700006E6574636F6E6E5FCD
:10E5600073656E643A20696E76616C696420636FCE
:10E570006E6E000081B8000870B588B004460D4684
:10E5800000BF24B1207800F0F000102808D000BFB0
:10E5900008A0F4F79BFC00BF6FF00F0008B070BD3F
:10E5A00000BF6A462946204600F016F80646304667
:10E5B000F4E700006E6574636F6E6E5F726563767C
:10E5C0005F7463705F706275663A20696E76616C25
:10E5D000696420636F6E6E0070B504460E46154682
:10E5E00000BF24B1207800F0F000102807D000BF51
:10E5F00007A0F4F76BFC00BF6FF00F0070BD00BF09
:10E600002C60AE6029460B48FFF7C2FBF6E700001E
:10E610006E6574636F6E6E5F726563765F74637050
:10E620005F706275663A20696E76616C696420631A
:10E630006F6E6E0039B800082DE9FE4306460C46A1
:10E6400015461F46DDF82880019402953B460122BD
:10E6500001A93046CDF8008000F002F8BDE8FE8345
:10E660002DE9F04F89B005460F4691469A46DDF8F0
:10E67000488000BF4DB900BF3AA0F4F727FC00BFA7
:10E680006FF00F0009B0BDE8F08F00BF00BF287821
:10E6900000F0F000102807D000BF39A0F4F716FCF6
:10E6A00000BF6FF00500EDE700BF95F8200000F017
:10E6B000020010B90AF0040008B1012000E00020B7
:10E6C0000090009828B1B8F1000F02D16FF005005A
:10E6D000D8E7002400260CE007EBC600406804449D
:10E6E00007EBC6004068A04202D96FF00500C9E7F9
:10E6F000761C4E45F0DB0CB90020C3E7B4F1004FA7
:10E7000009D3B8F1000F02D16FF00500BAE76FF03E
:10E7100000410C4600BF01950397ADF81090002111
:10E7200005918DF820A00694079101A91D48FFF7D7
:10E730002FFB8346BBF1000F11D1B8F1000F02D0BF
:10E740000798C8F80000009848B900BF0798A04291
:10E7500004D000BF14A0F4F7B9FB00BF00BF5846B7
:10E7600090E700006E6574636F6E6E5F7772697418
:10E77000653A20696E76616C696420636F6E6E0025
:10E780006E6574636F6E6E5F77726974653A206947
:10E790006E76616C696420636F6E6E2D3E74797065
:10E7A00065000000E5B80008646F5F777269746502
:10E7B000206661696C656420746F20777269746586
:10E7C00020616C6C20627974657300002DE9F05F44
:10E7D00004460E4617469846DDE90AB900BF3CB923
:10E7E00000BF4AA0F4F772FB00BF0020BDE8F09F15
:10E7F00000BF00BFB9F1000F06D100BF4AA0F4F777
:10E8000065FB00BF0020F1E700BF06B94F4E07B916
:10E810004E4FB8F1000F01D1DFF830810020606069
:10E82000A060E0604A4860610020208584F83100E3
:10E830006062E061C4F820B04648007884F8340093
:10E840000C98206143463A463146204600F09CF938
:10E850002046C84708B10020C8E700BF94F834003C
:10E86000FF2802D1002084F834004FF0000A3A4813
:10E87000056821E000BFA54204D100BF37A0F4F72E
:10E8800025FB00BF00BF0AF1010A00BFBAF1FF0F6C
:10E8900004DD00BF36A0F4F719FB00BF00BF95F8F8
:10E8A000340094F83410884205D194F83400401CA8
:10E8B00084F8340002E02D68002DDBD100BF002D6C
:10E8C000CCD194F83400FE2803D1002021490870EF
:10E8D00004E094F83400401C1E4908701E4800688B
:10E8E00020601D48046000BF00BF00BF00BF00BF24
:10E8F00000BF00BF00BF00BF00BF00BF00BF00BF20
:10E9000000BF00BF00BF204670E700006E6574695D
:10E91000665F6164643A20696E76616C6964206E3A
:10E9200065746966000000006E657469665F616405
:10E93000643A204E6F20696E69742066756E637448
:10E94000696F6E20676976656E00000054DB010810
:10E9500081EB0008140200200C0200206E6574692F
:10E960006620616C7265616479206164646564002D
:10E97000746F6F206D616E79206E65746966732C9B
:10E98000206D61782E20737570706F7274656420CD
:10E990006E756D6265722069732032353500000036
:10E9A00070B504460D462946204604F0B1FD2946BF
:10E9B000204608F02BFE70BD10B503460868DC68E1
:10E9C000A04201D1012000E0002040B909B9002097
:10E9D00000E00868D86000BF00BF012010BD002023
:10E9E000FCE70000F8B505460C46164600BF24B902
:10E9F00000BF16A0F4F76AFA00BF00BF00BF26B937
:10EA000000BF12A0F4F762FA00BF00BF2068696877
:10EA1000884201D1012000E00020A0B920680090C8
:10EA20006868306000BF00BF69463046FFF7B8FF36
:10EA30000CB9002000E0206868600121284600F041
:10EA400067F80120F8BD0020FCE70000696E7661E0
:10EA50006C696420706F696E7465720010B503464E
:10EA600008689C68A04201D1012000E0002040B964
:10EA700009B9002000E00868986000BF00BF0120CD
:10EA800010BD0020FCE7000070B505460DB9002060
:10EA900070BDA81CF1F78CFCC6B226B9A878302846
:10EAA00001D00020F4E70E48046812E094F8340026
:10EAB000B0420DD1287894F83210884208D1697894
:10EAC0003320005D814203D100BF00BF2046DFE755
:10EAD0002468002CEAD100BF00BF0020D8E7000066
:10EAE0000C02002002466AB10748016808E091F86C
:10EAF0003400401CC0B2904201D1084670470968FA
:10EB00000029F4D10020F9E70C0200207047000032
:10EB100070B504460D4600BF24B900BF0FA0F4F73E
:10EB2000D5F900BF00BF94F8310000F0040020B117
:10EB300094F8310000F0010000B970BD05F001004B
:10EB400050B1606840B194F8310000F0080018B18D
:10EB5000211D2046F7F768F900BFEEE76E6574697E
:10EB6000665F69737375655F7265706F7274733A0F
:10EB700020696E76616C6964206E65746966000058
:10EB800003466FF00B0070472DE9F84F80460C46A6
:10EB900015461E464FF00009CA4604B9114C05B986
:10EBA000104D06B90F4E0CB1206808B9012000E0E5
:10EBB0000020074627B16A4621464046FFF712FF6C
:10EBC0004A4629464046FFF749FF524631464046ED
:10EBD000FFF7F2FE27B96A4621464046FFF702FFDB
:10EBE000BDE8F88F54DB01080249086000BF00BF90
:10EBF000704700001002002010B5044600BF2CB979
:10EC000000BF0EA0F4F762F900BF10BD00BF94F87A
:10EC1000310000F0010078B100BF94F8310000F03D
:10EC2000FE0084F8310000BF94F8310000F00800C5
:10EC300010B12046F6F7CAFB00BFE6E76E657469BF
:10EC4000665F7365745F646F776E3A20696E766194
:10EC50006C6964206E6574696600000000B1C16172
:10EC60007047000010B5044600BF2CB900BF0EA0CD
:10EC7000F4F72CF900BF10BD00BF94F8310000F08C
:10EC8000040070B100BF94F8310000F0FB0084F87C
:10EC9000310000BF00BFE06910B12046E16988473C
:10ECA00000BF00BFE7E700006E657469665F7365CB
:10ECB000745F6C696E6B5F646F776E3A20696E7615
:10ECC000616C6964206E65746966000010B5044665
:10ECD00000BF2CB900BF11A0F4F7F8F800BF10BDB9
:10ECE00000BF94F8310000F00400A8B900BF94F808
:10ECF000310040F0040084F8310000BF2046F5F7F1
:10ED00003FF803212046FFF703FF00BFE06910B181
:10ED10002046E169884700BF00BFE0E76E6574697F
:10ED2000665F7365745F6C696E6B5F75703A2069BE
:10ED30006E76616C6964206E65746966000000001F
:10ED400010B5044600BF2CB900BF0CA0F4F7BEF804
:10ED500000BF10BD00BF94F8310000F0010058B9A9
:10ED600000BF94F8310040F0010084F8310000BF8A
:10ED700003212046FFF7CCFE00BFEAE76E65746909
:10ED8000665F7365745F75703A20696E76616C6951
:10ED900064206E657469660070B504460D460022F5
:10EDA0002946204600F002F870BD00002DE9F0472A
:10EDB00004460D46904600BF24B900BF1CA0F4F7DE
:10EDC00085F800BF00BF14B1B5F5803F02D3012024
:10EDD000BDE8F0870DB90020FAE7AEB220893044D3
:10EDE00080B2B04201DA0120F2E794F80C9009F009
:10EDF000800048B16068471B04F1100087420BD2C5
:10EE000000BF00BF0120E3E7B8F1000F02D0606847
:10EE1000471B01E00120DBE700BF00BF676060899E
:10EE2000304460812089304420810020D0E70000F8
:10EE30007020213D204E554C4C0000002DE9FE4F26
:10EE400082460E469046574600BF00BFB8F1010FFC
:10EE50000AD0B8F1410F06D0B8F5C17F0BD0B8F594
:10EE6000207F7AD161E000BF42463146002000F0A9
:10EE7000FBF804469CE0002400200290B14600BF4D
:10EE80000D20FEF7A3FD054635B914B1204600F06C
:10EE9000ABFB0020BDE8FE8FF81C20F0030040F221
:10EEA000EC51081A80B2484501DD484606E0F81CDE
:10EEB00020F0030040F2EC51081A80B28346002093
:10EEC000CDE9008005F110003844C01C20F003019A
:10EED0005B464A46284600F05DFC00BF287900F0FA
:10EEE000030020B100BF35A0F3F7F0FF00BF00BF63
:10EEF00000BFF81C20F0030040F2EC51081A04D1C6
:10EF000000BF3AA0F3F7E2FF00BF00BF0CB92C46E8
:10EF100001E0029805600295A9EB0B001FFA80F949
:10EF20000027B9F1000FABDC42E0F81C20F0030130
:10EF3000F01C20F00300084485B205F110001FFA10
:10EF400080F9F01C20F00300A84204D8F01C20F047
:10EF50000300484502D900209CE720E04846FEF720
:10EF6000D1FA04460CB9002094E70020CDE90080D6
:10EF700004F110003844C01C20F00301334632462F
:10EF8000204600F007FC00BF207900F0030020B10C
:10EF900000BF23A0F3F79AFF00BF00BF08E000BF47
:10EFA00000BF2AA0F3F792FF00BF00BF002071E767
:10EFB00000BF00BF00BF20466CE7000070627566AE
:10EFC0005F616C6C6F633A207062756620712D3ED4
:10EFD0007061796C6F61642070726F7065726C79AA
:10EFE00020616C69676E6564000000005042554600
:10EFF0005F504F4F4C5F42554653495A45206D75FF
:10F000007374206265206269676765722074686145
:10F010006E204D454D5F414C49474E4D454E540085
:10F02000706275665F616C6C6F633A2070627566C2
:10F030002D3E7061796C6F61642070726F706572C3
:10F040006C7920616C69676E65640000706275663A
:10F050005F616C6C6F633A206572726F6E656F757D
:10F0600073207479706500002DE9FC4107460D4658
:10F07000144600BF412C06D0012C04D000BF0DA0C7
:10F08000F3F724FF00BF00BF0C20FEF79FFC0646ED
:10F0900026B900BF00BF0020BDE8FC8100202B4640
:10F0A0002A463946CDE90040304600F073FB304631
:10F0B000F2E70000696E76616C69642070627566C3
:10F0C0005F747970650000002DE9FC5F06460C4610
:10F0D00017469846DDE90C9BB24600BF00BF0AF117
:10F0E000030020F003002044584504D900BF00BFAE
:10F0F0000020BDE8FC9FB9F1000F06D00AF1030023
:10F1000020F0030000EB090500E000250220234663
:10F1100022462946CDE90070404600F03BFB4046C0
:10F12000E7E7000070B506460D4600BF06B12DB9F1
:10F1300000BF15A0F3F7CAFE00BF70BD00BF344684
:10F1400004E0208929890844208124682068002857
:10F15000F7D100BF20896189884204D000BF18A080
:10F16000F3F7B4FE00BF00BF00BF206820B100BFAE
:10F170001FA0F3F7ABFE00BF00BF20892989084418
:10F180002081256000BFD8E7286820213D204E550A
:10F190004C4C2920262620287420213D204E554CF9
:10F1A0004C29202870726F6772616D6D65722076D0
:10F1B000696F6C617465732041504929000000003B
:10F1C000702D3E746F745F6C656E203D3D20702D18
:10F1D0003E6C656E20286F66206C617374207062CF
:10F1E000756620696E20636861696E290000000001
:10F1F000702D3E6E657874203D3D204E554C4C0080
:10F2000070B505460C4621462846FFF78BFF204681
:10F2100000F05CFB00BF00BF70BD0146002002E0B3
:10F22000421C90B209680029FAD170472DE9F041DB
:10F2300080460E461446218932464046FFF7FEFDC1
:10F24000074617B90020BDE8F0812146384600F096
:10F2500015F8054600BF25B100BF03A0F3F736FE41
:10F2600000BF00BF3846EEE7706275665F636F707F
:10F2700079206661696C65640000000070B5054620
:10F280000C4600BF00BF00BF3CB900BF07A0F3F7AA
:10F290001DFE00BF6FF00F0070BD00BF228900236C
:10F2A0002146284600F07CF8F6E70000706275669B
:10F2B0005F636F70793A20696E76616C6964207360
:10F2C0006F757263650000002DE9F05F8046894626
:10F2D00016461D464FF0000AD34600BFB8F1000F96
:10F2E00007D100BF1DA0F3F7F1FD00BF0020BDE86E
:10F2F000F09F00BF00BFB9F1000F06D100BF1FA0F3
:10F30000F3F7E4FD00BF0020F1E700BF444620E032
:10F3100035B16089A84203DC6089281A85B217E0FC
:10F320006089401B87B2B74200DD374662685119D9
:10F3300009EB0A003A46F0F7F5FF0BEB07001FFA5E
:10F3400080FB0AEB07001FFA80FAF01B86B200254B
:10F3500024680EB1002CDBD15846C8E77062756690
:10F360005F636F70795F7061727469616C3A206974
:10F370006E76616C69642062756600007062756605
:10F380005F636F70795F7061727469616C3A206954
:10F390006E76616C696420646174617074720000DF
:10F3A0002DE9F05F04460D4616469A4657464FF043
:10F3B000000800BF00BF00BF15B12889B04208DABD
:10F3C00000BF4DA0F3F782FD00BF6FF00F00BDE856
:10F3D000F09F00BF00BF24B120890AEB06018842DC
:10F3E00007DA00BF51A0F3F771FD00BF6FF00F0007
:10F3F000EDE700BF00BF6089C01B6989A1EB080170
:10F40000884203D36889A0EB080B02E06089A0EB77
:10F41000070B5E4501D2304600E058461FFA80F9DE
:10F420006A6802EB08016268D0194A46F0F77AFF71
:10F430004F44C844A6EB090086B200BF6089B842B9
:10F4400004D200BF45A0F3F741FD00BF00BF00BFDD
:10F450006889404504D200BF46A0F3F737FD00BFDE
:10F4600000BF688940450ED84FF000082D6800BFE6
:10F4700045B93EB100BF46A0F3F728FD00BF6FF0CD
:10F480000F00A4E700BF6089B8420DD100272468AF
:10F4900000BF44B93EB100BF41A0F3F717FD00BF64
:10F4A0006FF00F0093E700BF7DB16889298988421A
:10F4B0000BD100BF286838B100BF3DA0F3F706FDAF
:10F4C00000BF6FF0050082E700BF7CB16089218931
:10F4D00088420BD100BF206838B100BF34A0F3F7D9
:10F4E000F5FC00BF6FF0050071E700BF002E82D170
:10F4F00000BF00BF00206AE7706275665F636F70CF
:10F50000795F7061727469616C5F706275663A20D0
:10F51000636F70795F6C656E2062696767657220E2
:10F520007468616E20736F757263650070627566D2
:10F530005F636F70795F7061727469616C5F706234
:10F5400075663A20746172676574206E6F7420620C
:10F55000696720656E6F7567680000006F66667387
:10F5600065745F746F203C3D20705F746F2D3E6C3E
:10F57000656E00006F66667365745F66726F6D20FE
:10F580003C3D20705F66726F6D2D3E6C656E0000B5
:10F59000705F66726F6D20213D204E554C4C00000F
:10F5A000705F746F20213D204E554C4C00000000D0
:10F5B000706275665F636F70795F706172746961A4
:10F5C0006C5F70627566282920646F6573206E6FAA
:10F5D0007420616C6C6F77207061636B657420714F
:10F5E00075657565732100002DE9F047044664B91F
:10F5F00000BF24B900BF33A0F3F768FC00BF00BF11
:10F6000000BF00BF0020BDE8F08700BF00BF00269C
:10F6100054E001F051FF824600BFA07B002804DCCB
:10F6200000BF2BA0F3F752FC00BF00BFA07B401E21
:10F6300000F0FF0884F80E80504601F09BFFB8F1FF
:10F64000000F37D1276800BF00BF207B00F00F05F7
:10F65000607B00F0020078B1A14600BFD9F810002D
:10F6600020B900BF20A0F3F731FC00BF00BF204647
:10F67000D9F81010884719E0022D04D121460D2039
:10F68000FEF756F912E0012D04D121460C20FEF7B9
:10F690004FF90BE01DB92046FDF7ECFD06E000BF79
:10F6A00000BF1AA0F3F712FC00BF00BF701CC6B267
:10F6B0003C4602E000BF00BF002400BF002CA8D1E0
:10F6C0003046A0E77020213D204E554C4C000000F4
:10F6D000706275665F667265653A20702D3E726570
:10F6E00066203E203000000070632D3E6375737409
:10F6F0006F6D5F667265655F66756E6374696F6E68
:10F7000020213D204E554C4C00000000696E766172
:10F710006C69642070627566207479706500000001
:10F720002DE9F041074688463C46454612E060898F
:10F73000A8420ADC26466089281A85B2246800207F
:10F7400030603046FFF750FF04E02946204600F0C5
:10F75000E1F800250DB1002CE9D12046BDE8F0818B
:10F7600070B504460D4601222946204600F001F8F6
:10F7700070BD70B505460C461646002C04DA614291
:10F78000284600F0C7F870BD324621462846FFF7EC
:10F790000DFBF8E770B5DDE9044500260660416021
:10F7A0000281438104734573012686730026C67364
:10F7B00070BDF8B506460F4615466A4639463046CE
:10F7C00000F0F0F8044644B16089BDF800108842AA
:10F7D00003DDBDF8001060684554F8BD2DE9F04127
:10F7E00006460F4600BF26B900BF25A0F3F76EFB03
:10F7F00000BF00BF3089B84201DCBDE8F08130892C
:10F80000C01B1FFA80F83D4634460FE06089281A75
:10F8100085B22089A0EB08002081246800BF24B9AC
:10F8200000BF1DA0F3F752FB00BF00BF6089A842D4
:10F83000ECDB207B00F00F00B0B96089A84213D048
:10F84000607B00F0020078B9A088001B284481B2D8
:10F850002046FDF77FFF044600BF24B900BF14A077
:10F86000F3F734FB00BF00BF658160892081206809
:10F8700010B12068FFF7B8FE0020206000BFBCE791
:10F88000706275665F7265616C6C6F633A207020A0
:10F89000213D204E554C4C00706275665F7265616B
:10F8A0006C6C6F633A207120213D204E554C4C000A
:10F8B0006D656D5F7472696D2072657475726E65C9
:10F8C000642071203D3D204E554C4C0070B50446DF
:10F8D000A4B100BF01F0F0FD0546A07B401CA07361
:10F8E000284601F047FE00BF00BFA07B002804DCD3
:10F8F00000BF03A0F3F7EAFA00BF00BF70BD00002D
:10F900007062756620726566206F766572666C6FD0
:10F91000770000002DE9F04104460D4600BF24B9F0
:10F9200000BF15A0F3F7D2FA00BF00BF14B1B5F5C0
:10F93000803F02D30120BDE8F0810DB90020FAE735
:10F94000AEB200BF6089B04206DA00BF0DA0F3F787
:10F95000BDFA00BF0120EEE700BF67686068284479
:10F9600060606089801B60812089801B208100BFCE
:10F9700000BF0020DFE700007020213D204E554CE5
:10F980004C000000696E6372656D656E745F6D6139
:10F99000676E6974756465203C3D20702D3E6C6512
:10F9A0006E0000002DE9F04104460D461646324631
:10F9B0002946204600F004F807463846BDE8F081A5
:10F9C00030B503460C462146184603E045894D1BD9
:10F9D000A9B2006810B145898D42F7DD02B11180EE
:10F9E00030BD00002DE9F0470446884616463746EC
:10F9F0004FF0000A00BF44B900BF2AA0F3F766FA2F
:10FA000000BF6FF00F00BDE8F08700BF00BFB8F186
:10FA1000000F07D100BF29A0F3F758FA00BF6FF01D
:10FA20000F00F0E700BF00BF2089B04207DA00BF37
:10FA300029A0F3F74BFA00BF4FF0FF30E3E700BF18
:10FA40002CB1B8F1000F02D02089B04202DA6FF079
:10FA50000F00D8E7254617E000BF25B900BF26A054
:10FA6000F3F734FA00BF00BFB9466889484501D2B0
:10FA7000B5F80A9008EB0A014A466868F0F752FCAC
:10FA8000A7EB0907CA442D68002FE5D100BF0FB9C5
:10FA9000B24504D000BF1EA0F3F718FA00BF00BFA4
:10FAA0000020B0E7706275665F74616B653A20692B
:10FAB0006E76616C696420627566000070627566BE
:10FAC0005F74616B653A20696E76616C696420646D
:10FAD0006174617074720000706275665F74616B4E
:10FAE000653A20627566206E6F74206C617267657E
:10FAF00020656E6F75676800706275665F74616B14
:10FB0000653A20696E76616C696420706275660082
:10FB1000646964206E6F7420636F707920616C6C0F
:10FB200020646174610000002DE9F84F8346884627
:10FB3000154699466A4649465846FFF733FF04463C
:10FB4000002C36D02089BDF800102944884230DBD3
:10FB50002F46C24600BF6089BDF80010884204DC11
:10FB600000BF15A0F3F7B2F900BF00BF6089BDF870
:10FB70000010401AA84204DA6089BDF80010401A4B
:10FB800000E0284686B2BDF8002061688818324639
:10FB90004146F0F7C7FBB81B87B2B244002F06DD21
:10FBA0003A4651462068FFF71DFFBDE8F88F002058
:10FBB000FBE74FF0FF30F8E7636865636B20706226
:10FBC00075665F736B697020726573756C74000085
:10FBD00070B50446002500BF2068406820B100BF12
:10FBE0001CA0F3F773F900BF00BF2068007800F095
:10FBF000F000102817D0202821D1284607F02CFD2E
:10FC0000216848602068406860B120680078222838
:10FC100003D1012021684968087422681549506899
:10FC200007F04EFD0EE0284603F0D2FC2168486044
:10FC30002068406810B1206801F0D6F902E0FA208F
:10FC4000207170BD00BF2068406808B9FF20207196
:10FC500000BFF6E77063625F6E65773A207063629B
:10FC600020616C726561647920616C6C6F63617492
:10FC700065640000350D01082DE9F041044600BF20
:10FC800033480068844204D200BF32A0F3F71EF963
:10FC900000BF00BF00BF35480068844204D300BFE6
:10FCA00033A0F3F713F900BF00BF00BF207920B1E4
:10FCB00000BF36A0F3F70AF900BF00BF00BF2088DD
:10FCC000B0F5C84F04D900BF37A0F3F7FFF800BF65
:10FCD00000BF208800F098FE0546AC4219D0287974
:10FCE000B8B922480068854213D03A480068A84253
:10FCF00001D138480460288820802888B0F5C84F92
:10FD000007D02046FDF71EFD0746288800F07CFE40
:10FD10004780608800F078FE0646A64215D030790C
:10FD200098B92C480068A04201D12A480660208872
:10FD300030802088B0F5C84F07D03046FDF702FD6F
:10FD40000746208800F060FE4780BDE8F081000093
:10FD5000C4010020706C75675F686F6C65733A2032
:10FD60006D656D203E3D2072616D0000C801002070
:10FD7000706C75675F686F6C65733A206D656D2098
:10FD80003C2072616D5F656E64000000706C756789
:10FD90005F686F6C65733A206D656D2D3E75736598
:10FDA00064203D3D20300000706C75675F686F6CAB
:10FDB00065733A206D656D2D3E6E657874203C3D0F
:10FDC000204D454D5F53495A455F414C49474E458B
:10FDD00044000000D001002070B505460E462C46B8
:10FDE00000BF24B900BF21A0F3F770F800BF00BF27
:10FDF0006078012804D101212046FBF7F1FD11E0D4
:10FE0000607804280ED1606A40B1606A407A28B1F7
:10FE1000606A407A401EC1B2606A41720121204688
:10FE2000FBF76AFA94F8200000F01000E0B1606877
:10FE3000D0B16068B0F8640041F65E71884213DDAD
:10FE40006068B0F866002C280EDA00BF94F8200035
:10FE500000F0EF0084F8200000BFA06A20B100226B
:10FE600002212046A36A9847002070BD636F6E6E22
:10FE700020213D204E554C4C000000002DE9F04162
:10FE800005460E462948076800202949096881F877
:10FE9000590027480068001D08F08CFE50B924481E
:10FEA000006890F82C10012088402249096881439D
:10FEB00020480160681CD8B9D6B11F4948681C4960
:10FEC000096888601A4982680968CA60184909681F
:10FED000091D8268516016490968091D8160164A2A
:10FEE000134909684A6111460968491C11601AE002
:10FEF0007C190F4800684460BC4207D20C48016876
:10FF0000091D0E48006808F079FE0CE008480168F9
:10FF1000091D0B48006808F071FE0A480068844219
:10FF200001D208480460BDE8F0810000C002002052
:10FF3000AC020020C4020020C8560120B4020020F8
:10FF4000B0020020DC02002010B5044608F07CFE60
:10FF500031480068401C304908603048006840B9AA
:10FF60002E4804600846006801280DD100F02EFAE2
:10FF70000AE02B48006838B928480068C06AE16A7E
:10FF8000884201D82548046026480068401C25495D
:10FF9000086008460068606494F82C1001208840CE
:10FFA00021490968084320490860E16A01EB8101A1
:10FFB0001E4A02EB81014868A0608268E260211D50
:10FFC000826851608160E16A01EB8101174A02EBAE
:10FFD00081026261E16A01EB8101144A52F8211049
:10FFE000491CE26A02EB8202104B43F8221008F02F
:10FFF00077FE0B48006868B108480068C06AE16A8B
:020000040801F1
:10000000884207D24FF0805009490860BFF34F8FF4
:10001000BFF36F8F10BD0000BC020020AC020020B7
:10002000C8020020D8020020C4020020F85301209A
:1000300004ED00E010B508F007FE10480068D0B9E4
:100040000F4808F0CBFD0F4808F0C8FD0C480E49DA
:1000500008600C480D49086000221021052009F0B5
:10006000EDFB064908600846006820B108A1034876
:10007000006808F04DFF08F033FE10BDF4020020C8
:10008000DC560120F0560120EC020020F002002096
:10009000546D72510000000010B516E008F0D4FD58
:1000A0000C48C068C468201D08F084FD0A48006838
:1000B000401E0949086009480068401E0749086059
:1000C00008F00EFE204600F05FF8044800680028A3
:1000D000E4D110BDB4560120BC020020B8020020BB
:1000E00070B504460D46206C70B1216CE068014487
:1000F000E160D4E90210884201D32168E16028461A
:10010000226CE168F0F70EF970BD2DE9F04104466C
:100110000F4615464FF00008A66B206C48B92068C2
:1001200000282CD1A0680AF091F980460020A06038
:1001300025E07DB93946226C6068F0F7F3F8216C50
:10014000606808446060D4E90101884217D32068E0
:10015000606014E03946226CE068F0F7E3F8216C47
:10016000E068411AE1602168E068884203D2216CAE
:10017000A068411AE160022D01D106B1761E701C03
:10018000A0634046BDE8F08110B50446206B08F03E
:10019000E7FD204608F0E4FD10BD01464A6A22B1A1
:1001A0000A6B1268C2F1200000E0002070470000D6
:1001B0000146084A126812680AB9012200E00022CA
:1001C0000A600A6822B9034A1268D268106800E01F
:1001D00000207047EC02002030B54FF40C43174864
:1001E00000F007042CB1C01D20F00700134C041BC5
:1001F0001B1B0246124C22600024114D6C60D0186B
:10020000083820F007000F4C206000240D4D2D68A9
:100210006C600C4D2D682C601146441A4C60094CE2
:1002200024680C60084D4C682C60084D4C682C60AC
:100230004FF00044064D2C6030BD000004570120F3
:100240000003002008030020100300200C030020FE
:100250001C03002000BFFFF71FFF064800680128AD
:10026000F9D94FF0805004490860BFF34F8FBFF3B6
:100270006F8FF0E7F853012004ED00E010B504465D
:1002800054B10020A06020600021E16000231A46E4
:100290001946204609F098FB10BD2DE9F0410646AD
:1002A0000D4617469846069C0DB9246000E027606D
:1002B000E66325640121204609F008FB84F850809C
:1002C0000020A064BDE8F0812DE9F05F82460F4672
:1002D00090469B460A9E0C9C4FEA8801A522206B03
:1002E000F0F740F8A8F10100216B01EB800929F03B
:1002F000070909F0070008B9012000E0002028B92B
:100300004FF4587224A12DA0F2F7E0FD87B100252B
:1003100007E0795D04F134004155785D00B902E0F1
:100320006D1C102DF5D300BF00214320015502E0C4
:10033000002084F83400202E01D2012000E00020AB
:1003400028B940F2973214A11CA0F2F7BFFD202E6D
:1003500000D31F26E662E66400202065201D08F019
:100360004AFC04F1180008F046FC2461C6F12000A4
:10037000A06164620020606584F8580084F8590028
:100380005A465146484600F021FC20600B9808B1BF
:100390000B980460BDE8F09F2E2E5C2E2E5C4D69FC
:1003A00064646C6577617265735C4672656552540E
:1003B0004F535C7461736B732E6300004572726FF0
:1003C000723A2025732C2025640D0A0010B50024F4
:1003D00007E004EB84010F4A02EB810008F0FEFB0A
:1003E000641C202CF5D30C4808F0F8FB0B4808F0EF
:1003F000F5FB0B4808F0F2FB0A4808F0EFFB0A484F
:1004000008F0ECFB04480949086004480849086002
:1004100010BD0000F8530120785601208C560120B1
:10042000A0560120B4560120C8560120B002002079
:10043000B402002010B50146164800E000680368C9
:100440008B42FBD30246436813448B4204D143687A
:100450004C682344436001460A464B6813440468D1
:10046000A34211D10C4C03682468A34208D04B6806
:100470000468646823444B6003681B680B6005E0F4
:10048000054B1B680B6001E003680B60884200D0DD
:10049000016010BD00030020080300202DE9F04199
:1004A00004460D4616461F464FF00008656024615D
:1004B000B5420CD8F01BA169884202D34FF0010865
:1004C00011E0211D0948006808F098FB0BE0BE42CE
:1004D00004D2BD4202D34FF0010804E0211D0448BC
:1004E000006808F08BFB4046BDE8F081F002002078
:1004F000EC02002070B5054608F0A6FBA86B08B911
:10050000012400E0002408F0EBFB204670BD70B52C
:10051000054608F099FBA86BE96B884201D10124DC
:1005200000E0002408F0DCFB204670BDF1B5009827
:10053000846C00262CB940F6D53220A128A0F2F711
:10054000C5FCA06BE16B884201D2012000E00020D5
:1005500028B940F6D63219A121A0F2F7B7FCA06B5A
:10056000E16B884227D294F9455000226946204623
:10057000FFF7CBFD0646681C60B9606A08B9012028
:1005800000E00020B0B904F124000AF05DF888B161
:1005900001260FE07F2D01D0012000E0002028B9C6
:1005A00040F6F63205A10EA0F2F790FC681C40B2AE
:1005B00084F8450000BF3046F8BD00002E2E5C2EAA
:1005C0002E5C4D6964646C6577617265735C46721C
:1005D000656552544F535C71756575652E630000F7
:1005E0004572726F723A2025732C2025640D0A0023
:1005F00070B505460E460E480068C068C468201DE8
:1006000008F0D8FA94F8280000F0040028B1324627
:100610002946204600F0FEF805E094F8280000F096
:10062000FE0084F828002046216A884770BD00003B
:10063000EC02002070B586B08AE0029800280CDA3F
:1006400003AE2EB940F2063247A150A0F2F73EFCAD
:10065000D6E90020B168904700BF0298002877DBF8
:10066000049C606908B9012000E0002010B9201D39
:1006700008F0A0FA01A800F0F9F8054602980A2847
:1006800064D2DFE800F06305072E365306082F37E3
:1006900000BF00BF00BF94F8280040F0010084F8BC
:1006A00028000398A269811803462A462046FFF7CE
:1006B000F5FEA8B194F8280000F0040038B10398C2
:1006C000A26981182A46204600F0A4F805E094F8B3
:1006D000280000F0FE0084F828002046216A8847A0
:1006E00035E000BF94F8280000F0FE0084F82800F0
:1006F0002DE000BF94F8280040F0010084F82800A5
:100700000398A061A06908B1012000E0002028B989
:1007100040F2593214A11DA0F2F7D8FBA06941198B
:100720002B462A462046FFF7B9FE10E094F8280031
:1007300000F0020018B9204608F012FB05E094F81A
:10074000280000F0FE0084F8280000E000BF00BF91
:10075000002202A91148006809F0F4FA00287FF489
:100760006CAF06B070BD00002E2E5C2E2E5C4D6965
:1007700064646C6577617265735C4672656552543A
:100780004F535C74696D6572732E63004572726FAE
:10079000723A2025732C2025640D0A00F4020020F3
:1007A000F8B505460C4608F0E1FE684600F05EF834
:1007B0000646009820BB44B9B54206D809F0EAFFC6
:1007C00031462846FFF714FF1CE03CB10E48006894
:1007D000006808B9012000E000200446A91B224659
:1007E0000A48006808F040FC09F0D4FF50B94FF007
:1007F000805007490860BFF34F8FBFF36F8F01E050
:1008000009F0C8FFF8BD0000F0020020F40200204B
:1008100004ED00E070B504460D46164604E0A069FC
:1008200005442046216A8847A06941192B46324673
:100830002046FFF733FE0028F1D170BD094800685B
:10084000006808B9012000E0002020B14FF0FF301F
:100850000549086005E003480068C068006802496F
:1008600008607047B0020020DC02002070B504462A
:1008700009F0F2FC054607480068854204D200F002
:100880000BF80120206001E0002020600148056095
:10089000284670BDFC02002070B508E00D480068D5
:1008A000C06804684FF0FF312046FFF7A1FE0948F9
:1008B0000068006808B9012000E000200028EDD0A1
:1008C0000448056804480068024908600248056059
:1008D00070BD0000EC020020F00200200B48006810
:1008E000401C08B9012000E0002020B9E92208A13D
:1008F00016A0F2F7EBFA00BF502080F31188BFF387
:100900004F8FBFF36F8F00BF00BFFEE720030020B3
:100910002E2E5C2E2E5C4D6964646C657761726569
:10092000735C4672656552544F535C706F727461AC
:10093000626C655C525644535C41524D5F434D348A
:10094000465C706F72742E63000000004572726F17
:10095000723A2025732C2025640D0A0008B500BFCB
:100960006846FFF725FC044620460099FFF718FF6C
:10097000FFF760FEF4E770B5044608F065F994F9F6
:10098000455019E0A06C30B12046FFF7CFFD88B18B
:1009900008F070FC0EE0606A08B9012000E0002059
:1009A00038B904F1240009F04FFE18B108F062FCD8
:1009B00000E003E0681E45B2002DE3DC00BFFF202D
:1009C00084F8450008F08CF908F03EF994F9445099
:1009D00010E0206908B9012000E0002048B904F1C6
:1009E000100009F031FE08B108F044FC681E45B261
:1009F00000E001E0002DECDC00BFFF2084F84400A3
:100A000008F06EF970BD0000014602480068084415
:100A100070470000C40100202DE9F04104464FF06A
:100A2000000808F0A3FD4948006808B9FFF7D4FBA7
:100A3000474800682040002875D1002C23D004F1DD
:100A40000800A0421FD9083404F0070000281BD07A
:100A500004F00700C0F108002044A04211D904F0BE
:100A60000700C0F10800044404F0070008B90120A1
:100A700000E0002040B99C2236A144A0F2F726FAFB
:100A800002E0002400E00024002C4CD04348006821
:100A9000844248D8424E3046056801E02E462D6813
:100AA0006868A04202D228680028F7D12748006869
:100AB000854238D0306800F10808286830606868DE
:100AC000001B102813D92F1907F0070008B90120BF
:100AD00000E0002020B9CF221EA12CA0F2F7F6F9E9
:100AE0006868001B78606C603846FFF7A3FC2B49F0
:100AF00068680968081A2949086008460068294991
:100B00000968884203D225480068264908601049D0
:100B10006868096808436860002028602248006807
:100B2000401C2149086009F035FE08F0070008B9AB
:100B3000012000E0002028B94FF4887205A113A01D
:100B4000F2F7C4F94046BDE8F08100000803002038
:100B50001C0300202E2E5C2E2E5C4D6964646C6597
:100B600077617265735C4672656552544F535C7071
:100B70006F727461626C655C4D656D4D616E675C32
:100B8000686561705F342E63000000004572726F0B
:100B9000723A2025732C2025640D0A000C030020D6
:100BA0000003002010030020140300200648006802
:100BB00030B10549096801F15000096D491C016017
:100BC0000148006870470000AC020020001F4FF091
:100BD00080730360001F21F001030360001F054BB9
:100BE000036014380260001F6FF0020303602038B6
:100BF00070470000DD0801080146086870470000E2
:100C00002DE9F04706460F4615469A4600BF27B91C
:100C100000BF28A0F2F75AF900BF00BF00BF26B9F5
:100C200000BF2DA0F2F752F900BF00BF00BFBAF11C
:100C3000000F04D000BF30A0F2F748F900BF00BF9A
:100C400034461CB96FF00500BDE8F08700BF60684E
:100C5000B84204D000BF2EA0F2F738F900BF00BFA1
:100C600004F1100008B1206948B935B12989384626
:100C700004F086FA2846FEF7B7FC0020E4E71DB131
:100C8000A846B5F8089003E0DFF8A4804FF000090B
:100C9000414604F1100000F0F9FC10B14FF0FF30B4
:100CA000D2E7A06A20B14A4600212046A36A9847AD
:100CB0000020C9E7726563765F746370206D757399
:100CC00074206861766520612070636220617267BC
:100CD000756D656E74000000726563765F74637095
:100CE000206D757374206861766520616E20617275
:100CF00067756D656E74000065727220213D204538
:100D000052525F4F4B20756E68616E646C65640073
:100D1000726563765F7463703A20726563762066ED
:100D20006F722077726F6E6720706362210000001F
:100D300072D901082DE9F05F0746884616469946A4
:100D4000DDF828B000BFB8F1000F04D100BF28A023
:100D5000F2F7BCF800BF00BF00BF27B900BF2DA04D
:100D6000F2F7B4F800BF00BF3C4624B93046FEF7A6
:100D70003BFCBDE8F09F00BF6068404504D000BF69
:100D80002CA0F2F7A3F800BF00BF04F1100008B1D7
:100D9000206918B93046FEF727FCEAE70620FCF781
:100DA00015FE05461DB93046FEF71EFCE1E72E6034
:100DB0006E60B9F1000F01D1002001E0D9F8000008
:100DC000A860A5F80CB0B6F808A0294604F11000F8
:100DD00000F05CFC18B12846FCF712FFC9E7A06AD6
:100DE00020B1524600212046A36A984700BFC0E7C1
:100DF000726563765F756470206D757374206861C9
:100E0000766520612070636220617267756D656E22
:100E100074000000726563765F756470206D757391
:100E200074206861766520616E20617267756D65FA
:100E30006E740000726563765F7564703A20726547
:100E4000637620666F722077726F6E6720706362C0
:100E5000210000002DE9F84304460E461746984647
:100E60003D48056873E0E86900286FD181466869EC
:100E700048B13B46324621462846CDF80080FBF774
:100E800031FA814658E0CEB1A968B9B121460429AA
:100E900010DA214600290DD42046C11700EB51710C
:100EA000C910AA68515C224602F0070301229A4049
:100EB000114000E0002109B14FF00109E7B1B9F19B
:100EC000000F19D1E968B9B12146042910DA214689
:100ED00000290DD42046C11700EB5171C910EA68F2
:100EE000515C224602F0070301229A40114000E0C3
:100EF000002109B14FF00109B8F1000F1CD0B9F180
:100F0000000F19D12969B9B12146042910DA214607
:100F100000290DD42046C11700EB5171C9102A6970
:100F2000515C224602F0070301229A40114000E082
:100F3000002109B14FF00109B9F1000F05D00120DE
:100F4000E86105F1200000F019FD00BF2D68002DBB
:100F500089D1BDE8F8830000A40100202DE9F0410B
:100F600005460F4616462C4600BF24B900BF1AA0FE
:100F7000F1F7ACFF00BF00BF5CB36078012804D17B
:100F800001212046FAF72CFD06E06078042803D101
:100F900001212046FAF7B0F96068D0B16068B0F876
:100FA000640041F65E71884213DD6068B0F8660047
:100FB0002C280EDA00BF94F8200000F0EF0084F82F
:100FC000200000BFA06A20B1324602212046A36A59
:100FD00098470020BDE8F081636F6E6E20213D20B0
:100FE0004E554C4C0000000070B504466568214623
:100FF000284600F0C9FF0949284604F06BF8084963
:10100000284604F0D1FB02220649284603F0ACF83A
:101010000549284601F014FB70BD0000010C0108D1
:101020005D0F0108D9FD00082152000800B58DB000
:1010300000BF00BF002000907148006840F04000F1
:101040006F4908600846006800F04000009000BF4B
:1010500000BF00BF00BF00BF00200090084600682E
:1010600040F0080008600846006800F008000090A2
:1010700000BF00BF00BF00BF00BF002000900846B7
:10108000006840F0080008600846006800F00800AA
:10109000009000BF00BF00BF00BF00200090584874
:1010A0000830006840F001005549083108600846E2
:1010B000006800F00100009000BF00BF00BF0020EA
:1010C00000904F48006840F008004D49086008460D
:1010D000006800F00800009000BF00BF00BF0020C3
:1010E00000900846006840F010000860084600685C
:1010F00000F01000009000BF00BF00BF0020009073
:101100000846006840F0200008600846006800F0CB
:101110002000009000BF00BF00BF002000900846E4
:10112000006840F0400008600846006800F0400099
:10113000009000BF00BF0815089002200990012010
:101140000A9002200B900C200C9008A92D48F0F773
:101150001FFB2020089008A92B48F0F719FB10204E
:10116000089008A92848F0F713FB4FF60370089081
:101170000220099001200A9002200B9008A9224821
:10118000F0F706FB4FF68370089008A91F48F0F7A8
:10119000FFFA4FF23F00089008A91D48F0F7F8FA4F
:1011A0003F20089008A91748F0F7F2FA4FF02040C6
:1011B00018490860184848600420886000211548D4
:1011C000C16001611021416100218161C161416201
:1011D0004FF4805181620021C162016341638163E8
:1011E00000200190029006200390002004900790B8
:1011F00001AA01A90748F1F72BF80DB000BD0000C6
:101200003038024000180240000C0240001002403A
:1012100000140240A0040020040100A03EB50446D2
:1012200000BF3848384988610120FBF709FF31E0E9
:101230004FF4784035A110221346CDE900210290E9
:10124000C8226E211E20F9F7BBFB4FF4FA70F2F7AB
:101250003BF94FF6FF704223E622322100901E2018
:10126000F8F720FF4FF478402DA110221346CDE966
:1012700000210290C8226E211E20F9F7A1FB4FF435
:10128000FA70F2F721F900BF4FF480612948F0F7B6
:1012900081FB00BFF9F700FE0028C9D102E0264813
:1012A000F1F714FE1120F5F723F80028F7D002E03B
:1012B000052007F0FFFE1448807D022803D0124865
:1012C000807DFF28F4D107F0BFFC1C480B210023D0
:1012D0004FF48062CDE9001019A11D4808F076FF97
:1012E0001C480A2100238022CDE900101AA11D48C4
:1012F00008F06CFF1C48006807F01EFF07F0F0FCC8
:101300003EBD000041D00008644F01206C77495079
:1013100020496E6974206661696C65642121000052
:101320005265747279696E672E2E2E20202020203F
:101330002020000000140240F0DB0108080000201B
:101340006C7769705F64656D6F5F7461736B0000CB
:1013500099B000080C0000206C65645F7461736BC9
:10136000000000007DAB0008040000202DE9F843D8
:1013700005460E46174600BF25B900BF1CA0F1F771
:10138000A5FD00BF00BF00BF286820B900BF1CA09A
:10139000F1F79CFD00BF00BF06B96E467FB94FF064
:1013A000FF323146286808F0CDFC044600BF012C0E
:1013B00004D000BF17A0F1F789FD00BF16E0B846C2
:1013C00042463146286808F0BDFC044624B9002096
:1013D0003060401EBDE8F88300BF012C04D000BF80
:1013E0000CA0F1F773FD00BF00BF00BF0120F1E7C3
:1013F0006D626F7820213D204E554C4C000000005E
:101400006D626F782D3E6D627820213D204E554CE7
:101410004C0000006D626F7820666574636820661A
:1014200061696C6564000000F8B504460E4600BFB3
:1014300024B900BF12A0F1F749FD00BF00BF00BFF3
:10144000206820B900BF12A0F1F740FD00BF00BF27
:1014500006B96E4600223146206808F073FC054646
:101460001DB900203060401EF8BD00BF012D04D022
:1014700000BF0CA0F1F72AFD00BF00BF0120F3E779
:101480006D626F7820213D204E554C4C00000000CD
:101490006D626F782D3E6D627820213D204E554C57
:1014A0004C0000006D626F7820666574636820668A
:1014B00061696C656400000010B507F0C5FB012090
:1014C00010BD00002DE9F04105460E4600BF25B9CC
:1014D00000BF1AA0F1F7FAFC00BF00BF00BF2868E8
:1014E00020B900BF18A0F1F7F1FC00BF00BF76B92A
:1014F0004FF0FF31286808F0E5FC044600BF012CDE
:1015000004D000BF15A0F1F7E1FC00BF14E037469E
:101510003946286808F0D6FC04461CB94FF0FF3065
:10152000BDE8F08100BF012C04D000BF0BA0F1F793
:10153000CDFC00BF00BF00BF0120F1E773656D2047
:10154000213D204E554C4C0073656D2D3E73656DED
:1015500020213D204E554C4C0000000074616B6909
:101560006E672073656D6170686F72652066616972
:101570006C65640010B5044607F0B2FB10BD0000B6
:101580002DE9F04100F06CF9074600BF0F480468F0
:101590000CB9BDE8F0816068381AB0F1004F01D392
:1015A000012000E0002000B1F3E70849206808604E
:1015B000A568E66806496068086021460A20FCF7CD
:1015C000B7F90DB13046A847E0E7000060020020FF
:1015D000640200207047000010B5044600BF24B923
:1015E00000BF09A0F1F772FC00BF00BF00BF206878
:1015F00020B900BF08A0F1F769FC00BF00BF206858
:1016000007F0CCFC10BD00006D626F7820213D20FA
:101610004E554C4C000000006D626F782D3E6D629F
:101620007820213D204E554C4C00000070B50446FA
:101630000D4600BF24B900BF0DA0F1F747FC00BF65
:1016400000BF00BF002D04DC00BF0DA0F1F73EFC81
:1016500000BF00BF00220421284608F0EFF82060F8
:10166000206810B94FF0FF3070BD0020FCE700008B
:101670006D626F7820213D204E554C4C00000000DB
:1016800073697A65203E20300000000073B504467F
:1016900000BF24B900BF12A0F1F718FC00BF00BFC3
:1016A00000BF206820B900BF11A0F1F70FFC00BFF8
:1016B00000BF00231A4601A9206808F085F90546F5
:1016C000012D01D100207CBD00BF25B100BF0DA0C0
:1016D000F1F7FCFB00BF00BF4FF0FF30F3E7000065
:1016E0006D626F7820213D204E554C4C000000006B
:1016F0006D626F782D3E6D627820213D204E554CF5
:101700004C0000006D626F7820747279706F737492
:10171000206661696C65640070B5044600BF24B939
:1017200000BF0FA0F1F7D2FB00BF00BF00BF2068D1
:1017300020B900BF0EA0F1F7C9FB00BF00BF4FF0FA
:10174000FF31206808F0A0FC054600BF012D04D041
:1017500000BF0CA0F1F7BAFB00BF00BF70BD0000D6
:101760006D7574657820213D204E554C4C0000006D
:101770006D757465782D3E6D757420213D204E5534
:101780004C4C00006661696C656420746F20746164
:101790006B6520746865206D7574657800000000C5
:1017A00010B5044600BF24B900BF08A0F1F78EFBB6
:1017B00000BF00BF042008F02FF82060206810B997
:1017C0004FF0FF3010BD0020FCE700006D75746520
:1017D0007820213D204E554C4C00000070B5044649
:1017E00000BF24B900BF0EA0F1F770FB00BF00BF1F
:1017F00000BF206820B900BF0DA0F1F767FB00BF54
:1018000000BF206808F064FA054600BF012D04D02F
:1018100000BF0CA0F1F75AFB00BF00BF70BD000075
:101820006D7574657820213D204E554C4C000000AC
:101830006D757465782D3E6D757420213D204E5573
:101840004C4C00006661696C656420746F206769A8
:10185000766520746865206D7574657800000000F9
:1018600010B508F0F9FC10BD10B5044600BF24B94E
:1018700000BF0AA0F1F72AFB00BF00BF00BF20682D
:1018800020B900BF08A0F1F721FB00BF00BF20680E
:1018900007F084FB0020206010BD000073656D2000
:1018A000213D204E554C4C0073656D2D3E73656D8A
:1018B00020213D204E554C4C0000000070B50446E0
:1018C0000D4600BF24B900BF17A0F1F7FFFA00BF13
:1018D00000BF00BF35B1012D04D000BF15A0F1F746
:1018E000F5FA00BF00BF03220021012007F0A6FF88
:1018F0002060206810B94FF0FF3070BD012D10D16D
:1019000000231A461946206808F05EF8064600BF14
:10191000012E04D000BF10A0F1F7D8FA00BF00BF1D
:1019200000BF0020E9E7000073656D20213D204ED7
:10193000554C4C00696E697469616C5F636F756EBC
:101940007420696E76616C696420286E6F74203033
:10195000206F7220312900007379735F73656D5FAA
:101960006E65773A20696E697469616C2067697683
:1019700065206661696C65640000000070B504460E
:1019800000BF24B900BF10A0F1F7A0FA00BF00BF4C
:1019900000BF206820B900BF0EA0F1F797FA00BF82
:1019A00000BF00231A461946206808F00DF80546C6
:1019B00000BF012D05D025B100BF0BA0F1F786FABD
:1019C00000BF00BF70BD000073656D20213D204E3B
:1019D000554C4C0073656D2D3E73656D20213D2087
:1019E0004E554C4C000000007379735F73656D5F5A
:1019F0007369676E616C3A2073616E6520726574FD
:101A000075726E2076616C75650000002DE9F041FD
:101A100092B080460C4615461E46002700BF0020A7
:101A200000902A48006840F0805028490860084625
:101A3000006800F08050009000BF00BF00BF002091
:101A400000902348006840F480402149086008461F
:101A5000006800F48040009000BF00BF01200190AA
:101A6000000402900220079041050891CDF82880DB
:101A700009940B950C9601A8F0F79CF907461FB145
:101A8000012012B0BDE8F0810F200D9002200E90D1
:101A900000200F904FF4A05010904FF48050119000
:101AA00004210DA8F0F746F807460FB10120E8E73A
:101AB000EFF780FF41F20101884205D10548006837
:101AC00040F48070034908600020DAE740380240A3
:101AD00000700040003C02402DE9FF4706460F46DB
:101AE00090461C46DDF830A000BF002C04DC00BF8F
:101AF0000FA0F1F7EBF900BF00BFA14603A81FFA42
:101B000089F243463146CDE900A0384608F05EFB35
:101B1000054600BF012D04D000BF0AA0F1F7D6F999
:101B200000BF00BF03980290029804B0BDE8F087A0
:101B3000696E76616C696420737461636B73697A32
:101B4000650000007461736B206372656174696F76
:101B50006E206661696C6564000000002DE9F0414B
:101B600004460E46174600BFB4F1804F04D300BFB1
:101B700007A0F1F7ABF900BF00BFFFF771FE051931
:101B80003A463146284600F01FF8BDE8F0810000D3
:101B900054696D656F75742074696D6520746F6F1D
:101BA000206C6F6E672C206D6178206973204C5714
:101BB00049505F55494E5433325F4D41582F3420C0
:101BC0006D736563730000002DE9F04106460F4612
:101BD00090460A20FBF7FAFE04464CB900BF24B930
:101BE00000BF1FA0F1F772F900BF00BFBDE8F08190
:101BF00000202060A760C4F80C8066602848006858
